:020000022000DC
:1060000000000120756302005D6302005F6302000F
:106010006163020063630200656302000000000028
:1060200000000000000000000000000067630200A4
:1060300069630200000000006B6302006D630200F0
:1060400025C302006F630200BDC80200C1EE02005A
:106050006F6302006F630200B9C702006F63020042
:106060006F6302006F630200690103006F63020047
:106070006F6302006F6302006F6302006F630200D0
:106080006F630200CD7F02006F6302006F63020046
:106090006F6302006F6302007D3B03006F630200C9
:1060A0006F6302006F6302006F6302006F630200A0
:1060B0006F6302006F630200000000000000000038
:1060C0006F6302006F6302006F6302006F63020080
:1060D0006F6302006F6302006F6302000000000044
:1060E00000000000000000000000000000000000B0
:1060F00000000000000000000000000000000000A0
:10610000000000000000000000000000000000008F
:10611000000000000000000000000000000000007F
:10612000000000000000000000000000000000006F
:10613000000000000000000000000000000000005F
:10614000000000000000000000000000000000004F
:10615000000000000000000000000000000000003F
:10616000000000000000000000000000000000002F
:10617000000000000000000000000000000000001F
:10618000000000000000000000000000000000000F
:1061900000000000000000000000000000000000FF
:1061A00000000000000000000000000000000000EF
:1061B00000000000000000000000000000000000DF
:1061C00000000000000000000000000000000000CF
:1061D00000000000000000000000000000000000BF
:1061E00000000000000000000000000000000000AF
:1061F000000000000000000000000000000000009F
:10620000354936480A1A02D0072291438D4634494F
:1062100034480A1A06D00722914381F309880222E2
:1062200082F3148830483149314A00F044F831484B
:106230003149324A00F03FF831483249324A00F0E1
:106240003AF832483249334A00F035F83248334997
:10625000334A00F030F833483349344A00F02BF821
:1062600033483449344A00F026F83448344900228F
:1062700000F02CF833483449002200F027F8334866
:106280003349091A082902DB002202604160314AC1
:1062900090471F481F49884205D00268043003B464
:1062A000904703BCF7E700208646EC46002000211B
:1062B000294A9047FEE7884207D0521A05D0037852
:1062C00001300B700131013AF9D17047884202D098
:1062D00002700130FAE770470000012000E0002062
:1062E0000000012000000120808F0300D82A002038
:1062F000A42B0020D0630200D0630200D8720300F8
:10630000808F0300D82A0020D82A0020F4730300CD
:10631000F4730300F4730300F4730300F4730300D5
:10632000F4730300F4730300F47303007F8F03001E
:106330004C900300A42B0020A42B0020A42B0020B1
:10634000DCB50020DCB50020DCB50020DCB5002089
:10635000DCD500209D63020095060300FEE7FEE702
:10636000FEE7FEE7FEE7FEE7FEE7FEE7FEE7FEE705
:1063700000F002B8FFF7FCBF0F484FF00701884359
:1063800085460E4880470E48016841F4700101605F
:10639000BFF34F8FBFF36F8FFFF732BF09480A4932
:1063A0000A4A884207D0521A05D0037801300B7090
:1063B0000131013AF9D170470000012005B6020011
:1063C00088ED00E0F4730300D82A0020D82A0020CA
:1063D00000B585B00190019B002B0AD0074B43F01C
:1063E00001030393019B9B010293039B029898472F
:1063F00000E000BF05B05DF804FB00BF00740300BF
:1064000000B583B00190019B002B0AD04FF47A7045
:10641000FFF7DEFF019B013B0193019B002BF5D1B0
:1064200000E000BF03B05DF804FB08B50AF0D2FA43
:1064300000BF08BD00B589B0039002910192019B95
:10644000002B33D00023079303230693029A079B64
:106450001344019A194600200AF06CFA0590079A35
:10646000059B13440793019A059BD31A0193059B3F
:10647000002B13D10F4B1B7883F00103DBB2002BF1
:1064800013D10120FFF7BCFF069B013B0693069B3F
:10649000002B03D1074B00221A7007E0054B0122A5
:1064A0001A70019B002BD1D100E000BF00BF09B0E2
:1064B0005DF804FBA42B002000B585B00390029189
:1064C000054B00934023054A0299039800F012F807
:1064D00000BF05B05DF804FB35640200A82B002066
:1064E00082B0019000BF02B0704782B0019000BF3F
:1064F00002B0704700B5A1B00590049103920293D9
:10650000049802F057FC039B1593029B16930023FB
:10651000179300238DF8603000231993229B1A9360
:1065200000231F930FA91F9B0822049802F01CFD53
:1065300008231F93119B1293BDF84030ADF84C30E7
:10654000BDF84230ADF84E3000238DF851309DF843
:106550003C3003F00303DBB2012B26D10F9BC3F3C6
:1065600095231C939DF83C30C3F3C203DBB28DF836
:106570005030BDF83C30C3F38313DBB21B931B9B3D
:106580009A0009A91F9B049802F0EEFC1B9B9B003C
:106590001F9A13441F9312AA09A915AB009313461F
:1065A0001B9A1C9800F0DEFE2FE09DF83C3003F0B3
:1065B0000303DBB2022B28D1BDF83E30C3F38913AD
:1065C0009BB21E939DF83C30C3F3C203DBB28DF83F
:1065D00050301E9B082B28BF08231D9307A91F9B23
:1065E0001D9A049802F0C0FC1F9A1D9B13441F9330
:1065F0001E9A1D9BD31A1E9315AB12AA07A81D99AC
:1066000000F052FF1E9B002BE3D1049802F0E1FB47
:1066100000BF21B05DF804FB82B00190019BDB68F4
:1066200001225A7100BF02B07047000000B583B06C
:106630004FF0FF330193FFF7F8FE0421114800F0FB
:10664000ADFD0190019B002B03DA0F49412001F0C1
:10665000CBFC0C48FFF7E0FF01F042F804210B48A7
:1066600000F09CFD0190019B002B03DA06494820B5
:1066700001F0BAFC0548FFF7CFFF00BF03B05DF89B
:1066800004FB00BFD47303002C740300E473030005
:1066900000B583B001900091019B1B681B680099B5
:1066A0000198984700BF03B05DF804FB00B583B0C4
:1066B0000190019B1B685B680198984700BF03B07D
:1066C0005DF804FB00B583B00190019B1B689B68DB
:1066D0000198984700BF03B05DF804FB82B00190B9
:1066E0000B468DF80330019BDB689DF803201A717F
:1066F00000BF02B0704782B00190019BDB681B793C
:10670000184602B0704782B00190019BDB680122FD
:106710005A7100BF02B0704782B00190019BDB68E4
:106720005B79184602B0704700B585B001900091C2
:106730000C4B01221A700C4802F0A0FA0390039B44
:10674000002B01D0039B08E0084802F059FC084ADE
:10675000084BD31ADB0802930023184605B05DF8F6
:1067600004FB00BF502D0020387303007474030035
:10677000D47303004C730300024A034BD31ADB08A3
:1067800018467047D47303004C73030000B587B0FC
:1067900001900B468DF803309DF80330002B1FD07D
:1067A000FFF7EAFF04900023059313E0059B9B008D
:1067B0000E4A13440393039B1B881A46019B1B68D4
:1067C0009A4204D1019B059A1A60002309E0059BB7
:1067D00001330593059A049B9A42E7D3052300E011
:1067E0000023184607B05DF804FB00BFD82A00203C
:1067F00000B585B001900B468DF803309DF803205D
:1068000001AB11461846FFF7C1FF0346002B07D125
:10681000019BDB00054A13440393039B1B6800E0C4
:106820000023184605B05DF804FB00BF4C7303005D
:1068300084B001900B468DF80330019BDB00174AB2
:10684000134402939DF80330013B032B1CD801A293
:1068500052F823F0656802006D6802007568020056
:106860007F68020002238DF80F3011E004238DF8B9
:106870000F300DE0029B1B798DF80F3008E0029B72
:106880005B798DF80F3003E000238DF80F3000BFE7
:106890009DF80F30184604B0704700BF4C730300DA
:1068A00084B00190009100238DF80F30019B1B787C
:1068B00003F00403DBB2002B24D0019B1B78C3F34D
:1068C0000103DBB2012B02D0022B0CD017E0009B9E
:1068D0001B68019A1288C2F38312D2B213449A1C25
:1068E000009B1A600BE0009B1B68019A5288C2F360
:1068F000891292B213449A1C009B1A6000BF0123B4
:106900008DF80F309DF80F30184604B07047000026
:1069100000B58BB00023ADF826303E4801F0B9FC3D
:106920003D4801F0B6FC3D4B9B6804933C4B1B6813
:106930000693049A069B134002339B00374A134484
:106940000433089304AB19460898FFF7A9FF0346E0
:10695000002B09D0049A069B134002339B002F4A58
:10696000134404330893EDE700BF0023079311E0BD
:10697000049B5A1C0492069A1340079A920001A99C
:106980000A44264902339B000B445B681360079B53
:1069900001330793079B012BEAD99DF80430C3F319
:1069A0000103DBB2012B10D0022B1CD1BDF80A3041
:1069B000ADF82630BDF80630C3F389139BB203331C
:1069C0009A08049B1344049313E0BDF80A30ADF811
:1069D0002630BDF80430C3F38313DBB21A46049BA0
:1069E0001344049305E00F494FF4C27001F0FCFA20
:1069F00000BF094801F059FC0590059B002B02D00F
:106A0000049B064A9360BDF8263018460BB05DF82B
:106A100004FB00BF6831002064310020502D0020AD
:106A2000E82A00208474030000B585B000210748DF
:106A300001F0A0FB0390039B0293029B83F31003DE
:106A40000193019B184605B05DF804FB6C310020F2
:106A500000B589B00390029101920093039B1B0C37
:106A60000793FFF7E1FF0690FFF786FE0246079BBC
:106A7000934204D3214940F2A91001F0B5FA069BD4
:106A80001904009B5A1C0A9B1340079A0A431C498D
:106A900002339B000B445A60009A0A9B1340023356
:106AA0009B00174A134404330593039B03F0070329
:106AB000D9B2059A137861F3C5031370019B03F0F3
:106AC0000F03D9B2059A138861F389131380029BCF
:106AD000C3F31501059A136861F39F231360059AA8
:106AE0001378012161F301031370059A13786FF392
:106AF0008203137000BF09B05DF804FB84740300C7
:106B0000502D002000B58DB00390029113468DF8F2
:106B10000730039B02330A9301238DF827300023AB
:106B20008DF81B300DF11B03184601F0C3F9404BE3
:106B30005A68029B1A603F4B1A683D4B99683C4B60
:106B40005B68CB1A134401330B9314E001213A48DC
:106B500001F06FFBFFF7DCFE07900799364801F064
:106B600068FB344B1A68324B9968314B5B68CB1A1F
:106B7000134401330B930A9A0B9B9A42E6D89DF873
:106B80002730002B48D0002305939DF80730002BB9
:106B900017D09DF81430012262F301038DF81430F0
:106BA0009DF8143043F004038DF81430039B03F078
:106BB0000F03DAB2BDF8143062F38913ADF8143064
:106BC00016E09DF81430022262F301038DF81430B0
:106BD0009DF8143043F004038DF81430039BC3F385
:106BE00009039AB2BDF8163062F38F13ADF8163070
:106BF0000F4B5A680F4B1B68134002339B000C4A23
:106C0000134404330893059A089B1A60084B5A688A
:106C10000A9B1344064A53609DF81B30184601F046
:106C20005FF99DF8273018460DB05DF804FB00BFF2
:106C3000502D0020E82A00206C31002000B58BB0D8
:106C400005900491039202931F4B1B68079306ABB8
:106C5000012219460298FFF755FF0346002B24D066
:106C6000069B023309930023089311E0089B9B00C5
:106C7000039A1A44099B591C099107990B40126801
:106C8000124902339B000B445A60089B013308935E
:106C9000089A029B9A42E9D3069A079B00931346EF
:106CA000029A04990598FFF7D3FE084B1B78002B36
:106CB00005D000BF00F068F80346002BFAD100BFF2
:106CC0000BB05DF804FB00BFE82A0020502D002027
:106CD00000B583B001900091002300220099019833
:106CE000FFF7ACFF00BF03B05DF804FB00B587B051
:106CF000039002910192019B059305AA0123029939
:106D00000398FFF79BFF00BF07B05DF804FB00B5D9
:106D100087B00390029101920093019B0493009B22
:106D2000059304AA022302990398FFF787FF00BF87
:106D300007B05DF804FB00B58BB00390029101929F
:106D40000093019B0593009B06930C9B07930D9B5F
:106D500008930E9B099305AA052302990398FFF750
:106D60006DFF00BF0BB05DF804FB0000054B9A6897
:106D7000044B5B689A420CBF01230023DBB2184628
:106D8000704700BF502D002000B599B0FFF7EEFF0F
:106D90000346002B01D00023C0E19B4B0022C3F827
:106DA0001824BFF34F8F00BF974B9B680493974BFA
:106DB0001B681093049A109B134002339B00924A65
:106DC00013440433119300231793002316930023D5
:106DD0000F9304AB19461198FFF762FD0346002B91
:106DE00019D0894BD3F81834002B14D1864B5A682C
:106DF000049B9A4205D8844B5B68834A93600023C6
:106E00008CE1049A109B134002339B007E4A13448A
:106E100004331193DDE70023159311E0049B5A1C02
:106E20000492109A1340159A920001A90A447649D7
:106E300002339B000B445B681360159B0133159371
:106E4000159B012BEAD99DF8043003F00303DBB254
:106E5000022B40F09C80BDF80630C3F389139BB22F
:106E60000D93BDF80630C3F389139BB2502B28BF96
:106E700050239BB20C930C9BC3F309039AB2BDF849
:106E8000063062F38F13ADF806300C9B08330B937A
:106E90009DF80430C3F3C203DBB20F930B995C4837
:106EA00001F0F7FE1790179B002B00F0D380179886
:106EB00001F080FF01A9169B0822179802F036F80E
:106EC000169B08331693049BDA43109B134001333F
:106ED0009B000A930C9A0A9B9A4242D90A9B002B68
:106EE00008D0049A109B134002339B00464A134477
:106EF000043300E0474B08930A9B002B02D00A9B07
:106F0000DBB201E00C9BDBB28DF81F300A9B002B3B
:106F100001D0404B00E0002306930A9B002B06D0D3
:106F20000C9BDAB20A9BDBB2D31ADBB200E000237F
:106F30008DF817309DF81F20169B0899179801F0BF
:106F4000F5FF9DF81F30169A13441693069B002BED
:106F500016D09DF81720169B0699179801F0E6FFAA
:106F60000EE0049A109B134002339B00264A134400
:106F700004330993169B0C9A0999179801F0D6FFD0
:106F80000D9B03339A08049B1344049362E09DF81D
:106F9000043003F00303DBB2012B5BD1BDF80430F6
:106FA000C3F38313DBB2062B28BF0623DAB2BDF886
:106FB000043062F38913ADF80430BDF80430C3F334
:106FC0008313DBB202330E939DF80430C3F3C20384
:106FD000DBB20F930E9B9B0019460D4801F059FE42
:106FE0001790179B002B35D0179801F0E3FE01A9ED
:106FF000169B0822179801F099FF169B08331693E9
:10700000002315931DE000BF502D0020E82A00202A
:10701000387303005C2D0020049B5A1C0492109AC4
:10702000134002339B003F4A1344191D169B042250
:10703000179801F07BFF169B04331693159B0133C1
:107040001593BDF80430C3F38313DBB21A46159BC6
:107050009342E1D3179B002B40D0324BD3F810342E
:107060001493304BD3F81834002B1BD0179801F031
:10707000B0FE4DE000238DF84F301498FFF74CFB25
:107080000346002B02D001238DF84F309DF84F307E
:10709000002B03D017991498FFF7FAFA149BDB68BA
:1070A0001B681493149B002BE4D1179801F091FEF8
:1070B00000238DF803300DF10303184600F0FAFEAB
:1070C000184BD3F81834002B02D1049B154A936057
:1070D0009DF80330184600F003FF19E0114BD3F878
:1070E0001034129306E01298FFF7ECFA129BDB685B
:1070F0001B681293129B002BF5D10B4A0B4BD31A32
:10710000DB081B0443F0020309491846FFF7E0FDC2
:10711000FFF72CFE034683F00103DBB2184619B0DB
:107120005DF804FB502D00207C7303004C730300BA
:10713000C474030000B585B00023039323E0164B0D
:10714000D3F81034029301238DF807300FE0029832
:10715000FFF7D1FA03461A46039B934203D100235B
:107160008DF8073006E0029BDB681B680293029BE8
:10717000002BECD19DF80730002B01D0039B07E0DA
:10718000039B01330393039B092BD8DD4FF0FF339F
:10719000184605B05DF804FB502D002000B585B001
:1071A00001900B468DF80330FFF7C4FF0390039B5B
:1071B000B3F1FF3F01D1039B22E0039BDBB21946F1
:1071C0000198FFF78BFA104BD3F81034002B08D13D
:1071D0000D4A019BC2F81034019BDB6800221A6043
:1071E0000DE0094BD3F81034DA68019BDB681268B4
:1071F0001A60054BD3F81034DB68019A1A60039BC0
:10720000184605B05DF804FB502D002000B583B092
:107210000C4BD3F8103401930A4B01221A7009E089
:107220000198FFF770FA0198FFF740FA019BDB68BD
:107230001B680193019B002BF2D100BF00BF03B07C
:107240005DF804FB502D002082B00190009100BF3A
:1072500002B0704710B584B003900291039BDB88A5
:10726000002B0AD0039BDB881A461F4B0093134662
:107270001E4A1F49029801F055F9039B1B7A052B02
:107280002ED0039B5B7A002B12D0039B9B881A465F
:10729000039B1B7A19461046FFF7CAFA03461A46A3
:1072A000144B53F822301A461349029801F03AF968
:1072B000039B1B6819460298FFF7C6FF039B1B7AC6
:1072C0001A460E4B53F82240039B9B880021184618
:1072D000FFF78EFA034622460949029801F022F987
:1072E00000BF04B010BD00BFF874030008750300B0
:1072F00040750300002B002058750300EC2A002085
:107300005C75030000B585B00390029113468DF8BB
:107310000730039B1B7A052B0FD0039B5B7A002B56
:1073200006D00D4B1B681A460C49029801F0FAF87A
:107330000B49029801F0F6F807E09DF80730002BA2
:1073400003D00749029801F0EDF8029801F0C8F85F
:1073500000BF05B05DF804FB002B0020587503004A
:107360006875030030B58BB00790069105920493C1
:107370000E9B1B7B8DF827300E9B00221A730E99F3
:107380000498FFF767FF059B062B7FD801A252F8F0
:1073900023F000BFB1730200BB730200CB73020085
:1073A000DF730200FD7302002574020055740200B1
:1073B00007990E9801F0B6F869E0069B1B681A461B
:1073C00007990E9801F0AEF861E0069B1A68069BDB
:1073D00004331B6807990E9801F0A4F857E0069B48
:1073E0001A68069B04331968069B08331B680093D0
:1073F0000B4607990E9801F095F848E0069B19682E
:10740000069B04331868069B08331B68069A0C32E7
:1074100012680192009303460A4607990E9801F0FC
:1074200081F834E0069B1868069B04331C68069BB1
:1074300008331B68069A0C321268069910310968E5
:107440000291019200932346024607990E9801F09B
:1074500069F81CE0069B1C68069B04331D68069BAC
:1074600008331B68069A0C321268069910310968B5
:1074700006981430006803900291019200932B4605
:10748000224607990E9801F04DF800E000BF002257
:107490000E990498FFF736FF0E9B9DF827201A736C
:1074A00000BF0BB030BD00BF00B587B003900291A4
:1074B00001920093029B082B60D8009B1B7B8DF8E8
:1074C0001330009B00221A7300990198FFF7C2FE47
:1074D0000023059314E0059A029B9A4209D2039A6D
:1074E000059B13441B781A462649009801F01AF8A8
:1074F00003E02549009801F015F8059B0133059339
:10750000059B072BE7D92149009801F00BF80023D0
:10751000059326E0059A029B9A421BD2039A059B8B
:1075200013441B788DF812309DF812307E2B0AD848
:107530009DF8123018460FF0FBFA0346002B02D0DC
:107540009DF8123000E02E231A461149009800F0F1
:10755000E9FF03E00F49009800F0E4FF059B0133C9
:107560000593059B072BD5D9012200990198FFF7B8
:10757000C9FE009B9DF813201A7300E000BF07B0FE
:107580005DF804FB6C7503007475030078750300E7
:107590007C7503008075030000B583B00190019BEA
:1075A0001B781A460C4B9B5C002B05D0019B0433C7
:1075B000184606F04FFC0BE0019B1B781A46064B61
:1075C0009B5C002B04D1019B0C33184605F0D4FDC5
:1075D00000BF03B05DF804FBB432002000B587B0F3
:1075E0000390029113468DF8073000230593039B07
:1075F0001B781A46114B9B5C002B09D0039B04336C
:107600009DF807200299184606F086FC05900FE0C9
:10761000039B1B781A46094B9B5C002B08D1039BEC
:107620000C339DF807200299184605F01DFE0590C1
:10763000059B184607B05DF804FB00BFB43200207C
:1076400082B001900091034B01221A7000BF02B07A
:10765000704700BFB031002030B58DB003468DF8C3
:1076600007301A4B02AC1D460FCD0FC495E80F0032
:1076700084E80F00062302934FF0FF3303934FF08B
:10768000FF3304934FF0FF3305934FF0EB730893F0
:107690009DF80730002B01D00D4A00E0002202AB1C
:1076A00019460C4804F05AFC0B900B9B0A930A9B5A
:1076B000002B04D0084A43210A9800F0CBF8074A6F
:1076C0009DF80730137000BF0DB030BDC8750300C2
:1076D00041760200242B002084750300B131002084
:1076E00000B583B000238DF807309DF807301846A9
:1076F000FFF7B2FF00BF03B05DF804FB00B589B02F
:10770000039002910192019B8DF81F30124B0022D1
:107710001A709DF81F301A4602991048FFF75EFF55
:107720000690069B0593059B002B04D00C4A532121
:10773000059800F08FF800BF0A4B1B78002B07D08C
:10774000054B1B78DBB283F00103DBB2002BF3D1D6
:1077500000BF09B05DF804FBB0310020242B0020ED
:1077600084750300B131002000B585B0039002910B
:10777000054B00934023054A02990398FEF7BAFE91
:1077800000BF05B05DF804FBFD76020070310020FB
:1077900082B0019000BF02B07047000000B583B016
:1077A00001900548FFF7F8FE0020FFF755FF00BFE6
:1077B00003B05DF804FB00BF242B002086B00390CB
:1077C0000291019201238DF817309DF81730204A5D
:1077D000039B13601E4A029B53601D4A019B9360EA
:1077E000039B44F20102934212D0039B44F2020233
:1077F000934220D1019B164AD360154BDB681B686E
:10780000134A9361124BDB685B68114AD36112E043
:10781000019B0F4A13610E4B1B699B680C4A536115
:107820000B4B1B691B680A4A9361094B1B695B6818
:10783000074AD36100BF72B600BF00BF9DF8173082
:10784000DBB2002BFAD162B600BF00BF06B07047B2
:10785000B431002000B583B002900091019244F24F
:10786000010071466A4600F003F803B000BD00BF96
:1078700030B58BB007900691059272B600BFFFF746
:10788000C5FC00BFFFF780FA0346002BFAD1079B27
:1078900044F2020293422FD0079B44F20202934229
:1078A00069D8079B44F20102934237D0079B44F208
:1078B000010293425FD8079B012B05D0079B41F241
:1078C000010293420CD056E0394A3A4BD31ADB08F6
:1078D0001B0443F0010338491846FFF7F9F957E054
:1078E000334A344BD31ADB081B0443F001033349FA
:1078F0001846FFF7EDF94BE0059B09932C4A2D4BF9
:10790000D31ADB081B0443F00100099B5B681A468D
:10791000099B1B682A49FFF7FAF939E0059B089390
:10792000234A244BD31ADB081B0443F00104089BB1
:107930009D68089B9B68184601F0DCFB03461846CF
:10794000089B5B681946089B1B68069A0292019384
:10795000009103462A461B492046FFF7ECF9144ADA
:10796000144BD31ADB081B0443F0010316491846D5
:10797000FFF7AEF90CE00E4A0E4BD31ADB081B04DE
:1079800043F00103069A11491846FFF7AFF900BF0B
:107990000F4B1B6803F00103002B00D000BE059ABB
:1079A00006990798FFF70AFF00BF0BB030BD00BF74
:1079B0007C7303004C730300387603005876030091
:1079C0007C76030098760300C0760300D47603002B
:1079D000F0ED00E084B00190019B9B680393019B54
:1079E000DA68039BD31A184604B0704782B001903E
:1079F0000B468DF80330019B1A68019BDB680199E7
:107A000089880B4013449DF803201A70019BDB68A2
:107A10005A1C019BDA6000BF02B0704784B003902B
:107A20000B460192ADF80A30039B1A68039B9968D4
:107A3000BDF80A300B44039989880B4013441A7827
:107A4000019B1A7000BF04B0704700B583B001906D
:107A50000091009A00210198FFF7E0FF019B9B68CD
:107A60005A1C019B9A6000BF03B05DF804FB00B58F
:107A700083B001900B468DF803300198FFF7AAFF01
:107A80000246019B9B889A4207D89DF8033019460D
:107A90000198FFF7ABFF002300E00423184603B072
:107AA0005DF804FB00B583B0019000910198FFF7E9
:107AB00091FF0346002B05D000990198FFF7C5FF01
:107AC000002300E00523184603B05DF804FB000026
:107AD0002DE9F04383B0144800F05EFA034600221B
:107AE0001C461546114BD3E9002314EB020845EB65
:107AF0000309CDE900890E4BD3E90023DDE900013C
:107B0000904271EB030307D2DDE9002312F1807686
:107B100043F10007CDE90067DDE90023104619466F
:107B200003B0BDE8F08300BF382B0020D83100201F
:107B3000E031002008B5024800F03BFA00BF08BD64
:107B4000382B002000B585B0034600918DF8073032
:107B5000114A02AB1946104600F096FA0390039BB7
:107B6000002B13D0039B9DF807201A70039B009AEB
:107B70005A60094A02AB1946104600F09EFA0346C5
:107B8000002B01D0FFF7D6FF002300E004231846A6
:107B900005B05DF804FB00BFE831002000B587B0F8
:107BA00003900B4601928DF80B30039B002B04D100
:107BB000134940F22E2000F017FA019B002B04D14C
:107BC0000F4940F22F2000F00FFA019B002B01D14A
:107BD000072310E0039B1B680593059B019A5A61DC
:107BE0009DF80B30012B0CBF01230023DBB21A469A
:107BF000059B1A610023184607B05DF804FB00BF1F
:107C0000F8760300F0B587B0039002910192039BD0
:107C1000002B04D1164940F23E2000F0E5F9039B09
:107C20000593059B1B7FDBB2002B01D000231CE0DA
:107C3000059B019A9A61FFF74BFF02460B4602999A
:107C400000200C460546161943EB0507059BC3E9C2
:107C50000267059B1B69002B02D0059B029A1A61E3
:107C600005990020FFF76EFF0346184607B0F0BDE8
:107C7000F876030000B585B00190019B002B04D17C
:107C800009494FF4157000F0AFF9019B0393039B72
:107C900000221A7703990120FFF754FF0346184684
:107CA00005B05DF804FB00BFF876030000B587B0AF
:107CB0000390029113468DF8073000230593039B30
:107CC0001B781A46114B9B5C002B09D0039B043395
:107CD0009DF807200299184606F01EF905900FE05E
:107CE000039B1B781A46094B9B5C002B08D1039B16
:107CF0000C339DF807200299184605F0B5FA059057
:107D0000059B184607B05DF804FB00BFB4320020A5
:107D100000B585B0019000238DF80F30019B1B78D2
:107D20001A46114B9B5C002B08D0019B043318466C
:107D300006F0B0F903468DF80F300EE0019B1B787A
:107D40001A46094B9B5C002B07D1019B0C3318464C
:107D500005F012FB03468DF80F309DF80F301846E2
:107D600005B05DF804FB00BFB432002000B585B05B
:107D700003468DF807309DF8073019461048FFF785
:107D800076FE0390039B002B15D10E48FFF7C0FF32
:107D9000034683F00103DBB2002B0CD00A490848EC
:107DA000FFF780FE0346002B05D101220649054856
:107DB000FFF77CFF0390039B184605B05DF804FBBA
:107DC000FC310020402B0020F831002082B0EFF37E
:107DD00010830093009B019372B600BF019B18466D
:107DE00002B0704762B600BF00BF704700B585B0F3
:107DF0000190FFF7EBFF0390164B9B68002B1BD104
:107E0000144B01229A60144BD3F88020134B13407B
:107E1000104A1360104B114AC3F880200E4BD3F860
:107E200084300C4A53600C4B4FF0FF32C3F884206F
:107E3000019B00221A7002E0019B01221A70039B31
:107E4000002B01D1FFF7CEFF0023184605B05DF8E7
:107E500004FB00BF0C32002000E100E0FC06FFBD87
:107E600000B585B003468DF80730104B9B68002B9A
:107E700016D09DF80730002B12D1FFF7A7FF039013
:107E80000B4A0A4B1B681360094A084B5B68536036
:107E9000064B00229A60039B002B01D1FFF7A2FF43
:107EA0000023184605B05DF804FB00BF0C3200202B
:107EB00000E100E000B583B0019000F02BF803462C
:107EC000012B03D00549432000F08EF80198FFF7FD
:107ED0008DFF00BF03B05DF804FB00BF34770300E3
:107EE00000B583B003468DF8073000F013F8034661
:107EF000012B03D00649512000F076F89DF8073099
:107F00001846FFF7ADFF00BF03B05DF804FB00BFEC
:107F10003477030084B0EFF305830193019BC3F32F
:107F200008030393039B002B0DD1EFF314830093FD
:107F3000009B0293029B03F00103002B0CBF012363
:107F40000023DBB200E00123184604B070470000B4
:107F500082B003468DF807309DF90730002B0DDB0A
:107F60009DF8073003F01F0206499DF907305B09B1
:107F7000012000FA02F2403341F8232000BF02B092
:107F8000704700BF00E100E082B00190019BD3F890
:107F90000435184602B0704700B583B00190019BCC
:107FA0001B681846FFF7F0FF0346184603B05DF85C
:107FB00004FB00B583B00190019B93F9043018468F
:107FC000FFF7C6FF00BF03B05DF804FB08B5044B24
:107FD0001B68044A12681046984700BF08BD00BFDE
:107FE000183200201C32002000B585B003460091F5
:107FF000ADF80630BDF806300293009B039302AB48
:108000001A46002144F20200FFF732FC00BF05B01F
:108010005DF804FB86B001900091019B53E8011FBD
:108020008AB2D88902449889824228BF121A1889D4
:10803000824202BFBFF32F8F002307E0C2EA010292
:1080400043E801200028E9D14FF001038DF80F30FB
:10805000059002910492029A009B1A609DF80F30DD
:10806000DBB2184606B0704784B00190019951E820
:10807000013FC3EA034341E80132002AF7D10392EA
:10808000029300BF04B0704700B585B00190009125
:10809000009B19460198FFF7BDFF0346002B07D050
:1080A000019B1B68009A128813440393039B00E012
:1080B0000023184605B05DF804FB00B583B00190BD
:1080C0000091009B1A88009B5B889A4204D101981A
:1080D000FFF7CAFF012300E00023184603B05DF854
:1080E00004FB00B585B001900091009B5B099B00EB
:1080F000019A1A44009B03F01F03012101FA03F3C4
:108100001946104600F04DF8039000BF05B05DF829
:1081100004FB00B585B001900091009B5B099B00BA
:10812000019A1A44009B03F01F03012101FA03F393
:10813000DB431946104600F064F8039000BF05B019
:108140005DF804FB82B001900091009B5B099B00ED
:10815000019A13441A68009B03F01F0322FA03F3E9
:1081600003F00103002B14BF01230023DBB21846E8
:1081700002B0704710B487B001900091019B009A43
:1081800053E8004F104643E8000191F0000FF7D18B
:10819000059404900391059B184607B05DF8044BC5
:1081A000704710B487B001900091019B009A53E88A
:1081B000004F44EA020043E8000191F0000FF6D1BD
:1081C000059404900391049B184607B05DF8044B96
:1081D000704710B487B001900091019B009A53E85A
:1081E000004F04EA020043E8000191F0000FF6D1CD
:1081F000059404900391059B184607B05DF8044B65
:10820000704710B487B001900091019B009A53E829
:10821000004F04EA020043E8000191F0000FF6D19C
:10822000059404900391049B184607B05DF8044B35
:10823000704710B487B001900091019B009A53E8F9
:10824000004F04EB020043E8000191F0000FF6D16B
:10825000059404900391049B184607B05DF8044B05
:10826000704710B487B001900091019B009A53E8C9
:10827000004FA4EB020043E8000191F0000FF6D19B
:10828000059404900391049B184607B05DF8044BD5
:10829000704700B583B0019001210198FFF781FF7D
:1082A0000346184603B05DF804FB00B583B00190A7
:1082B00000210198FFF78DFF0346184603B05DF8D3
:1082C00004FB000000B583B001900B468DF803302D
:1082D000019B002B03D10849E820FFF785FE019B95
:1082E000DA689DF803300199098A01FB03F313440E
:1082F000184603B05DF804FB7077030000B583B047
:1083000001900091019B002B03D10849F520FFF754
:108310006BFE009B019AD2689B1A019A128AB3FBEA
:10832000F2F3DBB2184603B05DF804FB707703008C
:1083300000B585B00190019B002B01D10E234CE0CC
:10834000019B1B68002B03D12649FF20FFF74CFE41
:10835000019B5B68002B04D122494FF48070FFF72A
:1083600043FE019B9B68002B04D11E4940F2011083
:10837000FFF73AFE019BDB68002B04D119494FF44B
:108380008170FFF731FE019B1B8A002B04D1154938
:1083900040F20310FFF728FE019B9A68019B5B687F
:1083A000D31A8DF80F30019B1B68019A52681A602E
:1083B00007E0019B1A681368591C11609DF80F2093
:1083C0001A709DF80F305A1E8DF80F20002BF0D137
:1083D000019B1B6800221A710023184605B05DF846
:1083E00004FB00BF7077030000B585B00190019BCE
:1083F000002B04D11F494FF49270FFF7F5FD0023C5
:10840000039300238DF80A300DF10A031846FFF795
:1084100051FD019B1B681A68019B5B689A421FD93A
:10842000019B1B681A68013A1A601B681B78194681
:108430000198FFF747FF0390019B9A68019B1B6817
:108440001B68D31A8DF80B30019B1B681B799DF8B4
:108450000B209A4204D9019B1B689DF80B201A71CE
:108460009DF80A301846FFF73BFD039B184605B000
:108470005DF804FB7077030010B584B001900091A3
:10848000019B002B04D1154940F24710FFF7ACFDCA
:10849000009B002B04D111494FF4A470FFF7A4FDF9
:1084A000009B039300238DF80B300DF10B0318464E
:1084B000FFF700FD019B1B681C68621C1A60039992
:1084C0000198FFF71BFF034623709DF80B301846F9
:1084D000FFF706FD00BF04B010BD00BF70770300BA
:1084E00000B583B00190019B002B03D10C493120D2
:1084F000FFF77AFD019B9B68002B0CD0019B5B6909
:10850000019A1069019A1168019A92689847019B33
:1085100000229A6000E000BF03B05DF804FB00BFDA
:10852000A87703000EB400B584B00190019B002B26
:1085300003D118494220FFF757FD019B5B69002BCF
:1085400003D114494320FFF74FFD019B1B68002B0B
:1085500003D110494420FFF747FD019B5B68002BC6
:1085600003D10C494520FFF73FFD059B002B0AD0A6
:108570000023039306AB039303AB1A4605990198B6
:1085800000F0B8F900E000BF04B05DF804EB03B000
:10859000704700BFA877030000B583B001900B4679
:1085A0008DF803309DF803300A2B03D10D2101987B
:1085B000FFF7F2FF019B1A68019B9B68581C019909
:1085C000886013449DF803201A70019B9A68019BF0
:1085D0005B689A4202D30198FFF782FF00BF03B0A5
:1085E0005DF804FB00B587B00390029101920093FF
:1085F00000230593009B03F00103002B24D00BE024
:10860000029B01330293059B013305939DF81330C0
:1086100019460398FFF7C0FF029B1B788DF81330B3
:108620009DF81330002BEBD106E0019B013B019339
:1086300020210398FFF7B0FF019A059B9A422ED99B
:10864000019B002BF1D12AE0029B002B0BD002985A
:108650000EF0F5FA059006E0019B013B0193202105
:108660000398FFF799FF019A059B9A420FD9019B46
:10867000002BF1D10BE0029B01330293059B0133E8
:1086800005939DF8133019460398FFF785FF029B69
:108690001B788DF813309DF81330002BEBD100BF01
:1086A00007B05DF804FB000000B589B003900291AB
:1086B00001920093029B07930123069307E0079A18
:1086C000019BB2FBF3F30793069B01330693079AD2
:1086D000019B9A42F3D2009A069B9A4201D9009BD1
:1086E00006930B9B03F00103002B22D10A9B002B66
:1086F0001FD00B9B03F00203002B06D0009B002B26
:1087000003D130238DF8173002E020238DF8173085
:1087100008E00A9B013B0A939DF81730194603981D
:10872000FFF73AFF0A9B002B03D0069A0A9B9A4256
:10873000EFD301230793009B012B03D9009B013B3F
:10874000009309E0029A079BB2FBF3F30493049AA7
:10875000019B9A4200D205E0079B019A02FB03F3BA
:108760000793E8E7029A079BB2FBF3F30493049B99
:10877000079A02FB03F3029AD31A0293154A049B49
:1087800013441B7819460398FFF706FF079A019BCD
:10879000B2FBF3F30793079B002BE3D10B9B03F092
:1087A0000103002B11D00A9B002B0ED006E00A9B80
:1087B000013B0A9320210398FFF7EEFE0A9B002B52
:1087C00003D0069A0A9B9A42F1D300BF09B05DF824
:1087D00004FB00BF0878030000B589B00590049140
:1087E00003920293049B002BB8BF5B4206930123C4
:1087F000079307E0039B069A92FBF3F30693079B0C
:1088000001330793039B069A9A42F3DA029A079B75
:108810009A4201D9029B07930A9B002B0AD0049B22
:10882000002B04DB0B9B03F00403002B02D00A9BFC
:10883000013B0A930B9B03F00203002B02D0029B27
:10884000002B16D00B9B03F00103002B11D10A9BC8
:10885000002B0ED006E00A9B013B0A9320210598CD
:10886000FFF79AFE0A9B002B03D0079A0A9B9A42B5
:10887000F1D3049B002B07DA049B5B4204932D2168
:108880000598FFF789FE08E00B9B03F00403002B1B
:1088900003D02B210598FFF77FFE0B9B03F002030B
:1088A000002B19D00B9B03F00103002B14D1029B6A
:1088B000002B11D10A9B002B0ED006E00A9B013B36
:1088C0000A9330210598FFF767FE0A9B002B03D01F
:1088D000079A0A9B9A42F1D304990B9B01930A9B36
:1088E0000093029B039A0598FFF7DEFE00BF09B0D4
:1088F0005DF804FB00B58FB0059004910392059BD1
:10890000002B04D1AD4940F25220FFF76DFB059BCF
:108910005B69002B04D1A9494FF41570FFF764FB84
:10892000059B1B68002B04D1A44940F25520FFF79A
:108930005BFB059B5B68002B04D1A04940F25620ED
:10894000FFF752FB049B002B00F09381049B1B78E4
:108950008DF83730049B013304939DF83730002B9A
:1089600000F07E819DF83730252B40F06D8100238B
:108970000A9301230C93049B1B788DF837309DF8E4
:108980003730302B0DD0302B1BDC2B2B11D02D2B67
:1089900017D10A9B43F001030A93049B013304930C
:1089A00012E00A9B43F002030A93049B01330493F1
:1089B0000AE00A9B43F004030A93049B01330493E7
:1089C00002E000230C9300BF0C9B002BD3D10023AB
:1089D00009939DF837302A2B0CD1039B1B68191D76
:1089E000039A11601B68099A13440993049B01338D
:1089F00004931AE0049B1B788DF837309DF83730CC
:108A00002F2B12D99DF83730392B0ED8049B013308
:108A10000493099A13469B0013445B001A469DF881
:108A200037301344303B0993D3E700230B93049B67
:108A30001B788DF837309DF837302E2B1DD1049BD5
:108A400001330493049B1B788DF837309DF8373041
:108A50002F2B12D99DF83730392B0ED8049B0133B8
:108A600004930B9A13469B0013445B001A469DF82F
:108A700037301344303B0B93E4E7049B1B788DF8AD
:108A800037309DF837306C2B03D09DF83730682B8A
:108A900007D1049B01330493049B1B788DF8373076
:108AA000EFE79DF83730252B00F0C480252BC0F26E
:108AB000C680782B00F3C380582BC0F2C080583B8F
:108AC000202B00F2BC8001A252F823F0C18B0200DF
:108AD0003F8C02003F8C02003F8C02003F8C020062
:108AE0003F8C02003F8C02003F8C02003F8C020052
:108AF0003F8C02003F8C0200518B0200738B0200FE
:108B00003F8C02003F8C02003F8C02003F8C020031
:108B1000738B02003F8C02003F8C02003F8C0200EE
:108B20003F8C02003F8C02003F8C0200018C02004F
:108B30003F8C02003F8C0200E58B02003F8C02005C
:108B4000978B02003F8C02003F8C0200C18B020019
:108B5000039B1B68191D039A11601B680C930C9BE7
:108B60008DF81F309DF81F3019460598FFF714FD4A
:108B700066E0039B1B68191D039A11601B680C9328
:108B80000A9B0193099B00930B9B0A220C99059861
:108B9000FFF722FE54E0039B1B68191D039A116026
:108BA0001B680C930C990A9B0193099B00930B9BE8
:108BB0000A220598FFF778FD42E000BFD477030052
:108BC000039B1B68191D039A11601B680C930C9979
:108BD0000A9B0193099B00930B9B10220598FFF7BA
:108BE00063FD2DE0039B1B68191D039A11601B6830
:108BF00008930A9B099A08990598FFF7F3FC1FE070
:108C0000039B1B68191D039A11601B680C9330218C
:108C10000598FFF7C1FC78210598FFF7BDFC0C997A
:108C20000023019308230093082310220598FFF7DF
:108C30003BFD05E025210598FFF7AEFC00E000BFF5
:108C4000049B0133049305E09DF8373019460598DD
:108C5000FFF7A2FC049B1B78002B7FF477AE00E0AB
:108C600000BF059B1B7B002B04D00598FFF738FC49
:108C700000E000BF0FB05DF804FB00BF00B583B09B
:108C800001900198FFF754FB0346184603B05DF8C6
:108C900004FB00B58BB001900091019B1B8A043B43
:108CA0000793009A079B1344DA1C079BB2FBF3F36C
:108CB0008DF81B300198FFF797FB0590059B002B63
:108CC00001D1002338E0059B00221A71059B012287
:108CD0005A71079B9AB2059BDA80059B09939DF810
:108CE0001B30013B0493099B019A1A6000230893EF
:108CF0001DE00198FFF778FB0390039B002B0ED03B
:108D0000059B5B790133DAB2059B5A71099B039A83
:108D10001A60039B019A1A60039B099304E005986B
:108D200000F00EF8002307E0089B01330893089A2F
:108D3000049B9A42DDD3059B18460BB05DF804FBFB
:108D400000B58BB00190019B0793079B5B798DF871
:108D50001B30019B08939DF81B30013B05930023BA
:108D6000099305E0089B1B680893099B013309934D
:108D7000099A059B9A42F5D3089B1B680493019BB3
:108D80000893002309930BE0089B1B680393089941
:108D90000498FFF771FB039B0893099B0133099328
:108DA0009DF81B30099A9A42EED300BF00BF0BB06A
:108DB0005DF804FB00B585B00190019B0393039B14
:108DC000043301211846FFF734FA00BF05B05DF8FF
:108DD00004FB00B587B00190019B0593059B04330C
:108DE00001211846FFF73DFA0346039303AB0493B2
:108DF000049B1B78002B02D10198FFF7A1FF00BF55
:108E000007B05DF804FB000000B591B0039002913B
:108E100001920093039B002B03D14349B620FFF737
:108E2000E3F8039B0993039B0F93099BDB881A4686
:108E3000099B5B7902FB03F3043B0893009A089BB0
:108E40009A4203D33849C420FFF7CEF8099BDB8848
:108E50000793009B1A1D079BB2FBF3F30E93009B35
:108E60000433079AB3FBF2F2079901FB02F29B1A53
:108E70000D93019B1A68009B1344089A9A4203D2EF
:108E8000089A009BD31A01E0019B1B680C93019B7D
:108E90000C9A1A6005E00F9B1B680F930E9B013B19
:108EA0000E930E9B002BF6D100230B93079A0D9B7C
:108EB000D31A0A930A9A0C9B934228BF13460A932B
:108EC0002AE0029A0B9B134406930F9A0D9B1344BE
:108ED000043305939DF84830002B05D00A9A059974
:108EE00006980DF050FE04E00A9A069905980DF0D8
:108EF0004AFE00230D930F9B1B680F930C9A0A9B4D
:108F0000D31A0C930B9A0A9B13440B93079A0C9B4E
:108F1000934228BF13460A930C9B002BD1D100BF6C
:108F200000BF11B05DF804FB1878030000B589B0EC
:108F30000590049103920293039B079307AA0023D1
:108F40000093029B04990598FFF75EFF079B039A25
:108F50009A4203D00349F620FFF746F800BF09B054
:108F60005DF804FB1878030000B589B00590049102
:108F700003920293039B079307AA01230093029B8A
:108F800004990598FFF740FF079B039A9A4204D083
:108F900004494FF48070FFF727F800BF09B05DF86F
:108FA00004FB00BF1878030000B583B00190019B5B
:108FB000002B03D106497220FFF716F8019B00220F
:108FC0001A60BFF35F8F00BF00BF03B05DF804FB02
:108FD000A078030008B5064B00221A700548FFF779
:108FE000E3FF0549054800F029F80023184608BDAD
:108FF00028320020243200201C7903002C3200206B
:1090000082B00190019B9B6800229A60019B9B6843
:1090100000221A61019B9B6800225A61019B9B6898
:109020000022DA60019B9B6800225A60019B9B68CA
:1090300000221A6000BF02B07047000000B583B084
:1090400001900091019B002B03D110495020FEF7A5
:10905000CBFF009B002B03D10C495120FEF7C4FF2E
:10906000019B009A1A60019B1B681A68019B5A6059
:10907000019B5A68019B1B685B689A4202D1019B65
:1090800000225A6000BF03B05DF804FB287903009A
:1090900000B583B00190019B002B03D114496320DC
:1090A000FEF7A2FF019B1B68002B03D1104964202F
:1090B000FEF79AFF019B5B68002B14D0019B5B6855
:1090C0001A46019B1B689B6813441A46019B5A6011
:1090D000019B5A68019B1B685B689A4204D1019B03
:1090E00000225A6000E000BF03B05DF804FB00BF3F
:1090F0002879030000B585B00190019800F00EF8C2
:109100000390039B002B01D0039B00E0024B184609
:1091100005B05DF804FB00BFC079030086B0019084
:10912000164B0593164B04931FE0049A059BD31A24
:10913000DB10DA0F13445B10DB00059A1344039332
:10914000039B1B680293029A019B9A4202D9039BDC
:1091500004930AE0029A019B9A4203D2039B0833CC
:10916000059302E0039B5B6804E0059A049B9A4226
:10917000DBD30023184606B0704700BFC07D030054
:10918000E87E030000B583B00190019B1B68184680
:1091900000F0A3F80346002B04D105494FF4F67004
:1091A000FEF722FF4FF0A043184603B05DF804FB22
:1091B000E87E030000B585B00190084611461A46C6
:1091C00003468DF803300B468DF8023013468DF8B8
:1091D000013001AB1846FFF7D5FF03909DF803203F
:1091E0009DF802305B001A439DF801309B001A4342
:1091F0009DF818301B0242EA03019DF81C301B0445
:10920000019A1943039B02F5E07243F8221000BF54
:1092100005B05DF804FB00B585B003900023019311
:10922000002300930023012201210398FFF7C2FFCE
:1092300000BF05B05DF804FB00B585B003900B4698
:109240008DF80B309DF80B30002201920022009225
:10925000002200210398FFF7ADFF00BF05B05DF8C5
:1092600004FB00B585B0019001AB1846FFF78AFFFB
:109270000390019B012202FA03F31946039800F0C0
:1092800018F800BF05B05DF804FB00B585B001908B
:1092900001AB1846FFF776FF0390019B012202FA0B
:1092A00003F31946039800F00EF800BF05B05DF80F
:1092B00004FB82B001900091019B009AC3F808253D
:1092C00000BF02B0704782B001900091019B009AEC
:1092D000C3F80C2500BF02B0704784B00190019B19
:1092E0005B09029300230393029B002B03D14FF0F1
:1092F000FF33039300BF019B03F01F030193039A05
:10930000019B22FA03F303F00103002B14BF012396
:109310000023DBB2184604B0704782B00190009180
:10932000009A019BC3F8242500BF02B0704700B526
:1093300083B00190019B0433184605F0CBFB00BFBE
:1093400003B05DF804FB00B58FB003900291009369
:1093500013468DF8073000230D93029B09939DF867
:1093600007300A93009B0B939DF840300C93039BAE
:10937000043309A90022184605F0FAFC0D900D9B54
:1093800018460FB05DF804FB00B589B00590039254
:109390001A460B468DF8133013468DF812300F4BDA
:1093A00093F858301846FFF770FF9DF813209DF88A
:1093B00012300093039B05990948FFF7C4FF0790FB
:1093C000079B0693069B002B04D0064AF0210698C3
:1093D000FEF740FA00BF09B05DF804FB343200200C
:1093E0004C7F0300147F030008B5044B4FF080410D
:1093F0001846FFF792FF00BF08BD00BF00300040D5
:1094000088B00190019B1B789B098DF81F309DF857
:109410001F30022B06D0022B49DC002B02D0012B7F
:1094200030D044E0019B08331B789B09DBB21A461D
:10943000019B07331B789B001A44019B06331B7862
:109440009B0203F4406313440593019B05331B788F
:1094500003F00F030493019B0A331B78DB09DBB293
:109460001A46019B09331B785B0003F00603134483
:109470000393059B5A1C0499039B0B44073B02FA78
:1094800003F316E0019B09331B781A46019B08334E
:109490001B781B021A44019B07331B781B0403F43F
:1094A0007C1313440693069B01339B0201E000BF2B
:1094B0000023184608B0704700B585B003460091F8
:1094C0008DF8073013468DF80630594B93F823304A
:1094D000002B01D01123A7E000238DF80F30544B4F
:1094E000012283F823209DF90730002B1EDA062382
:1094F0008DF80F304E4B022283F823204C4B7722FD
:1095000083F828204A4B002283F82920484B002268
:1095100083F82A20464B002283F82B20444B00225C
:1095200083F82C20424BFF2283F82D209DF80F302A
:109530009DF8072002F07F02D1B23D4A13440A464B
:1095400083F82820009B1A0E9DF80F300133D1B20A
:10955000374A13440A4683F82820009B1A0C9DF8CA
:109560000F300233D1B2324A13440A4683F828201E
:10957000009B1A0A9DF80F300333D1B22C4A1344D2
:109580000A4683F828209DF80F300433009AD1B2A0
:10959000274A13440A4683F828209DF80730402BB9
:1095A00002D0482B04D007E095238DF80E3007E059
:1095B00087238DF80E3003E0FF238DF80E3000BFB7
:1095C0009DF80F3005331A4A13449DF80E2083F896
:1095D00028209DF80630022B02D0032B05D009E08D
:1095E000134B052283F8242009E0114B052283F850
:1095F000242004E00E4B012283F8242000BF9DF9B3
:109600000730002B03DB0A4B93F8243000E00123E2
:109610008DF80D309DF80D300E33DBB2054A062172
:109620000548FFF7B1FE0023184605B05DF804FBBE
:10963000343200206C3200205C32002000B589B04A
:10964000039001930B468DF80B301346ADF80830AC
:1096500001238DF81F30AA4BDB8BB3F5F67F00F0AA
:109660003281B3F5F67F00F34081B3F5F07F00F06F
:109670000B81B3F5F07F00F3388140F2D9129342A9
:1096800000F0E380B3F5ED7F80F22F81002B05D051
:1096900040F2C712934200F09E8026E1BDF80830E8
:1096A000002B04D197494FF4C870FEF79DFC944BF2
:1096B0009B8A002B04D1934940F29110FEF794FC51
:1096C0008F4B9A8A8E4BDA82E7E08D4B00221A8408
:1096D0008B4BFF2283F82820894B00221A83884B6A
:1096E000032283F823207CE0854B1B8C01339AB244
:1096F000834B1A84824B1B8C44F6206293420FD911
:10970000019B02221A707E4B0022DA830223F3E0CF
:10971000039B013303939DF80B30013B8DF80B3015
:109720009DF80B30002B03D0039B1B78FF2BEFD051
:109730009DF80B30002B41D0039B1B78FE2B35D1BD
:10974000039B013303939DF80B30013B8DF80B30E5
:109750006B4B042283F823209DF80B309BB2BDF89D
:109760000820934228BF1346ADF814300023069317
:109770000BE0039A069B1A44614BD968069B0B4485
:1097800012781A70069B01330693BDF81430069ABE
:109790009A42EED35A4ABDF814301383584BDA6814
:1097A000BDF814301344564AD3601AE0019B0522D9
:1097B0001A70534B0022DA8302239DE01023524A91
:1097C00001215248FFF7E0FD00238DF81F304C4B7C
:1097D00040F2C712DA839DF81F30002B01D101231C
:1097E0008AE0474B93F82330032B3FF47DAF32E000
:1097F000434B1B8BBDF80820D31AADF81630BDF8CB
:109800001630F02B02D9F023ADF816303C4BDA6855
:10981000BDF81630DBB201213C48FFF7B5FD384BEF
:10982000DA68BDF816301344354AD360344B1A8BCE
:10983000BDF8163013449AB2314B1A8300238DF8C9
:109840001F302F4B40F2D912DA839DF81F30002BC6
:1098500001D1012350E02A4B1B8BBDF808209A420E
:10986000C6D8274BDB8A013B9AB2254BDA8202230A
:10987000254A01212548FFF787FD00238DF81F3079
:109880001F4B4FF4F072DA839DF81F30002B01D18B
:10989000012331E000238DF80B30194BDB8A002BBC
:1098A0007FF413AF164BFF2283F828200223164AB9
:1098B00001211648FFF768FD00238DF81F30104B7B
:1098C0004FF4F672DA839DF81F30002B01D101238B
:1098D00012E00B4B002283F82320019B00221A7018
:1098E000074B0022DA83022306E000238DF81F30A5
:1098F000034B0022DA830323184609B05DF804FB0A
:1099000034320020147F03006C3200205C320020CF
:1099100000B593B003900B4601928DF80B30039B7A
:109920001B788DF84730039B01331B781A06039B85
:1099300002331B781B041A43039B03331B781B025F
:109940001343039A043212781343109301238DF8C2
:109950004630BE4B9B8BB3F51C7F00F3EB82B3F517
:10996000137F16DCB3F50E7F00F08C81B3F50E7F0C
:1099700000F3E082002B00F09380002BC0F2DA822B
:1099800040F22622934200F3D582B3F5047F51DAE8
:10999000D0E2A3F24D23232B00F2CC8201A252F895
:1099A00023F000BF459D0200359F0200359F020055
:1099B000359F0200359F0200359F0200AB9D0200DB
:1099C000359F0200359F0200359F0200359F02003F
:1099D000359F0200359F0200359F0200359F02002F
:1099E000359F0200359F0200359F0200359F02001F
:1099F000359F0200279E0200359F0200359F02001E
:109A0000359F0200359F0200359F0200359F0200FE
:109A1000359F0200359F0200359F02008B9E020099
:109A2000359F0200359F0200359F0200359F0200DE
:109A3000D19E0200A3F50473162B00F27B8201A2D3
:109A400052F823F0D19A0200359F0200359F0200A0
:109A50000D9B0200359F0200359F0200359F0200DA
:109A6000359F0200359F0200679B0200359F020070
:109A7000359F0200359F0200359F0200359F02008E
:109A8000359F0200359F0200359F0200359F02007E
:109A9000359F0200359F0200359F0200F59B0200B2
:109AA000012200214020FFF707FD0F900F9B0E932E
:109AB0000E9B002B05D0664A40F20F210E98FDF751
:109AC000C9FE00238DF84630604B4FF404729A8330
:109AD0009DF84630002B01D1012332E20122002102
:109AE0004020FFF7E9FC0F900F9B0D930D9B002B7F
:109AF00005D0574A40F212210D98FDF7ABFE002326
:109B00008DF84630514B40F213229A839DF846302F
:109B1000002B01D1012314E29DF8473023F0030309
:109B2000002B07D0019B04221A70484B00229A8315
:109B3000022306E203224FF4D5714820FFF7BCFC54
:109B40000F900F9B0C930C9B002B05D0404A4FF4B9
:109B500006710C98FDF77EFE00238DF846303B4BD6
:109B600040F219229A839DF84630002B01D101233F
:109B7000E7E19DF8473003F00403002B13D1334A8B
:109B8000937A032161F3020393729DF8473023F027
:109B90000303002B07D0019B04221A702B4B0022D9
:109BA0009A830223CDE1294B00221A84274B9B7A0A
:109BB00003F00703DBB2032B02D14FF0804300E038
:109BC00000230B9302220B99E920FFF775FC0F90FD
:109BD0000F9B0A930A9B002B05D01D4A40F22521BA
:109BE0000A98FDF737FE00238DF84630174B40F2F8
:109BF00026229A839DF84630002B01D10123A0E153
:109C00009DF8473003F00403002B56D00F4A937A97
:109C1000012161F3020393729DF8473023F004039E
:109C20008DF84730094B1B8C01339AB2074B1A84CD
:109C3000064B1B8CB3F5FA6F0CD9019B02221A70EC
:109C4000024B00229A8302237BE100BF34320020C2
:109C5000147F0300022200214120FFF72DFC0F900A
:109C60000F9B0793079B002B05D0A64A40F2372194
:109C70000798FDF7EFFD00238DF84630A24B4FF417
:109C80000E729A839DF84630002B01D1012358E1D2
:109C90009DF8473023F00303002B07D0019B0422DB
:109CA0001A70994B00229A8302234AE19DF84730AB
:109CB00003F00103002BB5D195E09DF8473023F068
:109CC0000303002B52D0019B04221A708E4B0022FA
:109CD0009A83022335E18C4B1B8C01339AB28A4B59
:109CE0001A84894B1B8CB3F5FA6F07D9019B0222AA
:109CF0001A70854B00229A83022322E1824B9B7AC1
:109D000003F00703DBB2032B02D14FF0804300E0E6
:109D100000230B9302220B99E920FFF7CDFB0F9054
:109D20000F9B0893089B002B05D0764A4FF41371C4
:109D30000898FDF78FFD00238DF84630724B40F2F6
:109D40004D229A839DF84630002B01D10123F8E083
:109D50009DF8473023F00303002B08D0019B042219
:109D60001A70694B00229A830223EAE000BF9DF833
:109D7000473003F00103002BADD1022200217A20ED
:109D8000FFF79AFB0F900F9B0993099B002B05D0BF
:109D90005C4A40F252210998FDF75CFD00238DF8E2
:109DA0004630594B40F253229A839DF84630002B9F
:109DB00001D10123C5E09DF8473023F00303002BB8
:109DC00007D0019B04221A704F4B00229A83022372
:109DD000B7E0109B03F08043002B04D04A4A937AEB
:109DE00043F008039372484B9B7A03F00703DBB2FE
:109DF000032B2CD001224FF400715020FFF75CFBA5
:109E00000F900F9B0693069B002B05D03D4A4FF405
:109E100018710698FDF71EFD00238DF846303A4B69
:109E200040F261229A839DF84630002B01D1012334
:109E300087E09DF8473023F00303002B07D0019BF8
:109E400004221A70304B00229A83022379E02E4BB1
:109E50002E4ADA602C4B01229A82012200214920ED
:109E6000FFF72AFB0F900F9B0593059B002B05D056
:109E7000244A40F26A210598FDF7ECFC00238DF896
:109E80004630214B40F26B229A839DF84630002BDE
:109E900001D1012355E09DF8473023F00303002B47
:109EA00007D0019B04221A70174B00229A830223C9
:109EB00047E0039B013303939DF80B30013B8DF882
:109EC0000B30114B0022DA830F4B4FF41C729A8334
:109ED0000DF113039DF80B1010220398FFF7AEFB52
:109EE0000346012B01D800232BE09DF81330002BF3
:109EF0000ED09DF81320019B1A70034B00229A8309
:109F000002231EE0147F0300343200207C32002044
:109F10000E48FFF775FA03460D4A53600C4B4FF499
:109F200000721A81019B00221A70094B00229A8349
:109F3000022306E000238DF84630054B00229A8369
:109F40000323184613B05DF804FB00BF7C320020E9
:109F50003432002000B589B003900B4601928DF891
:109F60000B3001238DF81F30404B9B8B40F2A22217
:109F7000934261D040F2A22293426BDC002B03D0CB
:109F8000B3F5267F21D065E0039B1B788DF81E304A
:109F90009DF81E3023F00303002B07D0019B042201
:109FA0001A70324B00229A8302235AE0039B01333A
:109FB00003939DF80B30013B8DF80B302B4B0022A7
:109FC000DA832A4B4FF426729A830DF113039DF81E
:109FD0000B104FF400720398FFF730FB0346012B80
:109FE00001D800233DE09DF81330002B08D09DF8E8
:109FF0001320019B1A701D4B00229A83022330E02C
:10A000001A4B9B8A012B1DD9012200214C20FFF7FE
:10A0100053FA0690069B0593059B002B05D0144A26
:10A0200040F2A1210598FDF715FC00238DF81F30A3
:10A030000E4B40F2A2229A839DF81F30002B01D1D3
:10A0400001230EE0019B00221A70084B00229A8324
:10A05000022306E000238DF81F30044B00229A8370
:10A060000323184609B05DF804FB00BF343200201A
:10A07000147F030000B58DB003900B4601928DF85C
:10A080000B3001238DF82F30AC4B9B8BB3F54C7FFD
:10A0900000F0C781B3F54C7F00F3EC81B3F5487F46
:10A0A00000F09081B3F5487F00F3E48140F20A327A
:10A0B000934200F03A8140F20A32934200F3DA818F
:10A0C000B3F53B7F00F0E380B3F53B7F00F3D28133
:10A0D000B3F5397F00F0B880B3F5397F00F3CA815A
:10A0E00040F2D322934200F08180B3F5357F80F2B5
:10A0F000C181002B04D040F2C322934237D0B9E192
:10A10000039B1B788DF823309DF8233023F0030345
:10A11000002B07D0019B04221A70884B00229A83DF
:10A120000223AEE1854B9B7A03F00703DBB2012BE0
:10A1300035D0824B9B8A012B31D9804B1B69012280
:10A1400019465920FFF7B8F90790079B0693069B1D
:10A15000002B05D07A4A40F2C2210698FDF77AFB1F
:10A1600000238DF82F30754B40F2C3229A839DF85F
:10A170002F30002B01D1012383E1039B1B788DF845
:10A1800023309DF8233023F00303002B07D0019BDD
:10A1900004221A70694B00229A83022371E1674BF3
:10A1A0009A8A664BDA82EFE0644B00221A83634B93
:10A1B000042283F82320614BFF2283F828205F4B81
:10A1C0009B8A012B01D9FC2200E0FE225B4B83F825
:10A1D000292002235B4A02215B48FFF7D5F80023C0
:10A1E0008DF82F30554B40F2D3229A839DF82F30B3
:10A1F000002B2FD1012344E1504B1B8BC3F500737F
:10A20000ADF82C30BDF82C30F02B02D9F023ADF88E
:10A210002C304A4BDB68494A128B9818BDF82C3019
:10A22000D9B20123474AFFF7AFF8444B1A8BBDF868
:10A230002C3013449AB2414B1A8300238DF82F30EF
:10A240003E4B4FF439729A839DF82F30002B02D188
:10A25000012316E100BF394B1B8BB3F5007FCBD335
:10A26000364BDB6803F50073344AD360334B03226B
:10A2700083F823200323334A01213348FFF784F86E
:10A2800000238DF82F302D4B4FF43B729A839DF8AD
:10A290002F30002B01D10123F3E0284B93F83A3003
:10A2A00003F01F038DF817309DF81730052B17D0DA
:10A2B0009DF817300B2B03D09DF817300D2B07D1CD
:10A2C000019B05221A701D4B00229A830223D8E0BD
:10A2D000019B04221A70194B00229A830223D0E0BA
:10A2E000164B00221A8444E0144B1B8C01339AB2A3
:10A2F000124B1A84114B1B8C44F62062934207D9EF
:10A30000019B02221A700D4B00229A830223B8E0AF
:10A3100010230C4A01210C48FFF736F800238DF872
:10A320002F30064B40F20A329A839DF82F30002BD3
:10A3300001D10123A5E000230A9315E03432002067
:10A34000147F03006C3200205C320020039A0A9BC9
:10A3500013441B78002B04D04C4B002283F823209D
:10A3600007E00A9B01330A939DF80B300A9A9A4240
:10A37000ECD3464B93F82330032BB5D0434BDB8A09
:10A38000013B9AB2414BDA82404BDB8A002B7FF4CF
:10A390000BAF3E4B9B8A012B64D93C4BFF2283F8C9
:10A3A00028203A4BFD2283F829200323384A022132
:10A3B0003848FEF7E9FF00238DF82F30334B4FF478
:10A3C00048729A839DF82F30002B01D1012358E069
:10A3D0002E4B00221A842D4B032283F823203CE0CD
:10A3E0002A4B1B8C01339AB2284B1A84274B1B8CA7
:10A3F00044F62062934207D9019B02221A70234B34
:10A4000000229A8302233CE01023214A01212148A3
:10A41000FEF7BAFF00238DF82F301C4B4FF44C721F
:10A420009A839DF82F30002B01D1012329E00023CE
:10A4300009930DE0039A099B13441B78002B04D069
:10A44000124B002283F8232007E0099B0133099374
:10A450009DF80B30099A9A42ECD30C4B93F82330B9
:10A46000032BBDD0019B00221A70084B00229A8357
:10A47000022306E000238DF82F30044B00229A833C
:10A48000032318460DB05DF804FB00BF34320020F2
:10A490006C3200205C32002000B58BB0019000913E
:10A4A000019BDB680993019B1B7C8DF82330A24B39
:10A4B000DB8A002B05D1A04B93F858301846FEF7E5
:10A4C000D0FE9D4B93F82330022B05D09A4B93F886
:10A4D0002330012B40F0C0809DF82330062B04D898
:10A4E000964940F25730FDF77FFD9DF82330063B3B
:10A4F0008DF82330099B06330993019B5B681B7819
:10A500004C2B14D19DF82330002B10D09DF8233014
:10A51000013B8DF82330099B0133099307E09DF837
:10A520002330013B8DF82330099B013309939DF8BB
:10A530002330002B03D0099B1B78FF2BEFD09DF815
:10A540002330002B0FD1019B5B681B784C2B08D16B
:10A550009DF8233001338DF82330099B013B09938B
:10A5600001E000230993099B002B53D1724B93F810
:10A570002230DBB2012B4DD001238DF809306E4B18
:10A5800093F82230DBB2052B21D0052B23DC022BE4
:10A5900002DC002B03DC1EE0042B14D01BE00023A4
:10A5A0008DF80830644B032283F8222000F0C2FAB1
:10A5B0000790079B002B1AD0604A40F2833107981E
:10A5C000FDF748F913E001238DF8083012E002236B
:10A5D0008DF808300EE003230693069B002B08D06D
:10A5E000564A4FF463710698FDF734F901E000BF55
:10A5F00000E000BF504B93F858301846FEF731FE8C
:10A600004D4B032283F822204B4B1B6802AA1046B5
:10A610009847D9E0484B93F82330022B18D1464B8A
:10A62000012283F82320099B1B788DF817309DF8B1
:10A63000173023F00103002B0AD141483E4B93F819
:10A6400024300E33DBB23F4A0621FEF79DFEBBE00D
:10A65000394B002283F8232006238DF80F30364B28
:10A6600093F82230DBB2013B042B00F2998001A267
:10A6700052F823F089A6020097A60200A1A70200C3
:10A68000E1A6020049A702002B4B022283F82220F8
:10A69000294B00229A830DF10F029DF823301946B1
:10A6A0000998FFF735F90346012B40F28580002316
:10A6B0008DF80C309DF80F308DF80D301E4B0322B5
:10A6C00083F822201C4B93F858301846FEF7C9FD3A
:10A6D000FEF78AFE184B1B6803AA104698476BE0EA
:10A6E0000DF10F029DF8233019460998FFF732FC4F
:10A6F0000346012B62D901238DF80C309DF80F30F1
:10A700008DF80D300C4B032283F822200A4B0022D7
:10A710009A82094B0022DA82074B002283F8232019
:10A72000054B93F858301846FEF79BFD024B1B680B
:10A7300003AA1046984741E034320020147F0300FA
:10A74000623200206C3200200DF10F029DF82330A0
:10A7500019460998FFF78EFC0346012B30D90223D6
:10A760008DF80C309DF80F308DF80D30184B03220A
:10A7700083F82220164B002283F82320144B00225A
:10A780009A82134B0022DA82114B93F85830184604
:10A79000FEF767FD0E4B1B6803AA104698470FE0B3
:10A7A00003230493049B002B0CD00A4A40F2D331BC
:10A7B0000498FDF74FF805E000BF04E000BF02E099
:10A7C00000BF00E000BF00BF0BB05DF804FB00BF9E
:10A7D00034320020147F030000B589B00390029149
:10A7E0001346ADF80630039B002B04D12E4940F2EE
:10A7F000DD30FDF7F9FB2D4B93F82230DBB2002B57
:10A8000001D108234CE0294B93F82230DBB2032B13
:10A8100001D0112344E0BDF80630002B01D10723FD
:10A820003EE0224B042283F82220204B9B7A03F047
:10A830000803DBB2002B04D1029B5B021B4A1361AD
:10A8400002E01A4A029B1361184A039BD360174A1D
:10A85000BDF806309382154ABDF80630D382134BFB
:10A8600000229A83BDF80630012B01D9522300E063
:10A8700051238DF81F300D4B19699DF81F300122AF
:10A880001846FEF719FE0690069B0593059B002BC4
:10A8900005D0054A40F2FD310598FCF7DBFF0023A7
:10A8A000184609B05DF804FB147F03003432002021
:10A8B00000B589B0039002911346ADF80630039BB2
:10A8C000002B04D13E4940F20540FDF78DFB3D4B86
:10A8D00093F82230DBB2002B01D108236BE0394B17
:10A8E00093F82230DBB2032B01D0112363E0BDF8D3
:10A8F0000630002B01D107235DE0324B052283F89F
:10A900002220304B9B7A03F00803DBB2002B04D1EA
:10A91000029B5B022B4A136102E02A4A029B1361ED
:10A92000284A039BD360274ABDF806309382254A04
:10A93000BDF80630D382234B00229A83BDF806303F
:10A94000012B14D11F4B1B69012219465820FEF719
:10A95000B3FD0790079B0593059B002B05D0184A74
:10A960004FF485610598FCF775FF002323E0154B34
:10A970009B7A03F00703DBB2012B08D1114B1B6953
:10A98000012219465920FEF797FD079007E0BDF810
:10A99000063001221946D720FEF78EFD0790079B4F
:10A9A0000693069B002B05D0054A40F237410698D6
:10A9B000FCF750FF0023184609B05DF804FB00BF08
:10A9C000147F03003432002000B58DB00390029153
:10A9D000524B93F82230DBB2002B01D0082398E0D1
:10A9E000029B002B0FD0039BDB78FF2B0BD0039B2C
:10A9F0005B78FF2B07D0039B1B78FF2B03D0039BB7
:10AA00009B78FF2B01D1072383E0039BDB78002B8E
:10AA10000BD0039B5B78002B07D0039B1B78002B8C
:10AA200003D0039B9B78002B04D13D4940F24C405E
:10AA3000FDF7DAFA039BDA78384B83F85820374B66
:10AA400093F858301846FEF7E6FB344B93F858302D
:10AA50001846FEF706FC039B9B788DF81430039B89
:10AA60001B788DF81530039B5B788DF81630FF232B
:10AA70008DF8173006238DF81830FF238DF8193024
:10AA80004FF08063079300238DF8203000238DF86A
:10AA9000213005A90023234A234803F045FC0B90ED
:10AAA0000B9B0A930A9B002B05D01D4A4FF48C6127
:10AAB0000A98FCF7CFFE194A029B1360174B01223C
:10AAC00083F82220154A937A6FF302039372134A94
:10AAD000937A6FF3C3039372104B002283F8232001
:10AAE0000E4BFF2283F828200A2300930F4B0122EC
:10AAF0000F490D48FEF727FC0B900B9B0993099B10
:10AB0000002B05D0064A40F26C410998FCF7A2FEE2
:10AB1000002318460DB05DF804FB00BF343200205E
:10AB2000147F030099A402004C7F03006C320020C4
:10AB30005C32002008B5124B93F82230DBB2002BB8
:10AB400001D108231AE00E4B93F82230DBB2032B1D
:10AB500001D0112312E00B48FEF7E9FB084B93F8F4
:10AB6000583000211846FEF767FB054B002283F89A
:10AB70002320034B002283F822200023184608BD1F
:10AB8000343200204C7F0300094B93F82230DBB2B3
:10AB9000032B07D0064B93F82230DBB2002B01D0F9
:10ABA000012300E0002303F00103DBB218467047E5
:10ABB00034320020054B93F82230DBB2022B01D94E
:10ABC000034B00E000231846704700BF34320020DA
:10ABD0003832002000BF704708B501E0FFF7FAFFE8
:10ABE000FFF7D2FF0346002BF8D100BF00BF08BD1E
:10ABF00000B593B00190019B5A78514B1A70514B9C
:10AC00001B681193119B9B691093019B1B78022B6E
:10AC100061D0022B7EDC002B02D0012B3CD079E0EE
:10AC2000019B5B78002B0FD0119B0F930F9800F0C6
:10AC3000F5F80E900E9B0D930D9B002B04D0424A0D
:10AC400058210D98FCF706FEFFF7B4FF03461A687B
:10AC5000109B1A60109B4FF400725A60394B1B68AE
:10AC60009B699B68002B60D000238DF82430019BEA
:10AC70005B78002B14BF01230023DBB28DF8253055
:10AC800000230A93109B9B690B93109B9B68119A5E
:10AC900009A91046984748E02A4B1B689B699B68A6
:10ACA000002B44D002238DF81830019B5B78002BD9
:10ACB00014BF01230023DBB28DF81930109B0C3335
:10ACC0000793109B9B690893109B9B68119A06A998
:10ACD000104698472BE01B4B1B689B699B68002B19
:10ACE00027D003238DF80C30019B5B78002B14BF19
:10ACF00001230023DBB28DF80D30109B0C3304933D
:10AD0000109B9B690593109B9B68119A03A91046A1
:10AD100098470EE003230C930C9B002B0BD00A4AA0
:10AD200088210C98FCF796FD05E000BF04E000BF09
:10AD300002E000BF00E000BF13B05DF804FB00BFFD
:10AD400090320020943200205C7F030000B58BB06D
:10AD5000039002910192039B002B03D12B49922077
:10AD6000FDF742F9039B0893089B9B690793089B97
:10AD70001B69B3F5007F01D0062343E0244B1B6819
:10AD8000002B01D011233DE0079B019A9A61079B9C
:10AD9000029A9A601E4A089B136000230993089B3D
:10ADA00014331C491846FFF70FFE0990099B002B2E
:10ADB0000DD1029B002B0AD1FFF70EFF164B1B781B
:10ADC000DBB2002B01D1002300E00D230993099B86
:10ADD000002B16D00E4B00221A60029B002B10D0C5
:10ADE00000238DF8103001238DF8113000230593D6
:10ADF000079B9B690693079B9B6804AA11460398CF
:10AE00009847099B18460BB05DF804FB5C7F030074
:10AE100094320020F1AB02009032002000B589B0DE
:10AE20000190019B002B03D11F49CA20FDF7DCF8DC
:10AE3000019B0793079B9B6906931C4B1B68079A12
:10AE40009A4201D011232AE0FFF79EFE0346002B11
:10AE500001D0112323E0FFF76DFE0590059B002B29
:10AE600002D1124B00221A60069B9B68002B15D062
:10AE700001238DF80830059B002B14BF012300230C
:10AE8000DBB28DF8093000230393069B9B69049382
:10AE9000069B9B6802AA114601989847059B184695
:10AEA00009B05DF804FB00BF5C7F03009432002012
:10AEB00000B589B001900091019B002B03D130496E
:10AEC000F620FDF791F8009B002B03D12C49F720C9
:10AED000FDF78AF8019B0693069B9B690593002367
:10AEE0000793284B1B68069A9A4201D0112343E02E
:10AEF000FFF74AFE0346002B01D011233CE0059BDF
:10AF0000009A0C3307CA83E80700009B9868009BEF
:10AF10001968009B5B689BB21A46FFF75DFC0790BF
:10AF2000079B002B0ED1059B9B68002B0AD1FFF7D6
:10AF300053FE154B1B78DBB2002B01D1002300E040
:10AF40000D230793059B9B68002B14D0079B002BB8
:10AF500011D002238DF8083001238DF80930059BAC
:10AF60000C330393059B9B690493059B9B6802AA82
:10AF7000114601989847079B184609B05DF804FBF5
:10AF80005C7F0300943200209032002000B589B02D
:10AF900001900091019B002B04D131494FF4947032
:10AFA000FDF722F8009B002B04D12D4940F2291017
:10AFB000FDF71AF8019B0693069B9B6905930023F6
:10AFC0000793284B1B68069A9A4201D0112343E04D
:10AFD000FFF7DAFD0346002B01D011233CE0059B6F
:10AFE000009A0C3307CA83E80700009B9868009B0F
:10AFF0001968009B5B689BB21A46FFF759FC0790E3
:10B00000079B002B0ED1059B9B68002B0AD1FFF7F5
:10B01000E3FD154B1B78DBB2002B01D1002300E0D0
:10B020000D230793059B9B68002B14D0079B002BD7
:10B0300011D002238DF8083001238DF80930059BCB
:10B040000C330393059B9B690493059B9B6802AAA1
:10B05000114601989847079B184609B05DF804FB14
:10B060005C7F0300943200209032002088B003906F
:10B070000B4601928DF80B30039B07939DF80B3024
:10B08000002B04D0012B0CD000BF062315E0019B40
:10B090000593059B002B02D0059B00221A7000230C
:10B0A0000BE0019B002B01D1072306E0019B0693D7
:10B0B000079B1A1D069B1A600023184608B07047AC
:10B0C00000B585B00190019B002B04D1074940F2E7
:10B0D0007D10FCF789FF019B0393039B9B690293FF
:10B0E000029B184605B05DF804FB00BF5C7F0300BF
:10B0F000BFF34F8F00BF064BDB6803F4E0620449E7
:10B10000044B1343CB60BFF34F8F00BF00BFFDE77D
:10B1100000ED00E00400FA0582B01B4B1B68B3F1A0
:10B12000FF3F0AD1194B1B68DBB20193184B1B6818
:10B130001B0903F00F03009305E0134B1B680193F9
:10B14000144B1B680093019B062B19D1009B033BFA
:10B15000032B13D801A252F823F000BF6DB10200F7
:10B1600071B1020075B1020079B10200012308E05B
:10B17000012306E0012304E0012302E0012300E0B3
:10B180000023184602B0704730010010E00F00F0B5
:10B19000E80F00F03401001082B0154B1B68DBB2E1
:10B1A0000193144B1B681B0903F00F030093019BD1
:10B1B000062B19D1009B033B032B13D801A252F895
:10B1C00023F000BFD5B10200D9B10200DDB1020009
:10B1D000E1B10200012308E0002306E0002304E0BF
:10B1E000002302E0002300E00023184602B070476D
:10B1F000E00F00F0E80F00F082B01B4B1B68B3F1CA
:10B20000FF3F0AD1194B1B68DBB20193184B1B6837
:10B210001B0903F00F03009305E0134B1B68019318
:10B22000144B1B680093019B062B19D1009B033B19
:10B23000032B13D801A252F823F000BF4DB2020035
:10B2400051B2020055B2020059B20200012308E0D7
:10B25000012306E0012304E0012302E0012300E0D2
:10B260000023184602B0704730010010E00F00F0D4
:10B27000E80F00F03401001082B0154B1B68DBB200
:10B280000193144B1B681B0903F00F030093019BF0
:10B29000062B19D1009B033B032B13D801A252F8B4
:10B2A00023F000BFB5B20200B9B20200BDB2020085
:10B2B000C1B20200012308E0002306E0002304E0FD
:10B2C000002302E0002300E00023184602B070478C
:10B2D000E00F00F0E80F00F082B01B4B1B68B3F1E9
:10B2E000FF3F0AD1194B1B68DBB20193184B1B6857
:10B2F0001B0903F00F03009305E0134B1B68019338
:10B30000144B1B680093019B062B19D1009B033B38
:10B31000032B13D801A252F823F000BF2DB3020073
:10B3200031B3020035B3020039B30200012308E053
:10B33000012306E0012304E0012302E0012300E0F1
:10B340000023184602B0704730010010E00F00F0F3
:10B35000E80F00F03401001082B0154B1B68DBB21F
:10B360000193144B1B681B0903F00F030093019B0F
:10B37000062B19D1009B033B032B13D801A252F8D3
:10B3800023F000BF95B3020099B302009DB3020001
:10B39000A1B30200012308E0002306E0002304E03B
:10B3A000002302E0002300E00023184602B07047AB
:10B3B000E00F00F0E80F00F082B0154B1B68DBB225
:10B3C0000193144B1B681B0903F00F030093019BAF
:10B3D000062B19D1009B033B032B13D801A252F873
:10B3E00023F000BFF5B30200F9B30200FDB3020081
:10B3F00001B40200012308E0002306E0002304E07A
:10B40000002302E0002300E00023184602B070474A
:10B41000E00F00F0E80F00F082B01B4B1B68B3F1A7
:10B42000FF3F0AD1194B1B68DBB20193184B1B6815
:10B430001B0903F00F03009305E0134B1B680193F6
:10B44000144B1B680093019B062B19D1009B033BF7
:10B45000032B13D801A252F823F000BF6DB40200F1
:10B4600071B4020075B4020079B40200002308E050
:10B47000002306E0012304E0012302E0012300E0B1
:10B480000023184602B0704730010010E00F00F0B2
:10B49000E80F00F03401001082B01B4B1B68B3F1C1
:10B4A000FF3F0AD1194B1B68DBB20193184B1B6895
:10B4B0001B0903F00F03009305E0134B1B68019376
:10B4C000144B1B680093019B062B19D1009B033B77
:10B4D000032B13D801A252F823F000BFEDB40200F1
:10B4E000F1B40200F5B40200F9B40200012308E04F
:10B4F000012306E0012304E0012302E0012300E030
:10B500000023184602B0704730010010E00F00F031
:10B51000E80F00F03401001082B01B4B1B68B3F140
:10B52000FF3F0AD1194B1B68DBB20193184B1B6814
:10B530001B0903F00F03009305E0134B1B680193F5
:10B54000144B1B680093019B062B19D1009B033BF6
:10B55000032B13D801A252F823F000BF6DB50200EF
:10B5600071B5020075B5020079B50200012308E04B
:10B57000012306E0012304E0012302E0012300E0AF
:10B580000023184602B0704730010010E00F00F0B1
:10B59000E80F00F03401001082B0134B1B680193D8
:10B5A000124B1B680093019B062B19D1009B033B98
:10B5B000032B13D801A252F823F000BFCDB502002F
:10B5C000D1B50200D5B50200D9B50200002308E0CC
:10B5D000002306E0002304E0012302E0012300E051
:10B5E0000023184602B070473001001034010010EB
:10B5F000024B034A1A6000BF704700BF542B002063
:10B600000090D00308B5FFF787FD0346002B06D056
:10B61000A04B1B681B0AA04A03F01F031360FFF72F
:10B62000BBFD0346002B02D09C4B9D4A1A60FFF7DE
:10B63000E3FD0346002B06D09A4B1B685B0B9A4A2E
:10B6400003F007031360FFF717FE0346002B05D036
:10B65000964BDB68954A23F08073D360FFF73CFE7E
:10B660000346002B0ED04FF080430022C3F80C217C
:10B670004FF080430022C3F810214FF08043002296
:10B68000C3F83825FFF768FE0346002B02D0884B2D
:10B6900003221A60FFF790FE0346002B0BD0854B68
:10B6A00005221A60844B01221A60844B00221A6022
:10B6B000834B3F221A60FFF7AFFE0346002B76D084
:10B6C0004FF080537F4AD3F80434C2F820354FF04E
:10B6D00080537C4AD3F80834C2F824354FF08053A5
:10B6E000784AD3F80C34C2F828354FF08053754AA5
:10B6F000D3F81034C2F82C354FF08053714AD3F888
:10B700001434C2F830354FF080536E4AD3F81834F1
:10B71000C2F834354FF080536A4AD3F81C34C2F86B
:10B7200040354FF08053674AD3F82034C2F844358F
:10B730004FF08053634AD3F82434C2F848354FF0B1
:10B740008053604AD3F82834C2F84C354FF0805308
:10B750005C4AD3F82C34C2F850354FF08053594A24
:10B76000D3F83034C2F854354FF08053554AD3F8EB
:10B770003434C2F860354FF08053524AD3F838342D
:10B78000C2F864354FF080534E4AD3F83C34C2F8C7
:10B7900068354FF080534B4AD3F84034C2F86C35CB
:10B7A0004FF08053474AD3F84434C2F87035FFF75E
:10B7B00073FE0346002B05D0434B1B68434A03F03E
:10B7C0004F031360FFF7A8FE0346002B0DD04FF088
:10B7D0008043D3F8003403F00103002B05D04FF071
:10B7E00080436FF00102C3F80024FFF7D5FE034643
:10B7F000002B05D0364B1B68354A43F48063136039
:10B80000344BD3F88830334A43F47003C2F888309D
:10B81000BFF34F8F00BFBFF36F8F00BF4FF01023F8
:10B82000D3F80032002B05DB4FF01023D3F804329D
:10B83000002B2BDA284B0122C3F8042500BF264B2E
:10B84000D3F80034002BFAD04FF010231522C3F8A0
:10B85000002200BF204BD3F80034002BFAD04FF069
:10B8600010231522C3F8042200BF1B4BD3F8003469
:10B87000002BFAD0184B0022C3F8042500BF164B4A
:10B88000D3F80034002BFAD0FFF732FCFFF7B0FEFC
:10B8900000BF08BD240300104035014074C00740BC
:10B8A0000DF0ADBA440200103C050040F0ED00E0A0
:10B8B000A005004010560040885600401856004031
:10B8C0001456004000C0004058020010E40E004032
:10B8D0003C17004000ED00E000E0014000B583B0FF
:10B8E0000190019B1B68184600F09DF80346002B51
:10B8F00004D105494FF4F670FCF776FB4FF0A043F6
:10B90000184603B05DF804FBB87F030000B585B0AE
:10B91000019001AB1846FFF7E1FF0390019B012264
:10B9200002FA03F31946039800F069F800BF05B066
:10B930005DF804FB00B585B0019001AB1846FFF738
:10B94000CDFF0390019B012202FA03F319460398ED
:10B9500000F05FF800BF05B05DF804FB00B585B0EE
:10B96000019001AB1846FFF7B9FF0390039BD3F892
:10B9700004350293029BDA43019B012101FA03F390
:10B980001A40039BC3F80825019B01229A40029BA1
:10B990001A40039BC3F80C2500BF05B05DF804FBFB
:10B9A00000B583B001900091009B002B03D101985A
:10B9B000FFF7C0FF02E00198FFF7A8FF00BF03B048
:10B9C0005DF804FB00B585B0019001AB1846FFF7A8
:10B9D00085FF0390039800F00AF80246019B22FAC3
:10B9E00003F303F00103184605B05DF804FB82B0D1
:10B9F0000190019BD3F80435184602B0704782B01D
:10BA000001900091019B009AC3F8082500BF02B085
:10BA1000704782B001900091019B009AC3F80C25F9
:10BA200000BF02B0704784B00190019B5B09029394
:10BA300000230393029B002B03D14FF0FF330393AA
:10BA400000BF019B03F01F030193039A019B22FA9D
:10BA500003F303F00103002B14BF01230023DBB227
:10BA6000184604B07047000000B585B00190019BF6
:10BA7000032B03D911493A20FCF7B6FA104A019B6F
:10BA800013441B781846FFF79DFF0346002B14BF95
:10BA9000012300238DF80F309DF80F30002B14BFC9
:10BAA00001230023DBB283F00103DBB203F00103C7
:10BAB000DBB2184605B05DF804FB00BFE47F03006D
:10BAC0000C80030000B583B00190019B032B03D9C8
:10BAD00007494120FCF788FA064A019B13441B786A
:10BAE00000211846FFF75CFF00BF03B05DF804FBC0
:10BAF000E47F03000C80030000B583B00190019B3C
:10BB0000032B03D907494720FCF76EFA064A019B2D
:10BB100013441B7801211846FFF742FF00BF03B012
:10BB20005DF804FBE47F03000C80030000B583B0E4
:10BB30000023019305E00198FFF7DEFF019B01332D
:10BB40000193019B032BF6D900BF00BF03B05DF842
:10BB500004FB00B583B00023019305E00198FFF7D3
:10BB6000B1FF019B01330193019B032BF6D900BF69
:10BB700000BF03B05DF804FB00B583B00190019BEA
:10BB8000032B03D907495F20FCF72EFA064A019BD5
:10BB900013441B781846FFF7E1FE00BF03B05DF8C1
:10BBA00004FB00BFE47F03000C80030000B583B0FA
:10BBB0000190019B032B03D90549CB20FCF714FA14
:10BBC000044A019B13441B78184603B05DF804FB3C
:10BBD000E47F03001080030082B003468DF8073035
:10BBE0009DF90730002B13DB9DF8073003F01F028F
:10BBF00009499DF907305B09012000FA02F2203360
:10BC000041F82320BFF34F8F00BFBFF36F8F00BFFA
:10BC100000BF02B0704700BF00E100E0044BD3F862
:10BC20000034002B14BF01230023DBB218467047F9
:10BC30000000014008B507F073FF034683F00103DD
:10BC4000DBB2002B03D109497B20FCF7CDF9FFF7CC
:10BC5000E5FF034683F00103DBB2002B04D000F0C4
:10BC600041FB034B00229A7000BF08BD1C800300FB
:10BC70009832002000B583B000230193184B1B7845
:10BC8000002B02D0852301931CE0154B00229A6003
:10BC9000134B00225A60124B00221A61104B0022F3
:10BCA000DA60104800F0E4FA019007F039FF03462B
:10BCB00083F00103DBB2002B01D000F0FFFA084B48
:10BCC00001221A70FFF7AAFF0346002B02D0044B93
:10BCD00001229A70019B184603B05DF804FB00BF77
:10BCE00098320020BDBD020084B00190019B1B680A
:10BCF0000393039B002B03D0039B1A68019B1A60DC
:10BD0000039B184604B0704700B583B0164B1B78F0
:10BD1000002B04D1154940F21710FCF765F9124BBE
:10BD2000DB68002B04D111494FF48C70FCF75CF9EF
:10BD300000238DF807300DF107031846FCF7BAF819
:10BD4000094BDB68013B084AD360074BDB68002BDB
:10BD500001D1FFF76FFF9DF807301846FCF7C0F8D8
:10BD600000BF03B05DF804FB983200201C80030084
:10BD700000B585B003468DF807309DF80730002BDD
:10BD800002D10C4B039301E00B4B03930398FFF795
:10BD9000ABFF0290029B002B06D0029B5B689DF8D4
:10BDA000072010469847F1E700BF00BF05B05DF8D7
:10BDB00004FB00BFA0320020A832002000B583B0F1
:10BDC00003468DF807309DF80730002B05D10A4B4C
:10BDD00001225A700020FFF7CBFF9DF80730012B9E
:10BDE00005D1054B01229A700120FFF7C1FF00BF6A
:10BDF00003B05DF804FB00BF9832002000B583B0AB
:10BE000001900091019B002B05D1054B01225A7036
:10BE10000020FFF7ADFF00BF03B05DF804FB00BFDB
:10BE20009832002000B585B0034600918DF80730A8
:10BE30009DF80730032B29D0032B35DC002B02D0D3
:10BE4000012B04D030E00020FFF7C6FE2DE00023D8
:10BE50008DF80F300DF10F031846FCF72BF8154B3A
:10BE60001B7883F00103DBB2002B01D0FFF702FF48
:10BE7000104BDB6801330F4AD3600E4B01229A70DE
:10BE80009DF80F301846FCF72BF80EE0094B1B7895
:10BE9000002B04D1084940F25220FCF7A5F800F02D
:10BEA0000DFAFFF731FF00E000BF00BF05B05DF8FD
:10BEB00004FB00BF983200201C80030000B589B04D
:10BEC00001900091009B0793019B1B788DF80C302B
:10BED000019B5B680493019B9B68DBB28DF8143077
:10BEE000019BDB680693074A079B52F823300649FB
:10BEF000079A51F8221003AA1046984700BF09B0CC
:10BF00005DF804FBAC320020B032002000B589B0EF
:10BF100001900091009B0793019B1B788DF80C30DA
:10BF2000019B5B680493019B9B68DBB28DF8143026
:10BF3000019BDB680693074A079B52F823300649AA
:10BF4000079A51F8221003AA1046984700BF09B07B
:10BF50005DF804FBAC320020B032002030B58FB069
:10BF6000039002910192039B1B780C9326490C9B32
:10BF7000019A41F82320029B1A6924490C9B41F83D
:10BF80002320029B5B7F1946214A0C9B13440A46DF
:10BF90001A70029B04AC1D460FCD0FC495E80F002C
:10BFA00084E80F000C9B089300230D93039B1B78E0
:10BFB0001A46174B9B5C002B0DD0039B181D019B51
:10BFC000002B01D0134A00E0002204AB194601F017
:10BFD000DBFE0D9014E0039B1B781A460C4B9B5C18
:10BFE000002B0DD1039B03F10C00019B002B01D012
:10BFF000094A00E0002204AB194601F053F80D9005
:10C000000D9B18460FB030BDAC320020B03200207E
:10C01000B4320020BDBE02000DBF020082B0034654
:10C020008DF807309DF90730002B0CDB9DF80730A9
:10C0300003F01F0205499DF907305B09012000FA52
:10C0400002F241F8232000BF02B0704700E100E097
:10C0500082B0034600918DF807309DF90730002B20
:10C060000ADB009BDAB20C499DF907305201D2B2CB
:10C070000B4483F800230BE0009BDAB207499DF8DC
:10C08000073003F00F03043B5201D2B20B441A767F
:10C0900000BF02B0704700BF00E100E000ED00E02B
:10C0A00082B00190019B1B0B5BB2184602B0704737
:10C0B00000B583B003460A468DF8073013468DF865
:10C0C00006309DF80630012B03D99DF80630032B6E
:10C0D0000BD99DF80630042B03D99DF80630072BA9
:10C0E00003D908496B20FBF77FFF9DF806209DF9D7
:10C0F000073011461846FFF7ABFF00BF03B05DF8ED
:10C1000004FB00BF5480030000B583B003468DF8E4
:10C1100007309DF907301846FFF780FF00BF03B0D6
:10C120005DF804FB82B003468DF807300F4A9DF995
:10C130000730002B00DA1F335B115BB252F823206B
:10C140009DF90730594203F01F0301F01F0158BF4A
:10C150004B425BB222FA03F303F00103002B14BF3E
:10C1600001230023DBB2184602B0704700E100E073
:10C1700082B001904FF08042019BC2F8083300BFAB
:10C1800002B0704782B003468DF807309DF8073043
:10C1900003F1804301221A6000BF02B0704784B0EF
:10C1A0000346ADF80630BDF8063003F180430022A7
:10C1B0001A60BDF8063003F180431B680393039BAC
:10C1C00000BF04B0704782B00346ADF80630BDF83A
:10C1D000063003F180431B68002B14BF01230023AA
:10C1E000DBB2184602B0704782B001904FF0804237
:10C1F000019BC2F8183500BF02B070474FF0804372
:10C20000D3F818341B0C03F00103002B14BF0123D7
:10C210000023DBB21846704700B583B006238DF8C3
:10C2200007304FF08040FFF73BFF03461846FFF70B
:10C2300079FF034683F00103DBB2002B13D04FF0EC
:10C240008040FFF72DFF03461A469DF80730194638
:10C250001046FFF72DFF4FF08040FFF721FF034608
:10C260001846FFF751FF00BF03B05DF804FB000064
:10C2700000B585B00190019B002B03D10D49A4208E
:10C28000FBF7B2FE002303930B4B1B79002B02D06C
:10C290008523039308E0084A019B1360064B0122A3
:10C2A0001A71054B00225A71039B184605B05DF8C0
:10C2B00004FB00BF88800300B832002008B5074B9C
:10C2C0001B79002B03D10649BD20FBF78DFEFFF73C
:10C2D000A3FF0120FFF788FF00BF08BDB832002090
:10C2E0008880030008B50D4B1B79002B03D10C4946
:10C2F000F720FBF779FE0220FFF73AFF4FF4827038
:10C30000FFF74DFF0C20FFF73DFF00BFFFF776FF63
:10C310000346002BFAD100BF00BF08BDB832002091
:10C320008880030008B54FF48070FFF74CFF034688
:10C33000002B14D04FF48070FFF731FF0120FFF77E
:10C3400017FF114B5B7983F00103DBB2002B06D0A2
:10C350000D4B01225A710C4B1B68002098474FF47B
:10C360008270FFF730FF0346002B0AD04FF4827033
:10C37000FFF715FF0220FFF7FBFE034B1B680120B0
:10C38000984700BF08BD00BFB832002000B583B099
:10C390000346ADF80630BDF80630184600F026F822
:10C3A00003461B68012B0CBF01230023DBB2184698
:10C3B00003B05DF804FB00B585B00346ADF8063068
:10C3C000BDF80630184600F011F803461A4600235F
:10C3D0001360BDF80630184600F008F803461B68E5
:10C3E0000393039B00BF05B05DF804FB82B00346D6
:10C3F000ADF80630BDF8063003F1804303F5C043C5
:10C40000184602B07047000082B00190034BD3F889
:10C410000423019B1340184602B07047006000409F
:10C4200082B00190054A019B03F5A27352F82330B4
:10C430001B0A03F01F03184602B07047006000405B
:10C4400082B00190064A019B03F5A27352F8233093
:10C450001B0C03F00303DBB2184602B0704700BFA9
:10C460000060004000B583B00190019B1B68184636
:10C4700000F096F80346002B04D105494FF4F670FE
:10C48000FBF7B2FD4FF0A043184603B05DF804FB84
:10C49000E880030000B585B001900B468DF80330AD
:10C4A00001AB1846FFF7DEFF0390019A039B02F5EC
:10C4B000E07253F82230019A23F44031039B02F5D5
:10C4C000E07243F82210019A039B02F5E07253F8E0
:10C4D00022309DF8032012041146019A1943039B50
:10C4E00002F5E07243F8221000BF05B05DF804FBCE
:10C4F00000B585B0019001AB1846FFF7B3FF03907C
:10C50000019A039B02F5E07253F822301B0C03F0F2
:10C510000303DBB2184605B05DF804FB86B0039058
:10C52000029101924FF0A0430493039B059319E0FD
:10C53000059B9B0006AA134453F8083CD3F820251A
:10C54000019B1A60059B9B0006AA134453F8083C04
:10C55000019A1268C3F82025019B04330193059BBF
:10C5600001330593039A029B1344059A9A42DFD341
:10C5700000BF00BF06B0704700B585B0019001ABA9
:10C580001846FFF76FFF0390019B012202FA03F3A5
:10C590001A46039BC3F8202500BF05B05DF804FBD5
:10C5A00084B00190019B5B09029300230393029BDB
:10C5B000002B03D14FF0FF33039300BF019B03F027
:10C5C0001F030193039A019B22FA03F303F0010373
:10C5D000002B14BF01230023DBB2184604B07047C0
:10C5E00084B001900091009B0393019BDB080293B0
:10C5F000019B03F0070301930122019B02FA03F35D
:10C600000399029A0A4412781340184604B07047FE
:10C6100082B00190044A019B1344303393F90030F7
:10C62000184602B0704700BFC032002082B00190AF
:10C63000034A019B52F82330184602B0704700BFEE
:10C64000C032002084B00190074A019B134450334C
:10C6500093F900308DF80F309DF80F3023F0C003B0
:10C66000184604B0704700BFC032002084B001906B
:10C67000074A019B1344503393F900308DF80F3073
:10C680009DF80F309B09DBB2184604B0704700BF1D
:10C69000C032002000B585B00190019A0121002030
:10C6A000FFF73CFF002303930BE0039B9B00019AE1
:10C6B00013441B68002B01D0012306E0039B0133C8
:10C6C0000393039B002BF0D00023184605B05DF8C0
:10C6D00004FB000000B587B00190002305935BE0E8
:10C6E000344A059B1344503393F90030B3F1FF3FB4
:10C6F0004ED00598FFF7A6FF049001990498FFF724
:10C700006FFF0346002B44D00598FFF7AFFF0346A9
:10C710008DF80F300498FFF7EBFE03468DF80E30CE
:10C720009DF80E30022B01D1032300E002238DF887
:10C730000D309DF80D3019460498FFF7ABFE0498B4
:10C74000FFF71AFF0498FFF763FF03461846FFF749
:10C750006DFF0290029B002B1BD09DF80F30032B26
:10C760000FD09DF80E30022B03D19DF80F30012B16
:10C7700007D09DF80E30032B0BD19DF80F30022B04
:10C7800007D19DF80F20029B11460498984700E0BE
:10C7900000BF059B01330593059B032BA0D901988E
:10C7A000FFF778FF0346002B97D100BF00BF07B00B
:10C7B0005DF804FBC032002000B589B00023069369
:10C7C000002300934FF48073ADF8123001230793D8
:10C7D0000023059321E0BDF812301846FFF7D6FD7F
:10C7E0000346002B0ED00798FFF70EFE0346002BE2
:10C7F00008D0BDF812301846FFF7DDFD069A079BFA
:10C8000013430693079B5B000793BDF81230043374
:10C81000ADF81230059B01330593059B072BDAD940
:10C820004FF4BE70FFF7B2FD0346002B0DD04FF45E
:10C83000BE70FFF7C0FD069B43F0004306936B46B6
:10C840001A4601210020FFF769FE069BDBB2002B90
:10C8500029D0012307930023059321E0079A069B23
:10C860001340002B16D00598FFF7DAFD03900598CA
:10C87000FFF7E6FD03468DF80B300598FFF7D6FE6F
:10C880000190019B002B05D09DF80B20019B1146C8
:10C8900003989847079B5B000793059B013305931B
:10C8A000059B072BDAD9069B002B03DA6B4618464B
:10C8B000FFF710FF00BF09B05DF804FB08B5064B99
:10C8C0001B68002B03D105495120FBF78DFB024B60
:10C8D0001B68984700BF08BD1C330020548103002B
:10C8E00082B00190019B044A934201D1034B00E0C6
:10C8F0000023184602B07047002000401C3300207F
:10C9000000B587B001900091019B002B03D11C4919
:10C910007720FBF769FB0198FFF7E2FF0590059B85
:10C92000002B25D000238DF8133000238DF80B3019
:10C930000DF10B031846FBF7BDFA059B1B79002B85
:10C9400003D001238DF8133005E0059B009A1A608F
:10C95000059B01221A719DF80B301846FBF7C0FAAF
:10C960009DF81330002B03D011230393039B02E0A7
:10C9700000230393039B184607B05DF804FB00BF38
:10C980005481030000B585B00190019B002B03D1B9
:10C990000A499B20FBF728FB0198FFF7A1FF0390B2
:10C9A000039B002B05D0039B00221A60039B0022EF
:10C9B0001A7100BF05B05DF804FB00BF548103008D
:10C9C00082B003468DF807309DF90730002B0CDB51
:10C9D0009DF8073003F01F0205499DF907305B09F8
:10C9E000012000FA02F241F8232000BF02B0704794
:10C9F00000E100E082B003468DF807309DF9073072
:10CA0000002B13DB9DF8073003F01F0209499DF945
:10CA100007305B09012000FA02F2203341F823209D
:10CA2000BFF34F8F00BFBFF36F8F00BF00BF02B0D7
:10CA3000704700BF00E100E082B0034600918DF82E
:10CA400007309DF90730002B0ADB009BDAB20C4956
:10CA50009DF907305201D2B20B4483F800230BE05A
:10CA6000009BDAB207499DF8073003F00F03043B3F
:10CA70005201D2B20B441A7600BF02B0704700BF19
:10CA800000E100E000ED00E082B00190019B1B0B93
:10CA90005BB2184602B0704700B583B003460A4641
:10CAA0008DF8073013468DF806309DF80630012BBF
:10CAB00003D99DF80630032B0BD99DF80630042BC3
:10CAC00003D99DF80630072B03D908496B20FBF7E3
:10CAD0008BFA9DF806209DF9073011461846FFF79E
:10CAE000ABFF00BF03B05DF804FB00BF8C81030007
:10CAF00000B583B003468DF807309DF9073018461E
:10CB0000FFF75EFF00BF03B05DF804FB00B583B024
:10CB100003468DF807309DF907301846FFF76AFF86
:10CB200000BF03B05DF804FB84B001900B46ADF884
:10CB30000230BDF80230019A134400221A60BDF899
:10CB40000230019A13441B680393039B00BF04B097
:10CB5000704782B001900B46ADF80230BDF802304C
:10CB6000019A13441B68002B14BF01230023DBB27E
:10CB7000184602B0704782B001900091019B009A64
:10CB8000C3F8042300BF02B0704782B00190009147
:10CB9000019BD3F80423009B1340002B14BF0123F7
:10CBA0000023DBB2184602B0704782B001900091BA
:10CBB000019B009AC3F8082300BF02B0704784B0FD
:10CBC0000190019BD3F880340393019B039AC3F82F
:10CBD0008024039B184604B0704782B00190019BEB
:10CBE0000422C3F8002500BF02B0704782B0019054
:10CBF000019B0022C3F8002500BF02B0704784B03B
:10CC0000039002910192039B019AC3F81425039BA0
:10CC1000029AC3F80C2500BF04B0704700B583B07A
:10CC200001904FF0FF324FF0FF310198FFF7E7FF1F
:10CC300000BF03B05DF804FB82B00190019BD3F804
:10CC40000C35184602B0704782B00190019BD3F8B2
:10CC50001435184602B0704782B00190019BD3F89A
:10CC60000835184602B0704782B00190019BD3F896
:10CC70001035184602B0704784B0039002910192BB
:10CC8000039B029AC3F80825039B019AC3F8102559
:10CC900000BF04B0704700B583B001904FF0FF3281
:10CCA0004FF0FF310198FFF7E7FF00BF03B05DF8D9
:10CCB00004FB82B00190019BD3F81835DBB2184613
:10CCC00002B0704782B001900B468DF803309DF89A
:10CCD0000320019BC3F81C2500BF02B0704782B03F
:10CCE00001900B468DF803309DF80330019A1344F0
:10CCF00001221A6000BF02B0704782B001900B465B
:10CD00008DF8033013468DF802309DF803209DF80E
:10CD100002301343DBB21A46019BC3F86C2500BFF7
:10CD200002B0704782B001900091019B009AC3F855
:10CD3000242500BF02B0704700B583B00190019B6D
:10CD40001B68184600F096F80346002B04D10549ED
:10CD50004FF4F670FBF748F94FF0A043184603B0C4
:10CD60005DF804FBB881030000B585B0019008466A
:10CD700011461A4603468DF803300B468DF80230F3
:10CD800013468DF8013001AB1846FFF7D5FF03902D
:10CD90009DF803209DF802305B001A439DF8013096
:10CDA0009B001A439DF818301B0242EA03019DF8CC
:10CDB0001C301B04019A1943039B02F5E07243F8EF
:10CDC000221000BF05B05DF804FB00B585B00390EC
:10CDD00000230193002300930023012201210398E3
:10CDE000FFF7C2FF00BF05B05DF804FB00B585B0DA
:10CDF00003900B468DF80B309DF80B30002201920A
:10CE000000220092002200210398FFF7ADFF00BF2F
:10CE100005B05DF804FB00B585B0039000230193D5
:10CE2000002300930023012200210398FFF79CFFB9
:10CE300000BF05B05DF804FB00B585B0019001AB03
:10CE40001846FFF779FF0390019B012202FA03F3D2
:10CE50001946039800F004F800BF05B05DF804FB24
:10CE600082B001900091019B009AC3F8082500BF91
:10CE700002B0704784B00190019B5B0902930023CC
:10CE80000393029B002B03D14FF0FF33039300BFAA
:10CE9000019B03F01F030193039A019B22FA03F302
:10CEA00003F00103002B14BF01230023DBB218465B
:10CEB00004B0704700B583B001900091009B1B68DF
:10CEC000B3F1FF3F09D0009B1B681846FFF7B4FF82
:10CED000009B1B681846FFF778FF009B5B68B3F167
:10CEE000FF3F05D0009B5B6800211846FFF77EFFDF
:10CEF000019B1A68009B9B6919461046FFF712FFB9
:10CF0000019B1868009B597D009B1B7D1A46FFF70B
:10CF1000F4FE019B1868009B1968009B5B681A4629
:10CF2000FFF76DFE009B1B7D012B22D1009B9B68B0
:10CF3000B3F1FF3F05D0009B9B6800211846FFF727
:10CF400055FF009BDB68B3F1FF3F09D0009BDB6816
:10CF50001846FFF771FF009BDB681846FFF735FFA7
:10CF6000019B1868009BD968009B9B681A46FFF7D5
:10CF700083FE00BF03B05DF804FB000000B583B082
:10CF800001900B468DF80330019B1B684FF48E71A6
:10CF90001846FFF7C9FD019B1B684FF4A2711846A4
:10CFA000FFF7C2FD019B1B680E491846FFF7E3FD22
:10CFB000019B1B681846FFF767FD03461A469DF85C
:10CFC000033019461046FFF767FD019B1B681846A2
:10CFD000FFF75AFD03461846FFF78AFD00BF03B06E
:10CFE0005DF804FB8000020000B583B00190019B56
:10CFF0001B6808491846FFF7D8FD019B1B681846B7
:10D00000FFF742FD03461846FFF780FD00BF03B05F
:10D010005DF804FB8402020000B587B00190019B1B
:10D020001B681846FFF708FE0590019B1B68184611
:10D03000FFF70AFE0490019B1B681846FFF70CFEE1
:10D040000390019B1B681846FFF70EFE0290019BA0
:10D050001B681846FFF7E2FD019B1B681846FFF7A7
:10D060001AFE059BB3F1FF3F02D00598FFF7D3FEF0
:10D07000049BB3F1FF3F02D00498FFF7CCFE029B64
:10D08000B3F1FF3F02D00298FFF7C5FE039BB3F157
:10D09000FF3F02D00398FFF7BEFE00BF07B05DF868
:10D0A00004FB000000B587B0039002910192029B3F
:10D0B000002B03D12D49AA20FAF796FF039B1B7979
:10D0C0001A462C2302FB03F3294A1344049300233A
:10D0D0000593049B93F82A30002B03D00823059373
:10D0E000059B3EE0039B1A68039B1B791946214B65
:10D0F00053F8213019461046FFF702FC0346002B77
:10D1000003D011230593059B2BE002990398FFF7A9
:10D11000D1FE049B019A5A60029B1A69049B1A6013
:10D12000049B5B68002B05D0029B1B7F194603986C
:10D13000FFF724FF039B1B681846FFF74EFD049B77
:10D1400000229A61049B0022DA61049B002283F88A
:10D150002920049B00225A61049B012283F82A2083
:10D16000059B184607B05DF804FB00BFEC81030087
:10D17000243300202082030000B585B00190019B7C
:10D180001B791A462C2302FB03F3114A1344039321
:10D19000019B1B681846FFF729FD039B5B68002B6A
:10D1A00002D00198FFF720FF0198FFF735FF019BA0
:10D1B0001B681846FFF7E6FB039B002283F82A2032
:10D1C000039B00225A6000BF05B05DF804FB00BF5E
:10D1D0002433002000B585B0019000914FF48E718A
:10D1E0000198FFF7A1FC009B9A68009B1B6A1344FF
:10D1F0001B788DF80F30009B1B6A5A1C009B1A622B
:10D200009DF80F3019460198FFF75CFD00BF05B08F
:10D210005DF804FB00B585B001900091009B5B694F
:10D22000039316E0009B93F82830DBB2002B01D06B
:10D23000002314E04FF48E710198FFF78AFC034637
:10D2400083F00103DBB2002BECD100990198FFF7CA
:10D25000C1FF009B1B6A039A9A42EBD80123184630
:10D2600005B05DF804FB000000B587B003900291A3
:10D270000192039B1B791A462C2302FB03F33C4AC1
:10D2800013440493049B93F82A30012B04D03949AA
:10D290004FF48C70FAF7A8FE029B002B04D135499D
:10D2A00040F21910FAF7A0FE019B002B04D131497E
:10D2B0004FF48D70FAF798FE039800F05DF803467E
:10D2C000002B03D011230593059B4CE0049B019A8E
:10D2D0005A61049B029A9A60049B00221A62049B82
:10D2E000002283F8282000230593039B1B684FF43A
:10D2F0008E711846FFF718FC039B1B68082118461F
:10D30000FFF7EDFC039B1B6804991846FFF762FFCB
:10D31000049B5B68002B25D1039B1B68049918466E
:10D32000FFF778FF034683F00103DBB2002B02D046
:10D330000F23059313E000BF039B1B684FF48E710E
:10D340001846FFF706FC034683F00103DBB2002B0F
:10D35000F2D1039B1B680C211846FFF7C0FC049B0D
:10D3600000225A61059B184607B05DF804FB00BF18
:10D3700024330020EC81030082B00190019B1B79D3
:10D380001946074A2C2301FB03F3134414331B688B
:10D39000002B14BF01230023DBB2184602B07047F4
:10D3A0002433002010B582B001900091009B9B694E
:10D3B000002B08D14FF484710198FFF7B5FB019859
:10D3C000FFF777FC13E04FF484710198FFF7ACFB93
:10D3D000009BDA68009B5B6AD4180198FFF769FC30
:10D3E00003462370009B5B6A5A1C009B5A6202B082
:10D3F00010BD00B589B003900291019201238DF810
:10D400001030029B0693019B0593039B5B68039A74
:10D41000116804AA1046984700BF09B05DF804FBE4
:10D4200000B587B00190009100238DF80830009B73
:10D430000493019B9B680393019B00225A61019B0B
:10D440005B68019A116802AA1046984700BF07B0AE
:10D450005DF804FB00B58BB0019000914FF40071B2
:10D460000198FFF792FB0346002B39D04FF49271DD
:10D470000198FFF76EFB0346002B31D04FF49271F9
:10D480000198FFF751FB4FF401710198FFF78DFBF5
:10D49000009B93F8293083F00103DBB2002B03D00B
:10D4A00004210198FFF71BFC02238DF80C30019832
:10D4B000FFF785FB03460693009B9B690593009B42
:10D4C000DB680493009B00229A61009B0022DA61D2
:10D4D000009B5B68009A116803AA1046984752E0C7
:10D4E00004210198FFF751FB0346002B4BD04FF46A
:10D4F00084710198FFF72DFB0346002B43D0009960
:10D500000198FFF74FFF009B9A69009B5B6A9A4264
:10D5100039D1009BDB69002B19D0009BDB68099394
:10D52000009B5B6A0893009BDA69009B9A61009BF1
:10D530001A69009BDA60009B0022DA61009B0022DE
:10D540005A62099A08990098FFF753FF1BE0009B65
:10D5500093F8293083F00103DBB2002B03D00421C0
:10D560000198FFF7BCFB4FF401710198FFF71DFB19
:10D57000009B00229A61009B596A009BDB681A4657
:10D580000098FFF736FF4FF48E710198FFF7E1FA2C
:10D590000346002B24D0009B5B690793009B1B6A0A
:10D5A000079A9A420DD9009B93F82830DBB283F09A
:10D5B0000103DBB2002B04D000990198FFF70AFEAB
:10D5C0000EE04FF48E710198FFF7AEFA009B5B6995
:10D5D000002B05D0009B5B6919460098FFF720FFE0
:10D5E0004FF4A2710198FFF7B4FA0346002B1CD048
:10D5F0004FF4A2710198FFF797FA009B93F8293036
:10D60000002B03D000210198FFF769FB009B9B6969
:10D61000002B0AD0009B00229A61009B596A009B54
:10D62000DB681A460098FFF7E4FE00BF0BB05DF818
:10D6300004FB000008B503490348FFF70BFF00BFD8
:10D6400008BD00BF243300200020004082B0034604
:10D650008DF807309DF90730002B0CDB9DF8073063
:10D6600003F01F0205499DF907305B09012000FA0C
:10D6700002F241F8232000BF02B0704700E100E051
:10D6800082B003468DF807309DF90730002B13DB7D
:10D690009DF8073003F01F0209499DF907305B0927
:10D6A000012000FA02F2203341F82320BFF34F8F0C
:10D6B00000BFBFF36F8F00BF00BF02B0704700BF55
:10D6C00000E100E082B0034600918DF807309DF93B
:10D6D0000730002B0ADB009BDAB20C499DF90730BA
:10D6E0005201D2B20B4483F800230BE0009BDAB264
:10D6F00007499DF8073003F00F03043B5201D2B2F3
:10D700000B441A7600BF02B0704700BF00E100E092
:10D7100000ED00E082B00190019B03F06043B3F1A3
:10D72000005F0CBF01230023DBB2184602B0704734
:10D7300082B00190019B1B0B5BB2184602B0704790
:10D7400000B583B003460A468DF8073013468DF8BE
:10D7500006309DF80630012B03D99DF80630032BC7
:10D760000BD99DF80630042B03D99DF80630072B02
:10D7700003D908496B20FAF737FC9DF806209DF97C
:10D78000073011461846FFF79DFF00BF03B05DF854
:10D7900004FB00BF2482030000B583B003468DF86C
:10D7A00007309DF907301846FFF750FF00BF03B060
:10D7B0005DF804FB00B583B003468DF807309DF992
:10D7C00007301846FFF75CFF00BF03B05DF804FBAD
:10D7D00084B001900B46ADF80230BDF80230019ADA
:10D7E000134400221A60BDF80230019A13441B68EA
:10D7F0000393039B00BF04B0704782B001900B46B7
:10D80000ADF80230BDF80230019A13441B68002BBA
:10D8100014BF01230023DBB2184602B0704782B068
:10D8200001900091019BD3F80022009BDB431A403A
:10D83000019BC3F8002200BF02B0704782B0019084
:10D840000091019B009AC3F8042300BF02B0704707
:10D8500082B001900091019B009AC3F8082300BF99
:10D8600002B0704784B00190019BD3F880340393D9
:10D87000019B039AC3F88024039B184604B07047A9
:10D8800082B00190019B0822C3F8002500BF02B0BE
:10D89000704782B00190019B0022C3F8002500BFB1
:10D8A00002B0704784B0039002910192039B029AE8
:10D8B000C3F80C25039B019AC3F8142500BF04B0DC
:10D8C000704700B583B001904FF0FF324FF0FF3149
:10D8D0000198FFF7E7FF00BF03B05DF804FB82B0DB
:10D8E0000190019BD3F80C35184602B0704782B006
:10D8F0000190019BD3F81435184602B0704782B0EE
:10D900000190019BD3F80835184602B0704782B0E9
:10D910000190019BD3F81035184602B0704784B0CF
:10D92000039002910192039B029AC3F80825039B7E
:10D93000019AC3F8102500BF04B0704700B583B04A
:10D9400001904FF0FF324FF0FF310198FFF7E7FFF2
:10D9500000BF03B05DF804FB82B001900B468DF868
:10D9600003309DF80330019A134401221A6000BF6E
:10D9700002B0704782B001900B468DF80330134619
:10D980008DF802309DF803209DF802301343DBB27E
:10D990001A46019BC3F86C2500BF02B0704782B0E5
:10D9A00001900091019B009AC3F8242500BF02B0AA
:10D9B000704784B0039002910192029A039BC3F8CE
:10D9C0004425039B019AC3F8482500BF04B0704763
:10D9D00082B00190019BD3F84C35184602B07047D5
:10D9E00082B00190019BD3F83C35184602B07047D5
:10D9F00000B583B00190019B1B68184600F096F8B3
:10DA00000346002B04D105494FF4F670FAF7ECFAFF
:10DA10004FF0A043184603B05DF804FB50820300AA
:10DA200000B585B00190084611461A4603468DF8A8
:10DA300003300B468DF8023013468DF8013001ABF0
:10DA40001846FFF7D5FF03909DF803209DF802309C
:10DA50005B001A439DF801309B001A439DF8183073
:10DA60001B0242EA03019DF81C301B04019A194372
:10DA7000039B02F5E07243F8221000BF05B05DF889
:10DA800004FB00B585B003900023019300230093AD
:10DA90000023012201210398FFF7C2FF00BF05B058
:10DAA0005DF804FB00B585B003900B468DF80B3094
:10DAB0009DF80B30002201920022009200220021EA
:10DAC0000398FFF7ADFF00BF05B05DF804FB00B59C
:10DAD00085B00390002301930023009300230122CB
:10DAE00000210398FFF79CFF00BF05B05DF804FB21
:10DAF00000B585B0019001AB1846FFF779FF0390A0
:10DB0000019B012202FA03F31946039800F004F87E
:10DB100000BF05B05DF804FB82B001900091019B4D
:10DB2000009AC3F8082500BF02B0704784B0019086
:10DB3000019B5B09029300230393029B002B03D1FB
:10DB40004FF0FF33039300BF019B03F01F030193CA
:10DB5000039A019B22FA03F303F00103002B14BF85
:10DB600001230023DBB2184604B0704700B583B030
:10DB700001900091009B1B68B3F1FF3F09D0009B0F
:10DB80001B681846FFF7B4FF009B1B681846FFF799
:10DB900078FF009B5B68B3F1FF3F05D0009B5B689B
:10DBA00000211846FFF77EFF019B1A68009B9B69C6
:10DBB00019461046FFF7F3FE019B1868009B597D3C
:10DBC000009B1B7D1A46FFF7D5FE019B1868009B42
:10DBD0001968009B5B681A46FFF764FE009B1B7D7B
:10DBE000012B22D1009B9B68B3F1FF3F05D0009B26
:10DBF0009B6800211846FFF755FF009BDB68B3F1D7
:10DC0000FF3F09D0009BDB681846FFF771FF009BC0
:10DC1000DB681846FFF735FF019B1868009BD96841
:10DC2000009B9B681A46FFF77AFE00BF03B05DF8C1
:10DC300004FB000000B583B001900B468DF8033063
:10DC4000019B1B684FF488711846FFF7C1FD019BCB
:10DC50001B684FF490711846FFF7BAFD019B1B68D3
:10DC60004FF492711846FFF7B3FD019B1B684FF408
:10DC7000A2711846FFF7ACFD019B1B684FF4AC7115
:10DC80001846FFF7A5FD019B1B680F491846FFF7D3
:10DC9000D5FD019B1B681846FFF74AFD03461A464F
:10DCA0009DF8033019461046FFF74AFD019B1B689B
:10DCB0001846FFF73DFD03461846FFF76DFD00BF10
:10DCC00003B05DF804FB00BF1003420000B583B051
:10DCD0000190019B1B6808491846FFF7B9FD019B9D
:10DCE0001B681846FFF724FD03461846FFF762FD40
:10DCF00000BF03B05DF804FB1003420000B587B01D
:10DD00000190019B1B681846FFF7E9FD0590019BF8
:10DD10001B681846FFF7EBFD0490019B1B68184633
:10DD2000FFF7EDFD0390019B1B681846FFF7EFFD21
:10DD30000290019B1B681846FFF7C3FD019B1B68FF
:10DD40001846FFF7FBFD059BB3F1FF3F02D0059896
:10DD5000FFF7BDFE049BB3F1FF3F02D00498FFF72D
:10DD6000B6FE029BB3F1FF3F02D00298FFF7AFFE71
:10DD7000039BB3F1FF3F02D00398FFF7A8FE00BF5B
:10DD800007B05DF804FB000000B587B00390029176
:10DD90000192029B002B03D12B49CF20FAF724F9E3
:10DDA000039B1B791A461346DB0013449B00274A4A
:10DDB0001344049300230593049B93F82030002B15
:10DDC00003D008230593059B3AE0039B1A68039B45
:10DDD0001B7919461E4B53F8213019461046FEF7A1
:10DDE0008FFD0346002B03D011230593059B27E0ED
:10DDF00002990398FFF7BAFE049B019A5A60029BAE
:10DE00001A69049B1A60049B5B68002B05D0029B77
:10DE10001B7F19460398FFF70DFF039B1B681846ED
:10DE2000FFF72EFD049B00229A61049B0022DA6119
:10DE3000049B00225A61049B012283F82020059B49
:10DE4000184607B05DF804FB8482030050330020BD
:10DE5000B882030000B585B00190019B1B791A467A
:10DE60001346DB0013449B002A4A13440393019B8F
:10DE70001B680293039B5B68002B02D00198FFF79D
:10DE800025FF20210298FFF7CAFC039B9B69002B0A
:10DE900008D04FF4A2710298FFF79AFC042102986F
:10DEA000FFF75AFD4FF4AC710298FFF791FC0C217B
:10DEB0000298FFF751FD00BF4FF4AC710298FFF7D5
:10DEC0009CFC034683F00103DBB2002BF4D1039BDF
:10DED0009B69002B0AD04FF4A2710298FFF78DFCCA
:10DEE000034683F00103DBB2002BE5D10298FFF774
:10DEF000D0FC0198FFF702FF0298FEF743FD039B59
:10DF0000002283F82020039B00225A6000BF05B046
:10DF10005DF804FB5033002000B589B003900291F6
:10DF20000192039B1B791A461346DB0013449B00A6
:10DF3000564A13440593059B93F82030012B04D0D7
:10DF4000534940F25310FAF74FF8029B002B04D1CB
:10DF50004F494FF4AA70FAF747F8019B002B04D100
:10DF60004B4940F25510FAF73FF8039B1B79002B01
:10DF700002D1019BFF2B04D945494FF4AB70FAF74E
:10DF800033F80298FFF7C6FB034683F00103DBB2C8
:10DF9000002B03D010230793079B73E0039800F036
:10DFA00079F80346002B03D011230793079B69E000
:10DFB000059B019A5A61059B029A9A600023079378
:10DFC000039B1B684FF490711846FFF701FC039BFD
:10DFD0001B684FF4AC711846FFF7FAFB039B1868F7
:10DFE000059B9968059B5B691A46FFF7E2FC039B5A
:10DFF0001B6808211846FFF7AFFC059B5B68002BE8
:10E000003FD1039B1B684FF490711846FFF7F5FB57
:10E0100003468DF81B30039B1B684FF4AC71184608
:10E02000FFF7EBFB03468DF81A309DF81B3083F0A9
:10E030000103DBB2002B06D09DF81A3083F00103F8
:10E04000DBB2002BDDD19DF81A30002B02D00F235C
:10E05000079313E0039B1B680C211846FFF77CFC19
:10E0600000BF039B1B684FF4AC711846FFF7C5FB5C
:10E07000034683F00103DBB2002BF2D1059B0022A3
:10E080005A61079B184609B05DF804FB5033002025
:10E090008482030082B00190019B1B791946084AD3
:10E0A0000B46DB000B449B00134414331B68002B0E
:10E0B00014BF01230023DBB2184602B0704700BF33
:10E0C0005033002000B589B00390029101920123E2
:10E0D0008DF81030029B0693019B0593039B5B68B0
:10E0E000039A116804AA1046984700BF09B05DF86A
:10E0F00004FB00B587B00190009100238DF8083033
:10E10000009B0493019B9B680393019B00225A612F
:10E11000019B5B68019A116802AA1046984700BFEC
:10E1200007B05DF804FB00B589B0019000914FF491
:10E1300092710198FFF761FB0346002B22D04FF448
:10E1400092710198FFF744FB02238DF80830019883
:10E15000FFF788FB034605930198FFF741FC034650
:10E160000493009BDB680393009B00229A61009B51
:10E170000022DA61009B5B68009A116802AA1046CF
:10E1800098473BE04FF488710198FFF736FB034650
:10E19000002B33D04FF488710198FFF719FB0198D9
:10E1A000FFF71EFC0790009B9B69079A9A4225D1B6
:10E1B000009BDB69002B17D0009BDB6806932021B6
:10E1C0000198FFF72CFB009BDA69009B9A61009B8A
:10E1D0001A69009BDA60009B0022DA61069A0799AF
:10E1E0000098FFF76FFF09E0009B00229A61009BF7
:10E1F000DB681A4607990098FFF764FF4FF4A27195
:10E200000198FFF7FAFA0346002B18D04FF4A271D9
:10E210000198FFF7DDFA009B9B69002B0FD0009B54
:10E2200000229A61009B0022DA610198FFF7D8FB77
:10E230000146009BDB681A460098FFF743FF4FF446
:10E2400090710198FFF7D9FA0346002B14D04FF4D0
:10E2500090710198FFF7BCFA0C210198FFF77CFB45
:10E26000009B5B69002B07D00198FFF7B1FB0346C9
:10E2700019460098FFF73DFF4FF4AC710198FFF786
:10E28000BCFA0346002B10D04FF4AC710198FFF795
:10E290009FFA009B5B69002B07D00198FFF798FB62
:10E2A000034619460098FFF724FF00BF09B05DF848
:10E2B00004FB000008B503490348FFF734FF00BF23
:10E2C00008BD00BF503300200020004000B589B0D9
:10E2D00001900091009B0793019B1B788DF80830FB
:10E2E000019B5B680393019B9B68DBB28DF8103048
:10E2F000019BDB680593019B1B69DBB28DF818302D
:10E30000074A079B52F823300649079A51F8221012
:10E3100002AA1046984700BF09B05DF804FB00BF91
:10E32000743300208033002010B58AB0039002912E
:10E3300001920093039B1B7809932249099B019A40
:10E3400041F823202049099B009A41F8232000230B
:10E3500008931E4B04AC0FCB84E80F00029B1B7884
:10E360008DF81030029B5B788DF81130029B9B7802
:10E370008DF81230029BDB788DF81330029B1B79ED
:10E380008DF81530029B5B798DF81630029B9B68E7
:10E390000693029B1B7B8DF81C30029B5B7B8DF8E8
:10E3A0001D30039B181D019B002B01D0084A00E083
:10E3B0000022099B04A900F0A5FA0890089B1846C2
:10E3C0000AB010BD7433002080330020BC820300EB
:10E3D000CDE2020082B003468DF807309DF9073088
:10E3E000002B0CDB9DF8073003F01F0205499DF957
:10E3F00007305B09012000FA02F241F8232000BF38
:10E4000002B0704700E100E082B003468DF80730AB
:10E410009DF90730002B13DB9DF8073003F01F0236
:10E4200009499DF907305B09012000FA02F2203307
:10E4300041F82320BFF34F8F00BFBFF36F8F00BFA2
:10E4400000BF02B0704700BF00E100E082B00346A9
:10E4500000918DF807309DF90730002B0ADB009BF7
:10E46000DAB20C499DF907305201D2B20B4483F85D
:10E4700000230BE0009BDAB207499DF8073003F058
:10E480000F03043B5201D2B20B441A7600BF02B014
:10E49000704700BF00E100E000ED00E082B00190B5
:10E4A000019B03F06043B3F1005F0CBF0123002325
:10E4B000DBB2184602B0704782B00190019B1B0B83
:10E4C0005BB2184602B0704700B583B003460A46F7
:10E4D0008DF8073013468DF806309DF80630012B75
:10E4E00003D99DF80630032B0BD99DF80630042B79
:10E4F00003D99DF80630072B03D908496B20F9F79B
:10E5000073FD9DF806209DF9073011461846FFF768
:10E510009DFF00BF03B05DF804FB00BFCC82030089
:10E5200000B583B003468DF807309DF907301846D3
:10E53000FFF750FF00BF03B05DF804FB00B583B0E8
:10E5400003468DF807309DF907301846FFF75CFF4A
:10E5500000BF03B05DF804FB82B001900B468DF85C
:10E5600003309DF80330019A134401221A6000BF62
:10E5700002B0704784B001900B46ADF80230BDF890
:10E580000230019A134400221A60BDF80230019A49
:10E5900013441B680393039B00BF04B0704782B011
:10E5A00001900B46ADF80230BDF80230019A1344D9
:10E5B0001B68002B14BF01230023DBB2184602B0F6
:10E5C000704782B001900091019B009AC3F8042328
:10E5D00000BF02B0704782B001900091019B009A89
:10E5E000C3F8082300BF02B0704782B00190019BBE
:10E5F0000722C3F8002500BF02B0704782B0019027
:10E60000019B0022C3F8002500BF02B0704784B010
:10E610000390029101920093039B029AC3F808258C
:10E62000039B019AC3F80C25039B009AC3F810259D
:10E6300000BF04B0704782B001900091009A019B26
:10E64000C3F8242500BF02B0704784B00390029144
:10E650000192029A039BC3F84425039B019AC3F8D5
:10E66000482500BF04B0704784B003900291019226
:10E67000029A039BC3F83425039B019AC3F83825FB
:10E6800000BF04B0704784B001900B468DF8033092
:10E6900013468DF802309DF80230002B14BF012381
:10E6A0000023DBB203939DF80330032B10D0032B20
:10E6B00013DC012B02D0022B05D00EE0039B43F0AC
:10E6C000020303930AE0039B43F00403039305E072
:10E6D000039B43F00603039300E000BF019B039AF2
:10E6E000C3F8542500BF04B0704782B001900B46B8
:10E6F0008DF803309DF80320019BC3F8C02500BFAF
:10E7000002B0704782B00190019B0122C3F85025EE
:10E7100000BF02B0704782B00190019B0022C3F895
:10E72000502500BF02B0704782B00190019B0122CA
:10E73000C3F8402500BF02B0704782B00190019B32
:10E740000022C3F8402500BF02B0704700B583B077
:10E750000190019B1B68184600F0B4F80346002B9B
:10E7600004D105494FF4F670F9F73EFC4FF0A04391
:10E77000184603B05DF804FBF882030000B585B0CD
:10E780000190084611461A4603468DF803300B46A1
:10E790008DF8023013468DF8013001AB1846FFF7B3
:10E7A000D5FF03909DF803209DF802305B001A43CB
:10E7B0009DF801309B001A439DF818301B0242EA75
:10E7C00003019DF81C301B04019A1943039B02F5B9
:10E7D000E07243F8221000BF05B05DF804FB00B5FD
:10E7E00085B00390002301930023009300230122AE
:10E7F00001210398FFF7C2FF00BF05B05DF804FBDD
:10E8000000B585B003900B468DF80B309DF80B30AA
:10E810000022019200220092002200210398FFF7BB
:10E82000ADFF00BF05B05DF804FB00B585B00390F7
:10E830000023019300230093002301220021039869
:10E84000FFF79CFF00BF05B05DF804FB00B585B085
:10E85000019001AB1846FFF779FF0390019B01225D
:10E8600002FA03F31946039800F018F800BF05B048
:10E870005DF804FB00B585B0019001AB1846FFF7C9
:10E8800065FF0390019B012202FA03F319460398E6
:10E8900000F00EF800BF05B05DF804FB82B00190F7
:10E8A0000091019B009AC3F8082500BF02B0704791
:10E8B00082B001900091019B009AC3F80C2500BF23
:10E8C00002B0704784B00190019B5B090293002362
:10E8D0000393029B002B03D14FF0FF33039300BF40
:10E8E000019B03F01F030193039A019B22FA03F398
:10E8F00003F00103002B14BF01230023DBB21846F1
:10E9000004B0704700B58DB0059004910392029356
:10E91000049B002B03D16C49AD20F9F765FB059BE7
:10E920001B791A461346DB0013449B00674A1344C5
:10E930000A930A9B1B7F002B03D008230793079B96
:10E94000BDE0059B1B680993059B1A68059B1B7915
:10E9500019465F4B53F8213019461046FDF7D0FF9A
:10E960000346002B03D011230793079BA7E00A9BC4
:10E97000039A1A600A9B029A5A60049B1B7B012B24
:10E9800005D8049B1B781846FFF774FF04E0049B2E
:10E990001B781846FFF75AFF049B1B781846002384
:10E9A000019300230093002300220121FFF7E6FEDC
:10E9B000049B5B78FF2B09D0049B5B780B930B982F
:10E9C000FFF758FF0B98FFF70AFF02E04FF0FF3305
:10E9D0000B93049B9B78FF2B07D0049B9B78089399
:10E9E00001210898FFF70CFF02E04FF0FF33089376
:10E9F000049B9A780A9B83F82020049BDA780A9B70
:10EA0000DA77049BDB78FF2B17D0049B1B79002B54
:10EA100005D0049BDB781846FFF72CFF04E0049B2D
:10EA2000DB781846FFF712FF049BDB781846FFF7E8
:10EA3000D6FE049B1A790A9B9A77049B1B78194689
:10EA4000089B0B9A0998FFF7E2FD049B9B68194607
:10EA50000998FFF7F0FD049B197B049B5B7B1A462A
:10EA60000998FFF710FE049B9B7919460998FFF758
:10EA70003CFE0998FFF7B9FD0A9B1B68002B15D0D7
:10EA8000059B1B681846FFF717FD03461A46049BB3
:10EA90005B7919461046FFF717FD059B1B68184662
:10EAA000FFF70AFD03461846FFF73AFD0A9B0022CE
:10EAB0005A770A9B01221A7700230793079B18466F
:10EAC0000DB05DF804FB00BF2C8303008C330020E5
:10EAD0006083030000B585B00190019B1B791A4645
:10EAE0001346DB0013449B002A4A13440393039B01
:10EAF0001B7F002B04D128494FF4AE70F9F774FA4C
:10EB0000039B1B68002B08D0019B1B681846FFF76E
:10EB1000D3FC03461846FFF711FD019B1B680293C7
:10EB2000039B1B68002B1BD01C490298FFF753FD69
:10EB3000039B5B7FDBB2002B12D014210298FFF7FE
:10EB40000BFD00BF4FF482710298FFF728FD0346CA
:10EB500083F00103DBB2002BF4D1039B00225A7730
:10EB6000039B93F82030FF2B05D0039B93F82030B4
:10EB70001846FFF75AFE0298FFF740FD019B1B68FD
:10EB80001846FDF7FFFE039B00221A7700BF05B071
:10EB90005DF804FB8C3300202C8303005201080035
:10EBA00000B583B00190019BDB7FFF2B0ED0019B52
:10EBB0009B7F002B05D0019BDB7F1846FFF75AFE99
:10EBC00004E0019BDB7F1846FFF740FE019B00221B
:10EBD0005A77019B00221A72019B1B68019A02F16D
:10EBE0000800019A52681146984700BF03B05DF8CB
:10EBF00004FB00B583B001900B468DF803309DF8FF
:10EC0000033083F00103DBB2002B04D040210198D4
:10EC1000FFF7E1FC03E040210198FFF7D2FC00BFC1
:10EC200003B05DF804FB00B583B001900091009B38
:10EC300003F00103002B03D00198FFF763FD02E00E
:10EC40000198FFF768FD009B03F00203002B03D03F
:10EC50000198FFF769FD02E00198FFF76EFD00BF24
:10EC600003B05DF804FB00B587B0039002910192F8
:10EC70000093019B1B68002B0AD0019B1B68184660
:10EC8000FFF70CFC034683F00103DBB2002B0ED12F
:10EC9000019B9B68002B11D0019B9B681846FFF7D6
:10ECA000FDFB034683F00103DBB2002B06D0029B81
:10ECB00000225A7710230593059B54E0019B1968A5
:10ECC000019B5B681A460398FFF7BFFC019B99689C
:10ECD000019BDB681A460398FFF7C6FC4FF48C7162
:10ECE0000398FFF747FC00990398FFF79CFF009BF0
:10ECF00003F00803002B03D110210398FFF72CFC2D
:10ED0000029B1B68002B1FD100BF4FF48C7103982E
:10ED1000FFF745FC034683F00103DBB2002BF4D17F
:10ED2000029BDB7FFF2B1BD0029B9B7F002B05D020
:10ED3000029BDB7F1846FFF79DFD11E0029BDB7F06
:10ED40001846FFF783FD0BE0009B03F00403002B44
:10ED50000CBF01230023DBB219460398FFF749FFDC
:10ED600000230593059B184607B05DF804FB0000DF
:10ED700010B586B0039002910192039B1B791A464D
:10ED80001346DB0013449B00394A13440593059B4B
:10ED90001B7F002B04D1374940F22D20F9F724F9CD
:10EDA000029B1B68002B08D1029B5B68002B04D0E0
:10EDB000304940F22E20F9F717F9029B9B68002B8F
:10EDC00008D1029BDB68002B04D02A4940F22F2097
:10EDD000F9F70AF9039B1B79002B07D1029BDB682B
:10EDE000FF2B03D8029B5B68FF2B04D921494FF40A
:10EDF0000C70F9F7F9F800230493059B5B7FDBB2F5
:10EE0000002B03D011230493049B2EE0059B1B6869
:10EE1000002B07D0019B03F01403002B02D1059BAC
:10EE200001225A77059B029A03F10C0413460FCB7B
:10EE300084E80F00059BDB7FFF2B0ED0059B9B7F9B
:10EE4000002B05D0059BDB7F1846FFF7FFFC04E095
:10EE5000059BDB7F1846FFF70DFD039B1868019BA0
:10EE6000029A0599FFF7FFFE0346184606B010BD4B
:10EE70008C3300202C83030000B583B001900091F7
:10EE80004FF48C710198FFF78AFB0346002B10D0DA
:10EE90004FF48C710198FFF76DFB009B1B68002BF2
:10EEA00004D1064940F29720F9F79EF80098FFF741
:10EEB00077FE00BF03B05DF804FB00BF2C830300A6
:10EEC00008B503490348FFF7D7FF00BF08BD00BFDF
:10EED0008C3300200030004000B583B00190019BCE
:10EEE0001B68184600F03EF80346002B04D1054984
:10EEF0004FF4F670F9F778F84FF0A043184603B0D6
:10EF00005DF804FB6483030000B585B001900B46F7
:10EF10008DF8033001AB1846FFF7DEFF0390019A2E
:10EF2000039B02F5E07253F82230019A23F440313A
:10EF3000039B02F5E07243F82210019A039B02F54D
:10EF4000E07253F822309DF8032012041146019A12
:10EF50001943039B02F5E07243F8221000BF05B08D
:10EF60005DF804FB84B00190019B5B0902930023D0
:10EF70000393029B002B03D14FF0FF33039300BF99
:10EF8000019B03F01F030193039A019B22FA03F3F1
:10EF900003F00103002B14BF01230023DBB218464A
:10EFA00004B0704700B583B00C4B1B78002B0FD01A
:10EFB0000023019308E0019B022B02D00198FCF78B
:10EFC0009BFD019B01330193019B032BF3D901E0CE
:10EFD000FCF7ACFD00BF03B05DF804FBB8330020C4
:10EFE0002DE9D04F92B003468DF83F3000231193A6
:10EFF00000231093CC4B1B78002B04D0CA4A00236B
:10F000001370FFF7CFFF9DF83F30172B00F23F82C0
:10F0100001A252F823F000BF79F0020091F0020043
:10F0200091F002002DF10200C9F1020045F2020048
:10F03000D9F20200F9F2020009F3020035F30200EE
:10F0400053F3020071F302008FF302009DF30200FC
:10F050009DF302009DF302009DF302009DF3020068
:10F0600031F402003FF4020053F4020067F402009E
:10F0700081F4020081F40200FFF794FFAB4B1846C5
:10F08000F8F7F8FD1190AA4A9DF83F301370FFE1A0
:10F090000020FCF7E9FC0346002B0DD00020FCF714
:10F0A0002BFD9DF83F30022B02D14FF4E16301E0CC
:10F0B0004FF47A6310930BE00020FCF703FD9DF8FA
:10F0C0003F30022B01D1C82301E04FF4C8731093E5
:10F0D000974A9DF83F301370944C109B0022009388
:10F0E00001924FF000024FF00003DDE9006739465E
:10F0F000CB03314643EA51433146CA0312F57A71D4
:10F10000029143F1000303934FF4FA624FF00003BE
:10F11000DDE9020107F017FC02460B461346002208
:10F1200019462046F8F76EFD1190B1E10020FCF77A
:10F130009BFC0346002B0DD00020FCF7DDFC9DF866
:10F140003F30032B02D14FF4487301E04FF47A6350
:10F1500010930BE00020FCF7B5FC9DF83F30032B2B
:10F1600001D1C82301E04FF4C8731093704A9DF891
:10F170003F3013706D4C109B0022049305924FF0AA
:10F1800000024FF00003DDE904673946CB03314646
:10F1900043EA51433146CA0312F57A71069143F1AD
:10F1A000000307934FF4FA624FF00003DDE9060114
:10F1B00007F0C9FB02460B461346002219462046BB
:10F1C000F8F720FD119063E10020FCF74DFC0346A9
:10F1D000002B06D00020FCF78FFC4FF47A631093CD
:10F1E00005E00020FCF76EFC4FF4C8731093504A02
:10F1F0009DF83F3013704D4C109B00229A46934669
:10F200004FF000024FF000034FEACB3343EA5A437A
:10F210004FEACA3212F57A71089143F1000309935B
:10F220004FF4FA624FF00003DDE9080107F08BFBB1
:10F2300002460B461346002219462046F8F7E2FC28
:10F24000119025E10020FCF70FFC0346002B0CD0A9
:10F250000020FCF751FC9DF83F30052B01D1C8235D
:10F2600001E04FF47A6310930BE00020FCF72AFCD6
:10F270009DF83F30052B01D1C82301E04FF4C8733E
:10F2800010932B4A9DF83F301370284C109B00229E
:10F29000984691464FF000024FF000034FEAC93301
:10F2A00043EA58434FEAC83212F57A710A9143F1A2
:10F2B00000030B934FF4FA624FF00003DDE90A01FB
:10F2C00007F041FB02460B46134600221946204632
:10F2D000F8F798FC1190DBE00020FCF74DFC144A95
:10F2E0009DF83F301370114B002240F266611846C2
:10F2F000F8F788FC1190CBE00020FCF7E3FB0C4A08
:10F300009DF83F301370C3E0074B01221A700120B3
:10F31000FCF732FC054B002240F266611846F8F714
:10F3200071FC1190B4E000BFB1330020C033002065
:10F33000B0330020594B01221A700120FCF71CFC4D
:10F34000574B00224FF400511846F8F75BFC119020
:10F350009EE0524B01221A700120FCF70DFC504B2D
:10F36000002240F266611846F8F74CFC11908FE0DD
:10F370004A4B01221A700120FCF7FEFB484B002289
:10F380004FF400511846F8F73DFC119080E0FCF76F
:10F39000E0FB444A9DF83F30137079E0424B184639
:10F3A000F8F768FC11909DF83F30C3F111031093FA
:10F3B000109B002B35D0119B002B32D1109B012BC1
:10F3C00028D9394C109B9BB21A46C82302FB03F381
:10F3D000DA171E4617464FF000024FF00003FB03FA
:10F3E00043EA5643F20312F57A710C9143F100039C
:10F3F0000D934FF4FA624FF00003DDE90C0107F0C2
:10F40000A2FA02460B461346002219462046F8F798
:10F41000F9FB11900220FCF755FB244B01221A70D6
:10F4200036E00220FCF768FB204B00221A702FE028
:10F43000FFF7B8FD1B4A9DF83F30137028E0FFF737
:10F44000B1FD0020FCF73EFB164A9DF83F301370DB
:10F450001EE0FFF7A7FD0120FCF734FB114A9DF8E1
:10F460003F30137014E0FFF79DFD0020FCF72AFBEE
:10F470000120FCF727FB0B4A9DF83F30137007E093
:10F48000FCF767FB074A9DF83F30137000E000BFB0
:10F49000119B184612B0BDE8D08F00BFB1330020D9
:10F4A000C0330020B0330020E0330020B833002008
:10F4B00000B585B003468DF8073000230393084B51
:10F4C0001B6803F00103002B05D09DF80730184698
:10F4D000FFF786FD0390039B184605B05DF804FB1B
:10F4E000B433002084B001900B468DF803301346EE
:10F4F0008DF8023000230393019B032B3CD89DF829
:10F500000230012B0BD19DF80330012B04D1019B5C
:10F51000DBB20E33DBB200E000238DF802309DF841
:10F520000330022B0FD0022B23DC002B16D0012B33
:10F530001FD11449019A13465B0013440B449DF8F4
:10F5400002201A701AE00F49019A13465B00134417
:10F550000B4401339DF802201A700FE00949019A0B
:10F5600013465B0013440B4402339DF802201A70CB
:10F5700004E00723039301E007230393039B18464A
:10F5800004B070470034002000B585B001900B46F0
:10F590008DF80330019B032B14D89DF80330002B0A
:10F5A00001D0032300E000238DF80F300198FCF711
:10F5B000FDFA02469DF80F3019461046FFF7A4FCED
:10F5C000002300E00623184605B05DF804FB00B5F3
:10F5D00083B0019001210198FFF7D6FF034618463A
:10F5E00003B05DF804FB00B583B0012200210020C8
:10F5F000FFF778FF0190019B002B04D0019B072BA4
:10F6000001D0019B1CE0072202210120FFF76AFFC5
:10F610000190019B002B04D0019B072B01D0019B83
:10F620000EE0042202210020FFF75CFF0190019B05
:10F63000002B04D0019B072B01D0019B00E000238D
:10F64000184603B05DF804FB00B583B00122022127
:10F650000020FFF747FF0190019B002B04D0019B86
:10F66000072B01D0019B1CE0072202210120FFF79C
:10F6700039FF0190019B002B04D0019B072B01D087
:10F68000019B0EE00A2200210020FFF72BFF0190D2
:10F69000019B002B04D0019B072B01D0019B00E0B4
:10F6A0000023184603B05DF804FB00B583B00020CA
:10F6B000FFF78DFF0190019B002B04D0019B062BCF
:10F6C00001D0019B0CE00120FFF781FF0190019B1D
:10F6D000002B04D0019B062B01D0019B00E00023EE
:10F6E000184603B05DF804FB00B585B001900091A9
:10F6F000019B1B88102B02D0112B18D02FE01A4B26
:10F700001B68002B0DD1FFF76EFF0390039B002BAE
:10F7100007D0164B1B68002B03D0144B1B680398B3
:10F720009847114B1B6801330F4A136017E00E4BCB
:10F730001B68013B0C4A13600B4B1B68002B0DD15F
:10F74000FFF782FF0390039B002B07D0074B1B683A
:10F75000002B03D0054B1B680398984700BF00BFE0
:10F7600005B05DF804FB00BF103400200C3400200D
:10F7700076DF704700BF18467ADF704700BF184633
:10F780007CDF704700BF18467FDF704700BF184618
:10F790008FDF704700BF184682B003468DF80730F0
:10F7A0009DF90730002B0CDB9DF8073003F01F029A
:10F7B00005499DF907305B09012000FA02F241F882
:10F7C000232000BF02B0704700E100E082B0034692
:10F7D00000918DF807309DF90730002B0ADB009B64
:10F7E000DAB20C499DF907305201D2B20B4483F8CA
:10F7F00000230BE0009BDAB207499DF8073003F0C5
:10F800000F03043B5201D2B20B441A7600BF02B080
:10F81000704700BF00E100E000ED00E0B1DF70479D
:10F8200000BF184633DF704700BF184600B583B0ED
:10F830000190019B1B68184600F074F80346002BEA
:10F8400004D105494FF4F670F8F7CEFB4FF0A04312
:10F85000184603B05DF804FB9083030000B585B043
:10F860000190084611461A4603468DF803300B46B0
:10F870008DF8023013468DF8013001AB1846FFF7C2
:10F88000D5FF03909DF803209DF802305B001A43DA
:10F890009DF801309B001A439DF818301B0242EA84
:10F8A00003019DF81C301B04019A1943039B02F5C8
:10F8B000E07243F8221000BF05B05DF804FB00B50C
:10F8C00085B00390002301930023009300230122BD
:10F8D00001210398FFF7C2FF00BF05B05DF804FBEC
:10F8E00000B585B0019001AB1846FFF79FFF03906C
:10F8F000039BD3F804350293029BDA43019B012159
:10F9000001FA03F31A40039BC3F80825019B012267
:10F910009A40029B1A40039BC3F80C2500BF05B018
:10F920005DF804FB84B00190019B5B090293002306
:10F930000393029B002B03D14FF0FF33039300BFCF
:10F94000019B03F01F030193039A019B22FA03F327
:10F9500003F00103002B14BF01230023DBB2184680
:10F9600004B0704700B583B04FF480410020F6F733
:10F97000DBFE0190019B0093009B002B04D0054A05
:10F9800063210098F7F766FFF6F750FE00BF03B05B
:10F990005DF804FBD083030000B583B0F9F71AFBD0
:10F9A0000190019B0093009B002B04D0044A6B2123
:10F9B0000098F7F74FFF00BF03B05DF804FB00BFEE
:10F9C000D083030000B58DB001900091019B1B888E
:10F9D000562B00F0CC80562B00F3DB80522B00F02E
:10F9E000A180522B00F3D580212B2DDC102BC0F2EF
:10F9F000D080103B112B00F2CC8001A252F823F0F2
:10FA00004FFA0200ADFA020093FB0200FFFA020077
:10FA100093FB020093FB020093FB020093FB0200A6
:10FA200093FB020093FB020093FB020093FB020096
:10FA300093FB020093FB020093FB020093FB020086
:10FA400093FB0200CDFA02003B2B7ED0A1E0594A85
:10FA5000594BD31ADB081B0443F0030357491846DC
:10FA6000F7F736F90720FFF723FD0B900B9B059363
:10FA7000059B002B04D0524A75210598F7F7EAFE42
:10FA8000019B9A884F4B1A804E4B1B8819464E4853
:10FA900003F0DEFB0B900B9B0493049B002B7AD0AE
:10FAA000474A78210498F7F7D5FE74E0414A424B63
:10FAB000D31ADB081B0443F0030344491846F7F745
:10FAC00007F9404B4FF6FF721A806FE000238DF864
:10FAD0000C3000238DF80D30019B9B8803AA114642
:10FAE0001846FFF755FE0B900B9B0793079B002BC7
:10FAF00053D0334A89210798F7F7ACFE4DE0314BDC
:10FB00001888002300228521FFF73EFE0B900B9BF7
:10FB10000693069B002B42D0294A8F210698F7F7BF
:10FB200099FE3CE0274B1888002300220021FFF7B4
:10FB300075FE0B900B9B0993099B002B31D0204A3B
:10FB400095210998F7F786FE2BE0019B9B881321EE
:10FB50001846FFF70DFE0B900B9B0893089B002B9C
:10FB600021D0174A9C210898F7F774FE1BE0019BEF
:10FB70009B8813211846FFF7FBFD0B900B9B0A9304
:10FB80000A9B002B11D00E4AA3210A98F7F762FEB8
:10FB90000BE000BF0AE000BF08E000BF06E000BFC6
:10FBA00004E000BF02E000BF00E000BF00BF0DB0F6
:10FBB0005DF804FB7C7303004C73030008840300AE
:10FBC000D08303007C2B002068A90020148403004C
:10FBD00000B587B003F050FF0590059B0493049B8C
:10FBE000002B04D0144AB0210498F7F733FE002309
:10FBF000019301AB1946012003F0F6FF0590059B28
:10FC00000393039B002B04D00B4AB6210398F7F70C
:10FC100021FE01AB184604F005F90590059B0293FF
:10FC2000029B002B04D0044ABA210298F7F712FE77
:10FC300000BF07B05DF804FBD083030000B587B0B8
:10FC40009DF80030012262F303038DF800309DF827
:10FC50000030012262F307138DF800306B46062254
:10FC60001A491846FFF78CFD0590059B0493049BE9
:10FC7000002B04D0164ACB210498F7F7EBFD01AB1B
:10FC800008220021184606F0A7FF1023ADF8043023
:10FC90003C23ADF806300023ADF808304FF4C873AC
:10FCA000ADF80A3001AB1846FFF766FD0590059BDD
:10FCB0000393039B002B04D0054AD5210398F7F743
:10FCC000C9FD00BF07B05DF804FB00BF248403003A
:10FCD000D083030000B583B001900091009B5A8847
:10FCE000114B1B889A421AD1009B1B8840F6772241
:10FCF000934214D1009B9B88033B9AB20B4B1A8012
:10FD00000B4A0C4BD31ADB081B0443F00300074BD0
:10FD10001B881A46054B1B880749F6F7F8FF00BFFA
:10FD200003B05DF804FB00BF7C2B00207E2B00207D
:10FD30007C7303004C7303002C84030000B585B072
:10FD40001049114803F062F90390039B0293029B50
:10FD5000002B04D00D4AE8210298F7F77BFDF7212C
:10FD6000094803F07EF90390039B0193019B002B4C
:10FD700004D0064AEB210198F7F76CFD00BF05B0EF
:10FD80005DF804FBD5FC020054A90020D0830300D9
:10FD900000B583B00190044AF0210198F7F75AFDAD
:10FDA00000BF03B05DF804FBD083030000B587B04B
:10FDB0000190019B1B78002B44D1002305932BE07D
:10FDC000019B1A69059B13441B781846F7F7CEFF71
:10FDD0000490049B002B19D0049B112B16D01B4AB6
:10FDE0001B4BD31ADB081B0443F00103049A194987
:10FDF0001846F6F77BFF049B0393039B002B05D06B
:10FE0000154A4FF480710398F7F724FD049B112BDA
:10FE1000D6D0059B01330593019B9B8A1A46059B0F
:10FE20009342CDD3019B1A69019B9B8A013B1344EA
:10FE30001B780D2B06D100BF0A20F7F797FF03466A
:10FE4000112BF9D000BF07B05DF804FB7C730300F1
:10FE50004C73030048840300D083030000B587B0CF
:10FE600000230193174B019301AB1946164803F089
:10FE7000CDF90590059B0493049B002B05D0134AF4
:10FE80004FF48A710498F7F7E5FC02AB04220021D5
:10FE9000184606F0A1FE0E4B029302AB19460D4820
:10FEA00003F0F6FB0590059B0393039B002B05D005
:10FEB000064A4FF48E710398F7F7CCFC00BF07B0E9
:10FEC0005DF804FB91FD020068A90020D0830300C7
:10FED000ADFD0200602B002000B585B00020FFF7CB
:10FEE000E7FA0390039B0293029B002B05D0134A71
:10FEF00040F221110298F7F7ADFCFFF7D6FB039013
:10FF0000039B0193019B002B05D00C4A40F2251165
:10FF10000198F7F79FFCFFF785FC0390039B009384
:10FF2000009B002B05D0054A40F229110098F7F7F5
:10FF300091FC00BF05B05DF804FB00BFD083030057
:10FF400000B585B003468DF807309DF80730002BCB
:10FF500011D0032B12D10220FFF7AAFA0390039BC2
:10FF60000293029B002B0BD0084A4FF49971029820
:10FF7000F7F770FC04E0FFF7AFFF02E000BF00E01E
:10FF800000BF00BF05B05DF804FB00BFD0830300D5
:10FF900000B5AFB001ABAC220021184606F01CFE44
:10FFA00002238DF8043000238DF8063005238DF8E8
:10FFB00007300123ADF85030124B159301238DF813
:10FFC00080304023239344F2506324930E4B2A93B2
:10FFD00001AB19460D4801F055FD2D902D9B2C933A
:10FFE0002C9B002B05D00A4A4FF4A9712C98F7F7E7
:10FFF00031FC0121054801F038FD00BF2FB05DF84C
:020000023000CC
:1000000004FB00BF802B002041FF020074A90020E8
:10001000D083030000B585B00190019B1B78002BB5
:1000200011D10B4B1B883B211846FFF7A1FB039016
:10003000039B0293029B002B05D0064A4FF4AE713E
:100040000298F7F707FC00BF05B05DF804FB00BF9E
:100050007C2B0020D083030000B583B00190054ABB
:1000600040F261110198F7F7F5FB00BF03B05DF8AE
:1000700004FB00BFD083030000B58BB001AB1C2292
:100080000021184606F0A8FD002301934FF4A03389
:1000900002934FF4F023039303238DF810300023D1
:1000A000ADF8123000238DF814300C4B06930C4B36
:1000B000079301AB184602F047F80990099B089393
:1000C000089B002B05D0074A40F273110898F7F7F8
:1000D000C1FB00BF0BB05DF804FB00BF15000300BF
:1000E00059000300D0830300114B0222C3F8F0250E
:1000F0000F4B0022C3F8F4250D4B4FF40032C3F828
:1001000018250B4B0122C3F81025094B0022C3F818
:100110001425074B0022C3F80023054B054AC3F8FA
:100120002C26034B0122C3F8302600BF704700BFC6
:1001300000700040C4AD00200A4B0122C3F8002526
:10014000084B01221A6000BF064BD3F80031002B88
:10015000FAD0044B0022C3F80021024B01225A605E
:1001600000BF70470070004000B587B03A4BD3F82D
:100170004031002B6CD0384BD3F8043303F4803378
:10018000002B65D0344B0022C3F84021FFF7D4FF89
:1001900000BF324BD3F80431002BFAD02F4B002292
:1001A000C3F804212E4B1B681BB2002B05DA2C4B25
:1001B0001B681B0C1B042A4A1360294B1B68DBB20B
:1001C0009BB203F03F039AB2254B1B689B09DBB23D
:1001D0009BB203F03F039BB29B019BB21344ADF86B
:1001E0001230BDF8122001AB1E49184606F0A5FCDE
:1001F00001AB184606F023FD034603931A4B1B88F8
:10020000059310E0184B1B881A46059B9B1A06AAFB
:10021000134413F8141C154A059B13440A461A701C
:10022000059B01330593104B1B881A46039B13440F
:10023000059A9A42E6DB039B9AB20B4B1B88134448
:100240009AB2094B1A800A4B1B680133084A1360A3
:1002500000BF07B05DF804FB00A000400070004044
:10026000C4AD0020748403004CA900201434002085
:1002700048A9002008B5124B0022C3F80425104BF2
:100280000122DA600E4B0622C3F810250C4B012226
:10029000C3F808250A4B0A22C3F84025084B4FF43F
:1002A0008032C3F8042306210A20FFF78FFA0A20C0
:1002B000FFF772FA024B01221A6000BF08BD00BFAF
:1002C00000A0004000B587B001238DF81730012150
:1002D000AF4804F065FAAF4AAF4BD31ADB081B04F2
:1002E00043F00303AD491846F6F7F2FC03230493E9
:1002F00013E0A84AA84BD31ADB081B0443F00303FE
:10030000A7491846F6F7E4FC002003F08DFF0346EA
:100310008DF81730049B013B0493049B002B03D002
:100320009DF81730002BE4D19DF81730002B0BD02F
:10033000984A994BD31ADB081B0443F003039949ED
:100340001846F6F7C5FC7EE1974B5B6997489847DE
:1003500003465B684FF48012B2FBF3F30393924BB6
:100360005B699248984703461A68039BB2FBF3F314
:100370000293884A884BD31ADB081B0443F003031B
:10038000029A8B491846F6F7B1FC824A824BD31A7F
:10039000DB081B0443F0030386491846F6F798FC74
:1003A00001228549854805F03BFE03468DF807305C
:1003B0009DF80730002B0BD0764A774BD31ADB0819
:1003C0001B0443F003037E491846F6F781FC3AE12B
:1003D000704A714BD31ADB081B0443F003037949BD
:1003E0001846F6F775FC7849784806F002FA034695
:1003F0008DF807309DF80730002B0BD0654A664B0F
:10040000D31ADB081B0443F0030371491846F6F7BF
:100410005FFC18E16F496D4806F04FFA03468DF80E
:1004200007309DF80730002B0BD05A4A5A4BD31A8D
:10043000DB081B0443F0030367491846F6F748FC42
:1004400001E1644B5B7A002B1FD0624B1B7A03F0F7
:100450001003002B0CD04F4A4F4BD31ADB081B0460
:1004600043F005035D4A5E491846F6F73FFC0CE091
:10047000484A494BD31ADB081B0443F00500554B8F
:100480001A68564B5749F6F742FC524B5B7A002BE1
:10049000C0D1404A404BD31ADB081B0443F005038C
:1004A00051491846F6F714FC3A4A3B4BD31ADB087D
:1004B0001B0443F003034D491846F6F709FC3322A9
:1004C0004B494C4805F0F0FD03468DF807309DF888
:1004D0000730002B0BD02F4A2F4BD31ADB081B04FD
:1004E00043F0030344491846F6F7F2FBABE0294A10
:1004F000294BD31ADB081B0443F003033F4918467A
:10050000F6F7E6FB3E4B1B78002B25D06B4647F2F7
:1005100031523C49374805F05DFF03468DF80730FE
:100520009DF80730002B0BD01A4A1B4BD31ADB085F
:100530001B0443F0030334491846F6F7C9FB0BE0EC
:10054000144A154BD31ADB081B0443F00303009A2B
:100550002E491846F6F7CAFB2A4806F070FB0246F9
:100560006B462849234805F035FF03468DF80730D0
:100570009DF80730002B4BD0064A074BD31ADB08F7
:100580001B0443F0030320491846F6F7A1FB4BE098
:10059000842B00207C7303004C73030078840300D9
:1005A000988403009C840300A07F03001886030046
:1005B000BC840300D0840300E8840300C8AD00209D
:1005C000EC840300FC84030018850300F8AF0020CE
:1005D0001C85030024B00020388503002DB00020C6
:1005E00050850300608503006C850300708503005F
:1005F000908503003CB000209C850300C08503006B
:100600004EA9002014340020D8850300E88503009B
:100610000E4A0F4BD31ADB081B0443F00303009A66
:100620000C491846F6F762FB0B4806F0BFF8074A7C
:10063000074BD31ADB081B0443F003030749184692
:10064000F6F746FB00BF07B05DF804FB7C730300C0
:100650004C730300E88503003CB00020FC850300D8
:1006600000B583B00321094801F0E4FA0190019B31
:100670000093009B002B05D0054A40F225210098ED
:10068000F7F7E8F800BF03B05DF804FB74A9002099
:10069000D083030008B51420FFF711F91E4A1F4B41
:1006A000D31ADB081B0443F003031D491846F6F771
:1006B0000FFBFFF757F9FFF7DDFDFFF76DF9FFF7C8
:1006C00087FAFFF7BBFAFFF739FBFFF7C7FBFFF726
:1006D0005FFCFFF7D1FCFFF7C3FFFFF705FD114BF0
:1006E0001B68B3F5FA6FFAD11420FFF7F9F80A4A3C
:1006F0000A4BD31ADB081B0443F0030308491846CE
:10070000F6F7E6FA074B00221A60074B00221A8020
:10071000FFF7D8FDE3E700BF7C7303004C730300D1
:100720001486030048A900204CA9002082B0204B69
:100730000193019B02221A61019B02225A61019BD3
:100740001C4A9A61019B1C4ADA61019B4FF40072BA
:100750001A62019B00229A62019B00225A62019B4D
:100760000022DA62019B134A9A64019B134ADA64FD
:10077000019B10221A65019B00229A65019B0022B1
:100780005A65019B0022DA65019B07330C4A106809
:100790001860019B0B4A10681860918892799980C3
:1007A0009A71019B20229A7100BF02B0704700BF6E
:1007B00064B2002034860300DCB20020DCB40020E8
:1007C000408603004486030000B589B0039002917F
:1007D000019200230693039BDB680593039B1B692F
:1007E0000493049A059B9A4205D9049A059BD31A4F
:1007F000013B079307E0039B9A680499059BCB1A7A
:100800001344013B0793039B9A68059BD31A079AED
:10081000934228BF13460793079A019B934228BF30
:1008200013460793039B5A68059B1344079A029942
:10083000184606F0A8F9069A079B13440693029AF5
:10084000079B13440293019A079BD31A0193059ABD
:10085000079B13440593039B9B68059A9A4201D119
:1008600000230593039B059ADA60019B002BB5D109
:10087000069B184609B05DF804FB00B589B00390EB
:1008800002910192039BDB680793039B9A68079B85
:10089000D31A0693069A019B9A420ED9039B5A6873
:1008A000079B1344019A0299184606F06CF9079ABF
:1008B000019B1A44039BDA601AE0069B0593039B95
:1008C0005A68079B1344059A0299184606F05BF98B
:1008D000019A069BD31A0593039B5868029A069BBC
:1008E0001344059A194606F04EF9039B059ADA60FF
:1008F00000BF09B05DF804FB86B00190019B1B6945
:100900000493019BDB680393049A039B9A4208D8E3
:10091000019B9A68039BD21A049B1344013B0593E5
:1009200004E0049A039BD31A013B0593059B1846E8
:1009300006B0704700B589B0039002910192029B06
:100940000693039B5A1C13465B001344DB00204AAA
:1009500013440593059B5B69022B29D0022B2ED8EB
:10096000002B02D0012B13D029E00598FFF7C4FF1C
:100970000490049A019B9A4202D20023079321E03B
:10098000019B0793019A06990598FFF776FF19E0F6
:100990000598FFF7B1FF0490019A049B934228BF8A
:1009A00013460793079A06990598FFF766FF09E033
:1009B000019A06990598FFF707FF079002E00023C8
:1009C000079300BF079B184609B05DF804FB00BF02
:1009D00064B2002008B5FFF7A9FE00BF08BD6DDFB7
:1009E000704700BF184679DF704700BF18467DDFAB
:1009F000704700BF184664DF704700BF184682B0DA
:100A000003460091ADF80630BDF80630DAB2009B1F
:100A10001A70BDF806301B0A9AB2009B0133D2B29D
:100A20001A700223184602B0704700B589B00390CF
:100A300002911346ADF80630029B1B8803F10902B0
:100A4000BDF806309A4201D90C2353E004AB184696
:100A5000FFF7C5FF0790079B0693069B002B01D06D
:100A6000069B47E0029B1B881A46039B13440822FF
:100A70001A70029B1B8801339AB2029B1A80029B58
:100A80001B881A46039B13441B221A70029B1B8867
:100A900001339AB2029B1A80029B1B881A46039B61
:100AA000981804AB01330622194606F06CF8029B35
:100AB0001B8806339AB2029B1A809DF8103023F0EF
:100AC0000103DBB2002B07D1029B1B881A46039B54
:100AD000134400221A7006E0029B1B881A46039BEF
:100AE000134401221A70029B1B8801339AB2029BA5
:100AF0001A800023184609B05DF804FB00B589B0E0
:100B0000039002910192ADF80230039B1B78012BF8
:100B100005D1039B5B78002B01D1072392E0019B59
:100B20001B889A1CBDF802309A420ED8039B1B7892
:100B3000012B0CD1019B1B881A46039B5B78134445
:100B40009A1CBDF802309A4201D90C237AE0019B2D
:100B50001B88BDF80220D31A9BB2023BADF81C30B3
:100B6000BDF81C30ADF81230019B1B880233029A8D
:100B700013440DF1120211461846FFF738FF069094
:100B8000069B0593059B002B01D0059B5AE0039B18
:100B90001B78022B06D0039B5B789AB2BDF812300B
:100BA0009A4209D3BDF81230BDF81C209A4203D3F3
:100BB00009238DF81F3017E008238DF81F30039BA1
:100BC0001B78012B0CD1039B5B789BB2BDF81C20DA
:100BD0009A4205D3039B5B789BB2ADF8123003E0D9
:100BE000BDF81C30ADF81230BDF81230FE2B01D923
:100BF0000C2327E0BDF81230DAB2019B1B8819469E
:100C0000029B0B440132D2B21A70019B1B88013344
:100C10009AB2019B1A80019B1B881A46029B1344BF
:100C20009DF81F201A70019B1B8801339AB2019B0B
:100C30001A80019B1A88BDF8123013449AB2019BA6
:100C40001A800023184609B05DF804FB00B589B08E
:100C5000039002911346ADF80630029B1B881A1DC3
:100C6000BDF806309A4201D90C233BE00DF1160382
:100C70001846FFF7B8FE0790079B0693069B002BCC
:100C800001D0069B2EE0029B1B881A46039B13444F
:100C900003221A70029B1B8801339AB2029B1A80AE
:100CA000029B1B881A46039B134419221A70029B4D
:100CB0001B8801339AB2029B1A80BDF81620029B52
:100CC0001B881946039B0B4419461046FFF797FEF5
:100CD00003461946029B1A888BB213449AB2029BB0
:100CE0001A800023184609B05DF804FB84B0029115
:100CF00001921A4603468DF80F301346ADF80C30BA
:100D0000019B1B88DA1CBDF80C309A4201D90C23D8
:100D100028E0019B1B881A46029B134402221A708A
:100D2000019B1B8801339AB2019B1A80019B1B888F
:100D30001A46029B134401221A70019B1B8801333F
:100D40009AB2019B1A80019B1B881A46029B13448E
:100D50009DF80F201A70019B1B8801339AB2019BEA
:100D60001A800023184604B0704784B002910192A3
:100D70001A4603468DF80F301346ADF80C30019B30
:100D80001B88DA1CBDF80C309A4201D90C2328E0EC
:100D9000019B1B881A46029B134402221A70019B76
:100DA0001B8801339AB2019B1A80019B1B881A464B
:100DB000029B13440A221A70019B1B8801339AB2CA
:100DC000019B1A80019B1B881A46029B13449DF8C5
:100DD0000F201A70019B1B8801339AB2019B1A8065
:100DE0000023184604B0704700B58FB003900193FC
:100DF0000B468DF80B3013468DF80A3000238DF822
:100E00003330109B1B88ADF8303000230D9371E018
:100E1000039B5A680D9B9B001A4405AB1068186031
:100E20000DF11B0105AB00221846FFF7E4FD0A9007
:100E30000A9B0993099B002B01D0099B7CE09DF83C
:100E40001B309DF80A209A4251D19DF83330002B77
:100E500001D0002300E002238DF82330109B1B8873
:100E60001A469DF81B301A449DF823301A44BDF8E9
:100E700044309A4201DD0C235EE09DF8333083F06C
:100E80000103DBB2002B16D0109B1B8801339AB2F2
:100E9000109B1A80109B1B881A46019B13449DF8D7
:100EA0000B201A70109B1B8801339AB2109B1A807A
:100EB00001238DF83330109B1B881A46019B1A447E
:100EC0000DF11B0105AB1846FFF795FD0A900A9B33
:100ED0000793079B002B01D0079B2DE0109B1A88DE
:100EE0009DF81B309BB213449AB2109B1A800D9B45
:100EF00001330D93039B1B881A460D9B934287DB9E
:100F00009DF83330002B16D0109B1A88BDF8303076
:100F1000D31A9BB2013BADF82E30BDF82E30FF2B1B
:100F200001D90C2308E0BDF83030019A1344BDF814
:100F30002E20D2B21A70002318460FB05DF804FBC1
:100F400000B58BB0059003930B468DF81330134614
:100F50008DF812309DF81310BDF8343001930C9BBE
:100F60000093039B02220598FFF73EFF0990099B1F
:100F70000893089B002B01D0089B14E09DF81210E9
:100F8000BDF8343001930C9B0093039B102205980D
:100F9000FFF72AFF0990099B0793079B002B01D0BD
:100FA000079B00E0002318460BB05DF804FB82B0FD
:100FB0000190019B1B88052B0AD9019B1B88B3F567
:100FC000486F07D9019B1B884FF6FF72934201D0EF
:100FD000072325E0019B5B88052B0AD9019B5B88D1
:100FE000B3F5486F07D9019B5B884FF6FF729342B8
:100FF00001D0072314E0019B1B884FF6FF72934238
:101000000DD0019B5B884FF6FF72934207D0019B86
:101010001A88019B5B889A4201D9072300E00023CC
:10102000184602B0704700B587B003900291019254
:10103000ADF80230019B1B889A1DBDF802309A4220
:1010400001D90C234DE00398FFF7B1FF0590059BF4
:101050000493049B002B01D0049B42E0019B1B885E
:101060001A46029B134405221A70019B1B88013308
:101070009AB2019B1A80019B1B881A46029B13445B
:1010800012221A70019B1B8801339AB2019B1A80AD
:10109000039B1A88019B1B881946029B0B44194627
:1010A0001046FFF7ACFC03461946019B1A888BB229
:1010B00013449AB2019B1A80039B5A88019B1B8898
:1010C0001946029B0B4419461046FFF798FC03464D
:1010D0001946019B1A888BB213449AB2019B1A805D
:1010E0000023184607B05DF804FB00B587B00390F5
:1010F00002910192ADF80230039B9B880233059365
:10110000019B1B881A46059B13449A1CBDF80230AC
:101110009A4201D90C2354E0059BFE2B01D90C23E4
:101120004FE0059BDAB2019B1B881946029B0B44DA
:101130000132D2B21A70019B1B8801339AB2019B13
:101140001A80019B1B881A46029B1344FF221A70C7
:10115000019B1B8801339AB2019B1A80039B1A885A
:10116000019B1B881946029B0B4419461046FFF74A
:1011700046FC03461946019B1A888BB213449AB267
:10118000019B1A80039B9B88002B19D0039B9B68B3
:10119000002B01D1072314E0019B1B881A46029BF8
:1011A0009818039B9968039B9B881A4605F0EBFCF3
:1011B000019B1A88039B9B8813449AB2019B1A8057
:1011C0000023184607B05DF804FB00B589B0039012
:1011D00002910192ADF80230039B9B6A002B01D172
:1011E000072372E000238DF81F3066E0039B996AA5
:1011F0009DF81F2013465B0013449B000B4406938D
:10120000069B9B8802330593059BFE2B01D90C237B
:101210005BE0059BDAB2019B1B881946029B0B44DD
:101220000132D2B21A70019B1B8801339AB2019B22
:101230001A80019B1B881A46029B134416221A70BF
:10124000019B1B8801339AB2019B1A80069B1A8866
:10125000019B1B881946029B0B4419461046FFF759
:10126000CEFB03461946019B1A888BB213449AB2EF
:10127000019B1A80069B9B88002B19D0069B9B68BC
:10128000002B01D1072320E0019B1B881A46029BFB
:101290009818069B9968069B9B881A4605F073FC74
:1012A000019B1A88069B9B8813449AB2019B1A8063
:1012B0009DF81F3001338DF81F30039B93F82C30BD
:1012C0009DF81F209A4291D30023184609B05DF87B
:1012D00004FB00B595B0059004910392002313938D
:1012E000039B1B88ADF84A30039B00221A80059BA4
:1012F00093F82D30002B0ED0BDF84A301A460399D2
:101300000498FFF792FB1390139B1193119B002BF2
:1013100001D0119BD8E0059B9B78002B0ED0BDF827
:101320004A301A4603990498FFF790FC1390139BD8
:101330001093109B002B01D0109BC5E0059BDB7820
:10134000002B10D0059BDB7858B2BDF84A30039AC9
:101350000499FFF7CBFC1390139B0F930F9B002B6B
:1013600001D00F9BB0E0059B5B68002B11D0059B63
:101370005B6893F90000BDF84A30039A0499FFF7BF
:10138000F4FC1390139B0E930E9B002B01D00E9B2D
:101390009AE0059B1B89002B14D0059B03F10800E4
:1013A000BDF84A300193039B0093049B062202215F
:1013B000FFF7C6FD1390139B0D930D9B002B01D0DF
:1013C0000D9B81E0059B1B8A002B14D0059B03F12C
:1013D0001000BDF84A300193039B0093049B072241
:1013E0000321FFF7ADFD1390139B0C930C9B002B77
:1013F00001D00C9B68E0059B1B8B002B14D0059B38
:1014000003F11800BDF84A300193039B0093049B3D
:1014100015221421FFF794FD1390139B0B930B9B44
:10142000002B01D00B9B4FE0059B1B6A002B0FD0BC
:10143000059B186ABDF84A30039A0499FFF7F3FD3B
:101440001390139B0A930A9B002B01D00A9B3BE04D
:10145000059B5B6A002B0FD0059B586ABDF84A308C
:10146000039A0499FFF741FE1390139B0993099B7C
:10147000002B01D0099B27E0059B93F82C30002B13
:101480000ED0BDF84A30039A04990598FFF79DFEE7
:101490001390139B0893089B002B01D0089B13E02B
:1014A000059B1B78002B0ED0BDF84A30039A049997
:1014B0000598FFF723FB1390139B0793079B002BC3
:1014C00001D0079B00E0139B184615B05DF804FBA4
:1014D00086B0039001921A460B46ADF80A301346C7
:1014E0008DF80930039B002B02D0019B002B01D10A
:1014F00000235CE00023ADF816300CE0BDF8163098
:10150000039A13441B789AB2BDF8163013449BB269
:101510000133ADF81630BDF816305A1CBDF80A304C
:101520009A420FDA019B1B88BDF816209A42E5D338
:10153000BDF816300133039A13441B789DF8092037
:101540009A42DBD1BDF81620BDF80A309A4201D389
:1015500000232CE0BDF816300233ADF81430BDF88E
:101560001630039A13441B78002B08D0BDF81630B0
:10157000039A13441B789BB2013B9BB200E000230B
:10158000ADF81230BDF81230002B08D0BDF8142091
:10159000BDF812301A44BDF80A309A4201DD00232A
:1015A00005E0019BBDF814201A80BDF812301846E2
:1015B00006B0704700B585B001900B46ADF802301B
:1015C00013468DF801300023ADF80C309DF8013042
:1015D00003AABDF802100198FFF77AFF0346ADF8A1
:1015E0000E30BDF80E30002B01D1002304E0BDF811
:1015F0000C301A46019B1344184605B05DF804FBF5
:1016000072DF704700BF184673DF704700BF18468F
:1016100082B00190019B93F83034184602B07047B5
:1016200084B00190002303930AE0019A039B1344C2
:101630001B78002B01D0012306E0039B01330393A9
:10164000039B052BF1D90023184604B07047000016
:1016500082B003468DF807309DF807305A1C074BBF
:1016600083FB02135910D317C91A0B469B000B4476
:10167000D11ACBB2184602B0704700BF67666666E3
:1016800082B001900091009BDB7B012B04D1009B79
:101690009A88019BA3F8242400BF02B0704700B5CC
:1016A00085B001900091019B002283F82E24009BBD
:1016B0009A88019BB3F824349A4216D1019B1B7976
:1016C00083F00103DBB2002B0FD00121019800F061
:1016D000B1FA0390039B002B07D0019B9B6B002B5F
:1016E00003D0019B9B6B0398984700BF05B05DF842
:1016F00004FB00B585B001900091009B1B88262B50
:101700001ED1009B1B7A012B03D0009B1B7A022B5E
:1017100017D1019B9B781846FFF79AFF034619469D
:10172000019800F087FA0390039B002B09D0019BDE
:101730009B6B002B05D0019B9B6B0398984700E0A7
:1017400000BF05B05DF804FB00B585B001900B4605
:101750008DF80330019B03F227431846FFF760FF23
:1017600003468DF80F309DF80330013B032B33D82F
:1017700001A252F823F000BF89170300AD17030040
:10178000C1170300CD170300019B9B79002B0DD0DF
:10179000019B93F8243083F00103DBB2002B05D0CA
:1017A0009DF80F30002B01D0012316E0019BDB795F
:1017B000002B05D09DF80F30002B01D002230CE048
:1017C000019B1B7A002B01D0032306E0019B5B7A6F
:1017D000002B01D0042300E00023184605B05DF87B
:1017E00004FB00BF82B001900091019B012283F8AD
:1017F0003120019B0022C3F82024019B03F22642E2
:10180000009B5A60009B00229A60009B02221A7083
:10181000009B80229A810023184602B0704782B054
:1018200001900091019B022283F83120019B93F8E3
:101830002430002B03D0009B07221A7002E0009B8B
:1018400003221A70019B1B699AB2009B9A81019B2B
:101850000022C3F82024019B03F22642009B5A6019
:10186000019BDA68009B9A600023184602B070471B
:1018700000B583B00190019B5B79002B0FD0019BD9
:1018800093F82E3483F00103DBB2002B07D00198CC
:10189000FFF7BEFE0346002B01D0012300E000232A
:1018A00003F00103DBB2184603B05DF804FB00B59A
:1018B00085B001900B468DF80330019BD3F81004DE
:1018C000019BB3F8143401221946FFF773FE03900D
:1018D000039B002B03D0039B9DF803201A70019BF0
:1018E00003F15400019B03F58261019B3C331A46CE
:1018F000FFF786FE0346184605B05DF804FB00B509
:1019000085B001900091019B5A69009B9A60019BF0
:101910009B699AB2009B9A81019B93F82430002B1B
:1019200004D0019B062283F83C2003E0019B0122A6
:1019300083F83C200198FFF79BFF0346002B13D050
:10194000009B02221A7504210198FFF7B0FF039053
:10195000039B0293029B002B01D0029B0FE0019B93
:10196000052283F8312003E0019B032283F8312014
:10197000019B03F58262019BC3F8202400231846D3
:1019800005B05DF804FB00B585B001900091019BA6
:10199000DA69009B9A60019B1B6A9AB2009B9A814C
:1019A000019B93F82430002B04D0019B062283F87E
:1019B0003C2003E0019B012283F83C200198FFF7C3
:1019C00057FF0346002B13D0009B02221A750421F7
:1019D0000198FFF76CFF0390039B0293029B002B7F
:1019E00001D0029B0FE0019B062283F8312003E027
:1019F000019B042283F83120019B03F58262019B45
:101A0000C3F820240023184605B05DF804FB82B01B
:101A10000190019B9B78002B06D0019B93F820300E
:101A2000002B01D000230AE0019B9B6A042B03D00A
:101A3000019B5B6A042B01D1002300E001231846BF
:101A400002B0704784B00190019B93F82430002BC2
:101A500003D0EE23ADF80E3002E01F23ADF80E30B8
:101A6000BDF80E30184604B0704782B001900B46A6
:101A70008DF80330019B9DF8032083F8302000BFD0
:101A800002B0704730B587B001900091009B002BE9
:101A900002D0019B002B01D10E23B8E0009B7833CC
:101AA0001846FFF7B4FF034683F00103DBB2002BB7
:101AB00001D00723ABE0019B00229A70019A009BA2
:101AC000141D03F178050FCD0FC40FCD0FC495E899
:101AD000070084E80700019B002283F83020009B68
:101AE000D3F8A420019B5A63009BD3F8A820019B44
:101AF0009A63019B4FF6FF72A3F82424019B03F520
:101B00008262019BC3F82024019B03F22643072233
:101B10000021184605F060F8019B1B7883F0010353
:101B2000DBB2002B03D0019BFF2283F85420019BE2
:101B300003F15502019BC3F810240198FFF782FFBF
:101B400003461A46019BA3F814240098019B03F155
:101B50005501019B03F214431A46FFF7BAFB0590A7
:101B6000059B0493049B002B01D0049B4FE0019B39
:101B700003F23122019BC3F818240198FFF762FF9A
:101B800003461A46019BA3F81C24009B03F13C006A
:101B9000019BD3F81814019B03F21C431A46FFF76C
:101BA00098FB0590059B0393039B002B01D0039B9F
:101BB0002DE0019B012283F85120019B9B699AB281
:101BC000019BA3F84820019B012283F83C20019B44
:101BD00000221A64019B002283F85020019B5A695D
:101BE000019B5A64019B03F15400019B3C331A464C
:101BF0000021FFF705FD0590059B0293029B002B3A
:101C000001D0029B03E0019B01221A70059B18463C
:101C100007B030BD82B00190019B1B68012B03D03F
:101C2000019B1B68022B01D1012300E00023184611
:101C300002B0704700B585B001900B468DF80330B7
:101C4000019B1B7883F00103DBB2002B01D008233A
:101C500009E1019B9DF803209A70019B03F2264342
:101C600007220021184604F0B7FF019B9B79002B47
:101C700003D0019B9B78012B0FD0019BDB79002BBC
:101C800003D0019B9B78012B07D0019BDB79002BB4
:101C900014D0019B9B78022B10D1019B5B6B002B16
:101CA00008D0019B012283F82D24019B5B6B082047
:101CB000984703E0019B002283F82D249DF8033010
:101CC00019460198FFF740FD03461A46019B9A709A
:101CD000019B5B6B002B20D0019B9B78032B03D0D7
:101CE000019B9B78042B18D1019B5B79002B14D0AE
:101CF000019B93F82E3483F00103DBB2002B0CD050
:101D0000019B002283F83024019B012283F82F24B9
:101D1000019B5B6B0720984703E0019B002283F83F
:101D20002F24019B3C3318220021184604F054FF55
:101D3000019B012283F83C20019B2C331846FFF7BE
:101D400069FF0346002B06D0019BDB6ADAB2019BD8
:101D500083F8512003E0019B012283F85120019B6D
:101D600093F82430002B12D0019B28331846FFF73C
:101D700051FF0346002B06D0019B9B6ADAB2019B00
:101D800083F8522003E0019B012283F85220019B3B
:101D9000002283F85020019B9B78042B31D801A2AC
:101DA00052F823F0F91D0300B91D0300C91D0300FB
:101DB000D91D0300E91D0300019B3C33194601981E
:101DC000FFF710FD03901DE0019B3C33194601987D
:101DD000FFF725FD039015E0019B3C331946019860
:101DE000FFF78DFD03900DE0019B3C3319460198F0
:101DF000FFF7C9FD039005E0019B002283F8312025
:101E000000E000BF019B9B78002B20D0019B03F1D9
:101E10005400019BD3F82014019B3C331A46FFF772
:101E2000EFFB0390039B002B01D0039B1BE0019B66
:101E300093F85420019B93F8303019461046FFF771
:101E4000E3FB0390039B002B01D0039B0BE0019B62
:101E50005B6B002B06D0019B5B6B019A92F83120E3
:101E6000104698470023184605B05DF804FB00BFF4
:101E700000B585B001900091009B0393019B1B88E6
:101E8000262B10D0262B13DC102B02D0112B05D0C3
:101E90000EE001990398FFF7F3FB0AE0019903981C
:101EA000FFF7FDFB05E001990398FFF722FC00E036
:101EB00000BF00BF05B05DF804FB75DF704700BFD1
:101EC000184676DF704700BF18467ADF704700BFBC
:101ED00018467BDF704700BF1846000084B00346F9
:101EE000ADF806300023039316E00F49039A13461A
:101EF0009B0013449B000B441B88BDF806209A42AC
:101F000007D1039A13469B0013449B00064A1344CF
:101F100006E0039B01330393039B002BE5D00023D2
:101F2000184604B0704700BF10B5002082B0019081
:101F30000B46ADF80230019BBDF802201A80019BD0
:101F400000221A72019B054903F10A020B4603CBDA
:101F50001060516000BF02B0704700BF40B5002064
:101F600082B00190019B4FF6FF721A8000BF02B051
:101F7000704788B00390029111461A460B46ADF89F
:101F800006301346ADF80430039B9B881A46BDF813
:101F9000063013440793039B9B881946039B9B8839
:101FA000BDF80620934228BF13469BB2CB1A069376
:101FB000039BDB881A46BDF8043013440593039B4A
:101FC000DB881946039BDB88BDF80420934228BFB9
:101FD00013469BB2CB1A0493029B5A88039B1B881F
:101FE0009A4205D3029B5A88039B5B889A4201D987
:101FF00000231CE0029B9B881A46069B934205D84F
:10200000029B9B881A46079B934201D200230EE055
:10201000029BDB881A46049B934205D8029BDB880F
:102020001A46059B934201D2002300E00123184683
:1020300008B0704700B583B00190064B9B69002B38
:1020400003D0044B9B690198984700BF03B05DF82B
:1020500004FB00BF24B5002000B585B00346009105
:10206000ADF80630BDF8063000991846FFF725FF99
:102070000390039B002B05D0039B112B02D00398E8
:10208000FFF7D8FF039B002B0CBF01230023DBB21B
:10209000184605B05DF804FB00B589B00190019BBE
:1020A0000793079B9BB21846FFF718FF0690069B05
:1020B000002B42D0069B1A7A224B1B7B9A4215D2E8
:1020C000079B9AB2069B0A3319461046FFF7C4FFD6
:1020D00003468DF813309DF81330002B2DD0069B4E
:1020E0001B7A0133DAB2069B1A7226E0069B0022A5
:1020F0001A72144B1B7C002B0FD0079B9BB23B2109
:102100001846FFF7DEFE0590059B002B05D0059BCA
:10211000082B02D00598FFF78DFF0A4B5B69002B57
:102120000BD000238DF80C30079B9BB2ADF80E301E
:10213000044B5B6903AA1046984700BF09B05DF8DD
:1021400004FB00BF24B5002030B587B00190019B8F
:10215000002B01D10E2353E02B4A019B14461D4650
:102160000FCD0FC495E8070084E80700264B274AE7
:102170001A60019B1B68002B11D0019B1B6818463D
:10218000FFF7A3FE0490049B002B01D0049B37E0D3
:10219000019B1A681D4B1068516803C308E01B4877
:1021A000FFF797FE0490049B002B01D0049B27E0CF
:1021B0000023059320E0059A13469B0013449B00DF
:1021C000134A134403930398FFF7CAFE059B5B0170
:1021D000104A1A44039B5A60039B04330E4A0021A1
:1021E0001846F5F7DBFC0490049B002B01D0032379
:1021F00006E0059B01330593059B002BDBD00023F4
:10220000184607B030BD00BF24B5002040B50020FF
:1022100010B50020F0B400209920030000B587B06D
:1022200003460091ADF80630009B5B7A002B1AD173
:10223000009B1B7A002B03D1164B5B68059302E0D1
:10224000144B9B680593009B5B68BDF806200599BD
:102250001846F5F7D7FC0490049B002B16D0049881
:10226000FFF7E8FE12E0009B00221A72094B5B693F
:10227000002B0BD001238DF80C30BDF80630ADF8E3
:102280000E30044B5B6903AA1046984700BF07B0A5
:102290005DF804FB24B5002000B585B00190019BDA
:1022A000DB7B8DF80F30019B9B88ADF80C309DF8DF
:1022B0000F30012B2CD14FF6FF70FFF70FFE02906D
:1022C000029B002B03D10420FFF7B4FE21E0BDF8F0
:1022D0000C3019460298FFF729FE029B03F10A0011
:1022E000019B03F110014FF6FF7340F2F312FFF769
:1022F00040FE03461A46029B5A72074BDB89002BAD
:1023000007D1BDF80C3002991846FFF787FF00E0AF
:1023100000BF05B05DF804FB24B5002000B587B010
:102320000190019B9B88ADF81630BDF81630184619
:10233000FFF7D4FD0490049B002B0ED0049B5B6838
:102340001846F5F797FC0390039B002B02D00398E7
:10235000FFF770FE0498FFF703FE00BF07B05DF8BB
:1023600004FB000000B587B00190019B0633059384
:10237000059B1A88194BDB899A422BD1059B5B89F7
:10238000022B27D1019B9B88ADF81230BDF812308B
:102390001846FFF7A3FD0390039B002B1AD0059B63
:1023A0000C33184600F074FA0346002B06D0BDF833
:1023B000123003991846FFF731FF0BE0039B5B686F
:1023C0001846F5F757FC0290029B002B02D00298AA
:1023D000FFF730FE00BF07B05DF804FB24B5002016
:1023E00000B585B00190019B9B88ADF80E30BDF81B
:1023F0000E301846FFF772FD0290029B002B15D09D
:10240000029B03F10A00019B03F108014FF6FF73E1
:1024100040F2F312FFF7ADFD03461A46029B5A72D3
:10242000BDF80E3002991846FFF7F8FE00BF05B060
:102430005DF804FB00B583B001900091019B1B88FF
:10244000502B12D0502B18DC122B12D0122B14DC74
:10245000102B02D0112B04D00FE00198FFF71CFFC6
:102460000CE00198FFF75AFF08E00198FFF77AFFA8
:1024700004E00198FFF7B4FF00E000BF00BF03B025
:102480005DF804FB30B58FB00190009100230293FA
:10249000009B002B1AD000230D9314E06B460D997E
:1024A0001846F5F74FFE0346002B09D0029B5A1C35
:1024B00002920D9A92B25B000EA90B4423F82C2CC9
:1024C0000D9B01330D930D9B132BE7D9019B1D46EB
:1024D00002AC0FCC0FC50FCC0FC594E8070085E800
:1024E000070001980FB030BD00B583B00346ADF8CA
:1024F0000630BDF80630132B01D900230CE0BDF8DF
:10250000063019460648F5F7ECFDBDF806301946C9
:102510000448F5F7E6FD0123184603B05DF804FB17
:1025200050B500204CB5002000B585B00346ADF88D
:102530000630002303930DE0039B9B00094A1344DC
:102540000433BDF8062011461846F5F7E2FD039B5B
:1025500001330393039B1D2BEED900BF00BF05B0D1
:102560005DF804FB48B5002000B583B00346ADF824
:102570000630BDF8063019460348F5F7CAFD00BF1E
:1025800003B05DF804FB00BF50B5002030B59BB030
:10259000184B9B68DB431893164B5A6818AB1146CF
:1025A0001846F5F72EFE189A6B4611461846FFF7A7
:1025B00069FF0DAC6D460FCD0FC40FCD0FC495E86C
:1025C000070084E80700002319930BE0199B5B00C8
:1025D0001AAA134433F8303C1846FFF7A5FF199B9D
:1025E000013319930D9B199A9A42EFD300BF00BF94
:1025F0001BB030BD48B5002000B583B001900B463C
:10260000ADF8023013468DF801309DF80130002BF3
:1026100006D0BDF8023019460198F5F762FD05E0D5
:10262000BDF8023019460198F5F773FD00BF03B0FD
:102630005DF804FB00B585B001900091019B9B887B
:10264000ADF80E30019B1B88103B0A2B00F28880EE
:1026500001A252F823F000BF85260300C126030023
:10266000612703006127030061270300612703003E
:102670006127030061270300612703002B27030064
:10268000CD260300FFF782FFBDF80E301846FFF796
:102690002BFF034683F00103DBB2002B05D0324A47
:1026A000F0210420F5F7D6F857E0019BDB7B022BE5
:1026B00053D1BDF80E3019462C48F5F712FD4CE009
:1026C000BDF80E301846FFF74FFF49E0019B1B7A1B
:1026D000C3F30313DBB28DF80D309DF80D30032BDF
:1026E0008CBF01230023DAB2BDF80E301946204812
:1026F000FFF782FF9DF80D30022B8CBF01230023D2
:10270000DAB2BDF80E3019461A48FFF775FF9DF88A
:102710000D30012B8CBF01230023DAB2BDF80E303F
:1027200019461548FFF768FF1AE0019B1B7A002B3A
:1027300015D1019B5B7AC3F3C003DBB2002B14BF3E
:10274000012300238DF80C309DF80C20BDF80E30CD
:1027500019460748FFF750FF01E000BF00E000BF47
:1027600000BF05B05DF804FB4C86030054B50020A3
:1027700060B500205CB5002058B5002000B583B0DE
:102780000346ADF80630BDF80630132B01D90023FF
:1027900006E0BDF8063019460348F5F7D3FC0346BA
:1027A000184603B05DF804FB4CB5002000B583B0BB
:1027B0000346ADF80630BDF806301846FFF7DEFFD9
:1027C0000346002B02D0BDF8063000E01423184663
:1027D00003B05DF804FB00B587B003900B4601928F
:1027E000ADF80A30019B002B01D10E2338E0019B8C
:1027F00000221A60039B002B01D10E2330E0039BC3
:102800001B68002B01D10E232AE0039BDB8803F019
:1028100003039BB2002B01D0072321E0BDF80A304F
:102820001846FFF7C3FF03468DF817309DF81730A1
:10283000142B01D1052313E0039B1B799DF817206E
:102840009A4201D304230BE0039B1B689DF81720D9
:102850000399C98801FB02F21A44019B1A60002304
:10286000184607B05DF804FB82B00190019B1B780D
:102870001AB2019B01331B781B021BB213431BB21C
:102880009BB2184602B07047AADF704700BF1846D7
:1028900000B585B001900198FFF7E6FF0346ADF85B
:1028A0000E30BDF80E3003F00103002B14BF0123DE
:1028B0000023DBB2184605B05DF804FB82B0034686
:1028C00000918DF80730009A13786FF303031370AB
:1028D000009A13786FF3071313709DF80730052BD8
:1028E0005BD801A252F823F0012903001729030045
:1028F000312903004B290300652903007F290300C8
:10290000009A13786FF303031370009A13786FF330
:102910000713137040E0009A1378012161F3030359
:102920001370009A1378012161F30713137033E0D9
:10293000009A1378012161F303031370009A13784E
:10294000022161F30713137026E0009A1378012126
:1029500061F303031370009A1378032161F30713E3
:10296000137019E0009A1378022161F303031370C6
:10297000009A1378012161F3071313700CE0009A99
:102980001378022161F303031370009A1378022174
:1029900061F30713137000BF00BF00BF02B07047A0
:1029A00000B595B0034602910192ADF80E30029B3E
:1029B0009B78002B03D101238DF81E3003E0029B8E
:1029C0009B788DF81E30029B1B88ADF81C3006AB3F
:1029D00003220021184604F0FFF8029B5B7C06AA44
:1029E00011461846FFF76AFF029B9A7C06AB01333B
:1029F00019461046FFF762FF029BDA7B9DF81A30FA
:102A000062F3C3038DF81A30029B1A7C9DF81A30CA
:102A100062F304138DF81A30029B1A7B9DF81A306A
:102A200062F300038DF81A30029B1B7D002B01D04E
:102A3000022200E001229DF81A3062F342038DF871
:102A40001A300DAB1C220021184604F0C5F8029B79
:102A50005B7B03F01003DBB2002B06D1029B5B7B98
:102A600003F02003DBB2002B24D004AB03220021AF
:102A7000184604F0B1F8029BDA7C04AB0133194626
:102A80001046FFF71BFF9DF81030012262F303038D
:102A90008DF810309DF81030012262F307138DF885
:102AA00010309DF81230012262F342038DF812308B
:102AB00004AB1293029B5B7B8DF83430029B9B7BB3
:102AC0008DF8353008AB14220021184604F084F844
:102AD00007AB089306AB0993029B9B88ADF82C309B
:102AE000029B9B68002B06D0029BDB88ADF8283048
:102AF000029B9B680C93029B9B69002B4FD005ABFC
:102B000003220021184604F067F8029B9B691B888A
:102B1000ADF83C30029B9B695B88ADF83E30029B70
:102B20009B695B680E9305AB1193029B9B691B7BB2
:102B300005AA11461846FFF7C1FE029B9B695A7B06
:102B400005AB013319461046FFF7B8FE029B9B699F
:102B50009A7A9DF8163062F3C3038DF81630029B03
:102B60009B69DA7A9DF8163062F304138DF81630FB
:102B7000029B9B691A7A9DF8163062F300038DF868
:102B80001630029B9B699B7B002B01D0022200E048
:102B900001229DF8163062F342038DF81630029B35
:102BA000DB69002B02D0029BDB69109308AA0DA9F8
:102BB000BDF80E00019BFFF767FE0346184615B0EF
:102BC0005DF804FB90DF704700BF1846A5DF704733
:102BD00000BF1846B5DF704700BF184682B00190AD
:102BE000019BF7221A80019B17225A80019B002229
:102BF0001A71019B00225A71019BFB229A71019B61
:102C00001B22DA7100BF02B07047000030B589B0F6
:102C100003460A46ADF806301346ADF80430BDF859
:102C20000430ADF81430BDF80430ADF81630002390
:102C3000ADF818300023ADF81A3003AB00221A604B
:102C40009A8003AA05A9BDF806301846FFF7BAFF17
:102C50000790079B002B39D01E4A1F4BD31ADB0865
:102C60001B0443F00104BDF806500798F6F742FA3A
:102C700003462A4619492046F4F749F8BDF80C30B6
:102C8000002B03D1BDF80E30002B0ED0114A124B91
:102C9000D31ADB081B0443F00100BDF80C301A46C0
:102CA000BDF80E300E49F4F732F8BDF81030002BA5
:102CB0000CD0084A084BD31ADB081B0443F001036D
:102CC000BDF8102007491846F4F710F8079B18467E
:102CD00009B030BDA47303004C7303009086030059
:102CE000DC8603001C87030010B586B001900091BC
:102CF000009B9B88ADF80E30BDF80E30DB00019ACA
:102D0000134406330593019B1A79059B9A71009B26
:102D1000DB7B012B02D0022B05D009E0019B1A8836
:102D2000059B1A8004E0019B5A88059B1A8000BF0E
:102D3000059B1A88059B5B889A4226D9059B1A88B1
:102D4000BDF80E3011461846FFF740FF0490049B73
:102D5000002B03D1059B01225A7116E0049B112B15
:102D600003D1059B01221A710FE0114A114BD31AAE
:102D7000DB081B0443F001040498F6F7BBF9034693
:102D80001A460D492046F3F7B1FF059B9A79059B3A
:102D9000DB799A4208D9059B9B799AB2BDF80E302F
:102DA00011461846FFF732FF00BF06B010BD00BF46
:102DB000A47303004C7303007487030000B583B051
:102DC00001900091009B9B88DB00019A134406331D
:102DD0001846FFF703FF00BF03B05DF804FB00B522
:102DE00087B001900091009B9B88ADF81630009B46
:102DF0005B89ADF81430BDF81630DB00019A13443E
:102E000006330493049B1B88BDF81420934228BF0B
:102E100013469AB2049B5A80049B5B88172B38BFD9
:102E200017239AB2049B5A80019B1B69002B15D073
:102E3000049B5B79002B11D040F67723ADF8083066
:102E4000BDF81630ADF80A30049B5B88ADF80C3045
:102E5000019B1B6902AA114601989847049B002216
:102E60005A71049B00221A7100BF07B05DF804FB81
:102E700010B588B001900091009B9B88ADF81A3086
:102E8000009BDB88ADF81830BDF81A30DB00019AE2
:102E9000134406330593BDF81830172B38BF17239A
:102EA000ADF81830059B1B88BDF81820934228BF49
:102EB00013469AB2059B5A80059B00221A71059B06
:102EC0001A88BDF81A3011461846FFF783FE07909E
:102ED000079B002B0FD0174A174BD31ADB081B0494
:102EE00043F001040798F6F705F903461A4613491B
:102EF0002046F3F7FBFE059B5B79002B16D1019B67
:102F00001B69002B13D040F67723ADF80C30BDF8C9
:102F10001A30ADF80E30059B5B88ADF81030019B80
:102F20001B6903AA11460198984700E000BF08B04A
:102F300010BD00BFA47303004C730300A8870300F7
:102F400030B591B001900091009B04AC1D1D0FCDD8
:102F50000FC40FCD0FC495E8070084E80700BDF843
:102F60001030ADF83E30BDF81420BDF83E30D1B27F
:102F7000019ADB0013440A465A73019B1B69002B1C
:102F800019D002AB00221A609A804DF67A23ADF870
:102F90000830BDF83E30ADF80A30BDF83E30019A39
:102FA000DB0013445B7B8DF80C30019B1B6902AA8C
:102FB00011460198984700BF11B030BD00B587B0E9
:102FC00001900091009B04330593059B1B88DB0057
:102FD000019A134406330493059B9B888DF80F30A8
:102FE000049B9B799DF80F20934228BF13468DF8D0
:102FF0000E30059B1B889DF80E2092B21146184694
:10300000FFF704FE00BF07B05DF804FB00B585B014
:1030100001900091019B002B01D10E231DE0019B2B
:10302000009A1A61019BF7221A80019BF7225A80AD
:10303000019BFB221A71002303930AE0039BDB0030
:10304000019A134406331846FFF7C8FD039B01336A
:103050000393039B002BF1D00023184605B05DF8C5
:1030600004FB82B001900B46ADF80230019B002BAF
:1030700001D10E230EE0BDF80230162B03D9BDF8A6
:103080000230F72B01D9072304E0019BBDF8022091
:103090001A800023184602B07047000010B586B0B1
:1030A00001900091009B0593019B9B88ADF8123025
:1030B000BDF81230002B40F09880019B1B88552BE7
:1030C00048D0552B55DC242B32DC102B51DB103B28
:1030D000142B4ED801A252F823F000BF3731030061
:1030E0004131030073310300733103007331030076
:1030F0007331030073310300733103007331030034
:103100007331030073310300733103007331030023
:103110007331030073310300733103007331030013
:103120007331030073310300693103005F31030021
:103130003A2B0AD01DE001990598FFF7D5FD19E05B
:1031400001990598FFF73AFE14E001990598FFF7F9
:1031500046FE0FE001990598FFF78AFE0AE0019903
:103160000598FFF7EDFE05E001990598FFF726FFAA
:1031700000E000BFBDF81230059ADB0013449B7AD3
:10318000002B33D0BDF81230059ADB001344DA88E7
:10319000BDF8123011461846FFF718FD0390039B47
:1031A000002B0ED1BDF81230059ADB00134400222B
:1031B0009A72BDF81230059ADB0013440122DA72CC
:1031C00014E0039B112B11D0094A0A4BD31ADB08D8
:1031D0001B0443F001040398F5F78CFF03461A46DD
:1031E00005492046F3F782FD00E000BF06B010BDA0
:1031F000A47303004C73030074870300B0DF7047AF
:1032000000BF184666DF704700BF184682B00190C5
:103210000091019B002B01D10E2316E0009B002B97
:1032200001D10E2311E0019B1B78DE2B01D1082375
:103230000BE0009B1A68019B5A60019BDE221A700A
:10324000019B4FF6FF725A800023184602B0704768
:1032500082B001900B46ADF80230019B002B01D1EA
:103260000E230AE0019B1B78DE2B01D0082304E02B
:10327000019BBDF802205A800023184602B0704717
:1032800000B585B00190019B1B7A002B18D0019BE3
:103290005B8800211846FFF7B5FF0390039B002BC6
:1032A00003D1019B00221A720AE0039B112B03D168
:1032B000019B01221A7203E0019B5B680398984707
:1032C00000BF05B05DF804FB00B583B0019000912C
:1032D000009B1B79012B0BD1009B1A88019B5B88FB
:1032E0009A4205D1019B01221A720198FFF7C8FF8B
:1032F00000BF03B05DF804FB82B00190009100BFF5
:1033000002B0704700B589B001900091009B1A8807
:10331000019B5B889A4236D1009B02330793079B3F
:103320001B78022B31D1079B1B7A042B07D0079BFC
:103330001B7A062B03D0079B1B7A052B27D102ABE8
:1033400000221A605A609A60DA6002238DF8083011
:103350004FF4C073ADF80C30079B1B7A052B02D1DC
:103360000023ADF80C30009B1B8802AA11461846BA
:10337000FFF744FF0690069B002B09D0019B5B687A
:103380000698984704E000BF02E000BF00E000BFDD
:1033900009B05DF804FB00B585B001900091009B79
:1033A000002B40D0019B002B3FD0009B0393039B3D
:1033B0001B78DE2B3BD1019B9A88039B5B889A424A
:1033C00002D10398FFF75CFF019B1B88512B18D09B
:1033D000512B2EDC112B1BD0112B2ADC012B02D000
:1033E000022B07D025E0019B043319460398FFF711
:1033F0006BFF21E0019B043319460398FFF77CFF24
:103400001AE0019B043319460398FFF77BFF13E092
:10341000019B9A88039B5B889A420CD1039B4FF6D1
:10342000FF725A8007E000BF06E000BF04E000BF63
:1034300002E000BF00E000BF05B05DF804FBA8DFBC
:10344000704700BF1846ADDF704700BF184662DF07
:10345000704700BF184600B58FB00190009100235F
:103460000393019B5869009B9B8803AA1946FFF7A9
:10347000B2F90D9005AB08220021184603F0ACFB11
:1034800004AB06930223ADF814300023ADF81630D8
:10349000009B9888019B1B8905AA1946FFF7D3FF5B
:1034A0000D900D9B002B26D1019B9B69002B22D0F8
:1034B000069B1846FFF7ECF90346002B1BD0039B35
:1034C000002B02D0039B01221A7007AB18220021A7
:1034D000184603F081FB02238DF81C30019B0893F2
:1034E000009B9B88ADF82430039B0A93019B9B694A
:1034F00007AA1046984700BF0FB05DF804FB00B55F
:103500008DB001900091009B06330B93019B58698D
:10351000009B9B8803AA1946FFF75DF90A9004AB4C
:1035200018220021184603F057FB019B0593009BCE
:103530009B88ADF81830039B07930B9B1A88019B5F
:103540001B899A4225D10B9B5B89022B21D1039BBE
:10355000002B38D00B9B0C331846FFF799F9034624
:10356000002B06D0039B01221A7002238DF8103025
:1035700005E0039B00221A7003238DF81030019B95
:103580009B69002B1FD0019B9B6904AA104698479A
:1035900019E00B9B1A88019B9B899A4214D1019BCD
:1035A0009B69002B10D000238DF810300B9B0C333F
:1035B00008930B9B5B89ADF82430019B9B6904AA9F
:1035C0001046984700E000BF00BF0DB05DF804FB57
:1035D00000B58BB001900091019B5869009B9B88BE
:1035E00002AA1946FFF7F7F80990099B002B1ED194
:1035F000029B1B78002B1BD0019B9B69002B17D0D3
:1036000003AB18220021184603F0E6FA01238DF8D7
:103610000C30019B0493009B9B88ADF81430029BF7
:103620000693019B9B6903AA1046984700E000BFE0
:103630000BB05DF804FB00B585B001900091009BD4
:10364000002B1ED0019B002B1BD0009B0393019BE2
:103650001B88572B10D0572B15DC102B02D0502B6A
:1036600005D010E001990398FFF7F5FE0CE00199F1
:103670000398FFF744FF07E001990398FFF7A8FFBD
:1036800002E000BF00E000BF05B05DF804FB0000F1
:1036900010B592B0019000914F4B0AAC0FCB84E86B
:1036A0000F00019B002B01D10E2391E0009B002B0A
:1036B00001D10E238CE0009B1A68019B9A61019A4C
:1036C0000AAB11461846FFF7C2FE1190119B1093EA
:1036D000109B002B01D0109B7AE0019B1B788DF88A
:1036E0003A300123ADF83830019B9A1C0EAB1946D5
:1036F0000120FFF7A4FE1190119B0F930F9B002B4D
:1037000001D00F9B64E002AB20220021184603F099
:1037100063FA0223ADF80830019B1B788DF80A305C
:10372000F423ADF80C300123ADF80E3001238DF8F1
:1037300014309DF8153043F008038DF815309DF8CE
:10374000153043F004038DF8153001238DF819303E
:1037500001238DF81A30019B5888019B03F10C025C
:1037600002AB1946FFF71CF91190119B002B01D0F9
:10377000119B2DE002AB20220021184603F02CFA09
:103780000323ADF80830019B1B788DF80A30F42331
:10379000ADF80C300123ADF80E3001238DF8143054
:1037A0009DF8153043F010038DF8153001238DF886
:1037B000193001238DF81A3001238DF81B30019B3D
:1037C0005888019B1A1D02AB1946FFF7E9F803461A
:1037D000184612B010BD00BFE087030082B0034658
:1037E0008DF807309DF90730002B0CDB9DF8073072
:1037F00003F01F0205499DF907305B09012000FA1B
:1038000002F241F8232000BF02B0704700E100E05F
:1038100082B003468DF807309DF90730002B09DB95
:103820000B4A9DF90730134493F80033DBB25B0970
:10383000DBB20AE0074A9DF8073003F00F03043BB0
:1038400013441B7EDBB25B09DBB2184602B0704743
:1038500000E100E000ED00E000B583B00190019BC5
:10386000002B03D10449C420F4F7BEFB019B5B6825
:10387000184603B05DF804FBF087030010DF7047C3
:1038800000BF184682B003468DF807309DF9073017
:103890001F2B0CDC9DF907300F4A22FA03F303F0CB
:1038A0000103002B14BF01230023DBB210E09DF9BC
:1038B00007303F2B0BDC9DF90730203B012202FA39
:1038C00003F3002B14BF01230023DBB200E001232C
:1038D000184602B0704700BFFC06FFBD82B00190E1
:1038E000019B072B07D8EC22019B42FA03F303F05C
:1038F0000103002B01D1002300E00123184602B090
:103900007047000000B583B003468DF807309DF97D
:1039100007301846FFF7B6FF0346002B02D142F2EC
:1039200001032EE09DF907301846FFF771FF0346AB
:103930001846FFF7D3FF0346002B02D142F20203E1
:103940001FE0124B9B68002B15D09DF907305B09D7
:103950000E4A52F823209DF8073003F01F0301217F
:1039600001FA03F319469DF907305B090A43074939
:1039700041F8232004E09DF907301846FFF72EFF99
:103980000023184603B05DF804FB00BF0C32002092
:1039900000B587B003468DF8073002AB14491846CE
:1039A000F5F74CFB17E002AB1846FFF755FF059003
:1039B000059B1B680493059B59689DF80720049B91
:1039C000104698470346002B01D111230BE002ABB0
:1039D0001846F5F75DFB02AB1846FFF73DFF0346BF
:1039E000002BE0D10023184607B05DF804FB00BFB0
:1039F0008088030000B587B003468DF8073002AB1E
:103A000011491846F5F71AFB12E002AB1846FFF70A
:103A100023FF0590059B1B680493059B59689DF83F
:103A20000720049B1046984702AB1846F5F730FB79
:103A300002AB1846FFF710FF0346002BE5D100BF8D
:103A400000BF07B05DF804FB8C88030000B583B0AD
:103A50001620FFF757FF0190019B0093009B002B5E
:103A600004D0044AA1210098F3F7F4FE00BF03B08C
:103A70005DF804FB4888030000B585B0234B1B7834
:103A8000002B01D008233CE0214B01221A700020BA
:103A9000FFF77EFF0346112B01D1002331E0002008
:103AA000FFF7A8FF1B4B1B68029300238DF807301C
:103AB0000DF107031846F4F7FDF902AB1649184655
:103AC000FFF7DCFE0390039B002B0CBF01230023B8
:103AD000DAB20E4B1A709DF807301846F4F700FA68
:103AE000039B002B01D0039B0BE0094B00221A70B3
:103AF0000A4B00221A70FFF7A9FF0120FFF77AFF97
:103B00000023184605B05DF804FB00BFC4B50020D3
:103B1000C6B500207C88030071780200C5B500207E
:103B2000014B1B7818467047C4B5002000B585B01E
:103B30006B4611491846F5F781FA10E06B461846B6
:103B4000FFF78AFE0390039B1B680293039B5A684E
:103B5000029B104698476B461846F5F799FA6B4654
:103B60001846FFF779FE0346002BE7D100BF00BFE0
:103B700005B05DF804FB00BF9888030008B5FFF7A7
:103B8000D5FF00BF08BD60DF704700BF184669DF82
:103B9000704700BF184661DF704700BF184600003D
:103BA00000B583B00190019B002B03D10449C420D0
:103BB000F4F71AFA019B5B68184603B05DF804FB42
:103BC000A488030082B00190019B002B01D10E2339
:103BD00004E0044B1A46019B1A600023184602B009
:103BE000704700BFD82A002010B586B00346009168
:103BF0008DF807300098FFF7E5FF0590059B002B37
:103C000001D0059BECE002AB0C220021184602F02B
:103C1000E3FF9DF807308DF8083001238DF80A3056
:103C20000623ADF80C30009B1A6802AB1946202021
:103C3000FFF7ADFF0590059B002B0FD06A4A6B4B39
:103C4000D31ADB081B0443F001040598F5F752FA78
:103C500003461A4666492046F3F748F802AB0C22A1
:103C60000021184602F0B8FF01238DF80930002327
:103C70008DF80A3000238DF80B30009B1A6802ABD8
:103C800019464020FFF783FF0590059B002B0FD0BE
:103C9000554A564BD31ADB081B0443F00104059820
:103CA000F5F728FA03461A4652492046F3F71EF85C
:103CB00002AB0C220021184602F08EFF9DF807305F
:103CC0008DF80830F723ADF80A30009B1A6802AB74
:103CD00019462320FFF75BFF0590059B002B0FD0B3
:103CE000414A424BD31ADB081B0443F001040598F8
:103CF000F5F700FA03461A463F492046F2F7F6FF69
:103D000002AB0C220021184602F066FF01238DF859
:103D10000830009B1A6802AB19460120FFF737FFF5
:103D20000590059B002B0FD02F4A304BD31ADB0890
:103D30001B0443F001040598F5F7DCF903461A4625
:103D40002E492046F2F7D2FF02AB0C220021184682
:103D500002F042FF4FF4B0630293009B1A6802AB7B
:103D60001946A120FFF713FF0590059B002B0FD0EC
:103D70001D4A1E4BD31ADB081B0443F001040598AF
:103D8000F5F7B8F903461A461D492046F2F7AEFF8B
:103D900002AB0C220021184602F01EFF9DF80830ED
:103DA0006FF300038DF80830009B1A6802AB1946C8
:103DB000A020FFF7ECFE0590059B002B0FD00A4AD0
:103DC0000A4BD31ADB081B0443F001040598F5F7EE
:103DD00091F903461A460B492046F2F787FF002364
:103DE000184606B010BD00BFB47303004C73030047
:103DF000008903004889030094890300DC890300DB
:103E0000288A03007C8A030082B04FF08053D3F8E5
:103E10000C319B020193019B03F10053184602B041
:103E20007047000010B584B00190019B1B6803939C
:103E30000198FFF7A8FE0290019B1B68039A9A4223
:103E400029D2224A224BD31ADB081B0443F0020377
:103E500020491846F2F73CFF1C4A1D4BD31ADB08D9
:103E60001B0443F00200019B1B68039A1A49F2F7F6
:103E70004EFF164A164BD31ADB081B0443F002040C
:103E8000FFF7C2FF0246019B1B68D31A1A4613496B
:103E90002046F2F72BFF029B002B03D1104B01228F
:103EA0001A700FE0094A0A4BD31ADB081B0443F0CF
:103EB00001040298F5F71EF903461A4609492046FF
:103EC000F2F714FF029B184604B010BDB473030050
:103ED0004C730300D08A0300008B0300348B030073
:103EE000C7B50020608B030000B5ADF5077D86AB3C
:103EF000A3F505731860244B1B7883F00103DBB234
:103F0000002B3BD14FF4FA73ADF806320DF20622C6
:103F100002AB11461846FFF73EFE8590859B002BAD
:103F200003D0859B052B22D129E002AB84937FAB84
:103F300016491846F5F782F811E07FAB1846FFF7EF
:103F40002FFE8390839B1B688293839B5A68829B7E
:103F50001146849898477FAB1846F5F799F87FABE0
:103F60001846FFF71DFE0346002BE6D1CAE7084AB4
:103F700040F23B118598F3F76DFC00E000BF0DF5B2
:103F8000077D5DF804FB00BFC7B50020B88B0300B8
:103F9000808B030000B583B00190019B002B03D1FF
:103FA0000449C420F4F720F8019B5B68184603B06D
:103FB0005DF804FBC48B03004BDF704700BF18465D
:103FC00000B589B0019004AB1846FFF7F5FF0790E4
:103FD000079B002B03D0079B052B20D124E002ABCD
:103FE00013491846F5F72AF811E002AB1846FFF717
:103FF000D1FF0690069B1B680593049A069B59689F
:10400000059B1046984702AB1846F5F741F802ABFE
:104010001846FFF7BFFF0346002BE6D1D3E7054A5A
:104020006B210798F3F716FC00BF09B05DF804FB9D
:10403000588C0300208C030000B585B003900291DA
:104040000192039B1B681B68002B03D10749F020DA
:10405000F3F7CAFF039B1B681B68019A0299039838
:1040600098470346184605B05DF804FB648C0300CE
:1040700010B582B001900091019B1B689B68002BDA
:1040800004D113494FF48970F3F7AEFF019B1B680D
:104090005B69002B04D10E4940F21310F3F7A4FF23
:1040A000009B1C68019B1B685B690198984703464D
:1040B0001B689C4201D3072306E0019B1B689B6899
:1040C0000099019898470346184602B010BD00BFFA
:1040D000648C030010B582B001900091019B1B68B5
:1040E000DB68002B04D113494FF49770F3F77CFF82
:1040F000019B1B685B69002B04D10E4940F22F1015
:10410000F3F772FF009B1C68019B1B685B690198B9
:10411000984703461B689C4201D3072306E0019B96
:104120001B68DB680099019898470346184602B05F
:1041300010BD00BF648C030000B585B003900B4632
:1041400001928DF80B30039B1B681B69002B04D177
:1041500008494FF4A370F3F747FF039B1B681B69E3
:104160009DF80B10019A039898470346184605B02E
:104170005DF804FB648C030000B583B00190019BE3
:104180001B685B69002B04D107494FF4AA70F3F751
:104190002BFF019B1B685B690198984703461846F3
:1041A00003B05DF804FB00BF648C030000B585B06C
:1041B00001900091009B9B688DF80F30154B1B7888
:1041C0009DF80F209A4203D313493F20F3F70CFFC9
:1041D000009B1B78032B17D8104B19689DF80F20F4
:1041E00013465B0013449B000B44009A52781A72EA
:1041F0000A4B19689DF80F2013465B0013449B007F
:104200000B4400229A7200E000BF00BF05B05DF8C9
:1042100004FB00BFCCB50020A08C0300C8B5002073
:1042200020BF00BF7047000000B585B003468DF881
:1042300007305D4B1B68002B03D15C495920F3F715
:10424000D3FE5B4B1B789DF807209A4201D30323D2
:10425000A6E0554B19689DF8072013465B001344F0
:104260009B000B441B68002B01D1032398E04E4BAD
:1042700019689DF8072013465B0013449B000B440C
:104280005B7ADBB203F00103002B0BD1464B1968BC
:104290009DF8072013465B0013449B000B445B7A98
:1042A000DBB27DE0404B19689DF8072013465B00A8
:1042B00013449B000B445B68002B0AD13A4B1968EE
:1042C0009DF8072013465B0013449B000B44394ABA
:1042D0005A60354B19689DF8072013465B0013445C
:1042E0009B000B4401229A722F4B19689DF80720FE
:1042F00013465B0013449B000B441B689DF807208A
:104300002D491846FFF798FE0390039B002B3CD1E4
:104310000AE0254B19689DF8072013465B001344FB
:104320009B000B445B6898471F4B19689DF807205A
:1043300013465B0013449B000B449B7ADBB2002BBB
:10434000E7D1194B19689DF8072013465B00134409
:104350009B000B441B7A002B17D1134B19689DF857
:10436000072013465B0013449B000B445B7AD9B2D1
:104370000D4B18689DF8072013465B0013449B0003
:10438000034421F00102D2B25A72074B19689DF81A
:10439000072013465B0013449B000B445B7ADBB29F
:1043A000184605B05DF804FBC8B50020A08C0300DA
:1043B000CCB5002021420300AD41030000B583B01D
:1043C00003468DF807300F4B1B68002B03D10E49B5
:1043D000B320F3F709FE0D4B1B789DF807209A4296
:1043E00001D301230AE0074B19689DF80720134603
:1043F0005B0013449B000B445B7ADBB2184603B0AE
:104400005DF804FBC8B50020A08C0300CCB50020EB
:1044100000B589B002910192009303468DF80F30E8
:104420003F4B1B68002B03D13E49BE20F3F7DCFD58
:104430003D4B1B789DF80F209A4202D2009B002B27
:1044400001D1042368E0364B19689DF80F2013460C
:104450005B0013449B000B441B68002B0ED0304BB9
:1044600019689DF80F2013465B0013449B000B4412
:104470005B7ADBB203F00103002B01D003234BE096
:10448000019B0493009B0593029B0693244B1968A0
:104490009DF80F2013465B0013449B000B44012240
:1044A0009A721F4B19689DF80F2013465B00134446
:1044B0009B000B441B6804AA11461846FFF7D8FD61
:1044C0000790079B002B26D10AE0154B19689DF831
:1044D0000F2013465B0013449B000B445B68984716
:1044E0000F4B19689DF80F2013465B0013449B0087
:1044F0000B449B7ADBB2002BE7D1094B19689DF87E
:104500000F2013465B0013449B000B441B7A002BC7
:1045100001D1002300E00123184609B05DF804FB37
:10452000C8B50020A08C0300CCB5002000B589B030
:1045300002910192009303468DF80F30484B1B689F
:10454000002B03D14749E520F3F74EFD464B1B787E
:104550009DF80F209A4202D2009B002B01D1042328
:1045600079E03F4B19689DF80F2013465B00134418
:104570009B000B441B68002B0ED0394B19689DF82B
:104580000F2013465B0013449B000B445B7ADBB2A5
:1045900003F00103002B01D003235CE0304B1968CA
:1045A0009DF80F2013465B0013449B000B445B7A7D
:1045B000DBB203F00403002B01D002234BE0019B8C
:1045C0000493009B0593029B0693254B19689DF865
:1045D0000F2013465B0013449B000B4401229A7288
:1045E0001F4B19689DF80F2013465B0013449B0076
:1045F0000B441B6804AA11461846FFF76BFD079091
:10460000079B002B26D10AE0154B19689DF80F2057
:1046100013465B0013449B000B445B689847104BA8
:1046200019689DF80F2013465B0013449B000B4450
:104630009B7ADBB2002BE7D1094B19689DF80F205C
:1046400013465B0013449B000B441B7A002B01D1E3
:10465000002300E00123184609B05DF804FB00BF09
:10466000C8B50020A08C0300CCB5002000B587B0F1
:10467000034600928DF807300B468DF80630454B07
:104680001B68002B04D144494FF48870F3F7ACFC4D
:10469000424B1B789DF807209A4201D3042375E012
:1046A0009DF80630022B4BD0022B6DDC002B02D084
:1046B000012B22D068E001238DF80B30354B1968AF
:1046C0009DF8072013465B0013449B000B441B68B6
:1046D0000DF10B0200211846FFF72EFD0390039BFE
:1046E000002B02D0039B112B04D19DF80B30002B23
:1046F000E4D100E000BF002348E0264B19689DF894
:10470000072013465B0013449B000B441B68002BDF
:1047100001D103233AE0009B04931E4B19689DF8D6
:10472000072013465B0013449B000B441B6818468C
:10473000FFF722FD03461A68049B1A60002325E058
:10474000144B19689DF8072013465B0013449B0027
:104750000B441B68002B01D1032317E0009B05933A
:104760000C4B19689DF8072013465B0013449B000F
:104770000B441B681846FFF7FFFC03465B689AB2C0
:10478000059B1A80002301E000BF0123184607B0F3
:104790005DF804FBC8B50020A08C0300CCB5002058
:1047A00000B583B001900091019B002B04D1084912
:1047B0004FF4A470F3F718FC064A019B1360009BAA
:1047C000DAB2054B1A7000BF03B05DF804FB00BFFE
:1047D000A08C0300C8B50020CCB5002084B00190A7
:1047E000019B01331B78ADF80E30BDF80E301B0273
:1047F0001AB2019B1B781BB213431BB2ADF80E30EB
:10480000BDF80E30184604B0704784B00190019B8B
:1048100003331B780393039B1B02019A0232127825
:1048200013430393039B1B02019A01321278134333
:104830000393039B1B02019A127813430393039B78
:10484000184604B0704782B001900B46ADF80230B4
:10485000019B5A1C0192BDF80220D2B21A70BDF819
:1048600002301B0AADF80230019B5A1C0192BDF8C0
:104870000220D2B21A7000BF02B0704782B001901D
:104880000091019B5A1C0192009AD2B21A70009BAF
:104890001B0A0093019B5A1C0192009AD2B21A7013
:1048A000009B1B0A0093019B5A1C0192009AD2B2F2
:1048B0001A70009B1B0A0093019B5A1C0192009ADC
:1048C000D2B21A7000BF02B0704786B00390029156
:1048D0000192039B0593029B0493019B002B0DD037
:1048E000049A531C0493059B591C059112781A7065
:1048F000019B013B0193019B002BF1D100BF06B04E
:10490000704786B0039002910192039B0593059B2B
:104910005A1C0592029AD2B21A70019B013B019374
:10492000019B002BF3D100BF00BF06B0704788B0D9
:10493000039002910192039B0793029B069300232D
:104940000593079B5A1C07921B781946069B5A1C15
:1049500006921B78CB1A0593019B013B0193019BA7
:10496000002B02D0059B002BEBD0059B184608B00E
:10497000704782B00190009102E0019B01330193E6
:10498000019B1B78002B05D0019B1B781A46009BCE
:104990009342F2D1019B1B78184602B0704700B5D4
:1049A00087B0019000238DF80F30019BDB78002B3E
:1049B00035D0019BDB6A0593019B5878019B03F17D
:1049C00030010123059AFFF7B1FD0346002B03D008
:1049D00001238DF80F3022E0019B0022DA70019B49
:1049E0001B6A059AD21A019B9B699A4217D2019BB6
:1049F0009B78049310E0019B9B69059A13440593EF
:104A0000019B5878019B03F130010123059AFFF7C0
:104A10008DFD049B013B0493049B012BEBD89DF877
:104A20000F30184607B05DF804FB00B585B0019063
:104A3000009100238DF80F30019BDB6A009A9A42A7
:104A40001ED00198FFF7ABFF03468DF80F309DF89D
:104A50000F30002B14D1019B5878019B03F13001DA
:104A60000123009AFFF7D4FC0346002B05D04FF03A
:104A7000FF33009301238DF80F30019B009ADA6217
:104A80009DF80F30184605B05DF804FB00B585B001
:104A900001900198FFF783FF03468DF80F309DF8D2
:104AA0000F30002B59D1019B1B78032B48D1019B60
:104AB0001B79012B44D1019B30334FF4007200214C
:104AC0001846FFF71EFF019B303303F5FF734AF6CC
:104AD00055211846FFF7B7FE019B3033224918468F
:104AE000FFF7CCFE019B303303F5F2731F491846E4
:104AF000FFF7C4FE019B303303F5F472019B1B6981
:104B000019461046FFF7BAFE019B303303F5F672E3
:104B1000019BDB6819461046FFF7B0FE019BDB697D
:104B20005A1C019BDA62019B5878019B03F130010A
:104B3000019BDA6A0123FFF7F9FC019B00221A713D
:104B4000019B5B78002200211846FFF78FFD03468A
:104B5000002B02D001238DF80F309DF80F3018463E
:104B600005B05DF804FB00BF5252614172724161B1
:104B700082B001900091009B023B0093019B5B6916
:104B8000023B009A9A4201D3002308E0019B5B8913
:104B90001A46009B03FB02F2019B9B6A13441846D2
:104BA00002B0704700B587B001900091019B1B686F
:104BB0000493009B012B04D9049B5B69009A9A42E1
:104BC00002D3012305938FE04FF0FF330593049B3D
:104BD0001B78032B62D0032B7CDC012B02D0022B31
:104BE00042D077E0009B0393039B5B08039A134436
:104BF0000393049B1A6A039B5B0A134419460498A7
:104C0000FFF713FF0346002B67D1039B5A1C039247
:104C1000C3F30803049A134493F830300293049BBF
:104C20001A6A039B5B0A134419460498FFF7FDFEBA
:104C30000346002B53D1039BC3F30803049A134488
:104C400093F830301B021A46029B13430293009BD9
:104C500003F00103002B02D0029B1B0902E0029B20
:104C6000C3F30B0305933FE0049B1A6A009B1B0AE6
:104C7000134419460498FFF7D8FE0346002B30D1A1
:104C8000049B03F13002009B5B0003F4FF731344A9
:104C90001846FFF7A3FD0346059325E0049B1A6A17
:104CA000009BDB09134419460498FFF7BEFE034638
:104CB000002B18D1049B03F13002009B9B0003F4EE
:104CC000FE7313441846FFF7A0FD034623F070431C
:104CD000059309E00123059306E000BF04E000BF4F
:104CE00002E000BF00E000BF059B184607B05DF87A
:104CF00004FB10B588B003900291019202238DF855
:104D00001F30029B012B40F2DA80039B5B69029A01
:104D10009A4280F0D480039B1B78032B00F09C8088
:104D2000032B00F3D580012B02D0022B72D0CFE0F1
:104D3000029B0693069B5B08069A13440693039B0B
:104D40001A6A069B5B0A134419460398FFF76DFE27
:104D500003468DF81F309DF81F30002B40F0B180C6
:104D6000039B03F13002069B591C0691C3F3080311
:104D700013440593029B03F00103002B0DD0059B08
:104D80001B785BB203F00F035AB2019BDBB21B012D
:104D90005BB213435BB2DBB201E0019BDBB2059A6D
:104DA0001370039B0122DA70039B1A6A069B5B0A4D
:104DB000134419460398FFF738FE03468DF81F3059
:104DC0009DF81F30002B7ED1039B03F13002069B20
:104DD000C3F3080313440593029B03F00103002B64
:104DE00003D0019B1B09DBB20EE0059B1B785BB275
:104DF00023F00F035AB2019B1B0A5BB203F00F03AF
:104E00005BB213435BB2DBB2059A1370039B0122C2
:104E1000DA705DE0039B1A6A029B1B0A1344194671
:104E20000398FFF702FE03468DF81F309DF81F30F0
:104E3000002B4AD1039B03F13002029B5B0003F479
:104E4000FF731344019A92B211461846FFF7FBFC18
:104E5000039B0122DA703BE0039B1A6A029BDB0989
:104E6000134419460398FFF7E0FD03468DF81F3001
:104E70009DF81F30002B2AD1019B23F07044039B27
:104E800003F13002029B9B0003F4FE7313441846A7
:104E9000FFF7BBFC034603F0704323430193039BDE
:104EA00003F13002029B9B0003F4FE73134401994B
:104EB0001846FFF7E3FC039B0122DA7008E000BF0D
:104EC00006E000BF04E000BF02E000BF00E000BF5A
:104ED0009DF81F30184608B010BD00B589B003908A
:104EE0000291019200238DF81F30039B1B680693EB
:104EF000029B012B04D9069B5B69029A9A4201D35B
:104F0000022351E0019B002B0FD04FF0FF3201999B
:104F10000698FFF7EEFE03468DF81F309DF81F3010
:104F2000002B02D09DF81F303EE002990398FFF756
:104F300039FE0590059B002B34D0059B012B01D138
:104F4000022331E0059BB3F1FF3F01D101232BE0A8
:104F5000002202990698FFF7CCFE03468DF81F3019
:104F60009DF81F30002B02D09DF81F301CE0069BDF
:104F70001A69069B5B69023B9A420BD2069B1B692E
:104F80005A1C069B1A61069B1B7943F00103DAB297
:104F9000069B1A71059B0293069B5B69029A9A42D3
:104FA000C3D300E000BF0023184609B05DF804FB3E
:104FB00000B589B001900091019B1B680493009B90
:104FC000002B0DD1049BDB680693069B002B04D0BD
:104FD000049B5B69069A9A421BD30123069318E04F
:104FE00000990198FFF7DEFD0390039B012B01D888
:104FF000012375E0039BB3F1FF3F01D1039B6FE0F9
:10500000049B5B69039A9A4201D2039B68E0009B70
:105010000693069B0793079B01330793049B5B69E9
:10502000079A9A4207D302230793079A069B9A424C
:1050300001D9002354E007990198FFF7B3FD0390CD
:10504000039B002B0ED0039B012B03D0039BB3F1DA
:10505000FF3F01D1039B43E0079A069B9A42DAD1B6
:1050600000233DE000BF4FF0FF3207990498FFF79F
:1050700040FE03468DF817309DF81730002B0AD1FB
:10508000009B002B07D0079A00990498FFF731FE88
:1050900003468DF817309DF81730002B16D1049B6E
:1050A000079ADA60049B1A69049B5B69023B9A4287
:1050B00004D2049B1B695A1E049B1A61049B1B7932
:1050C00043F00103DAB2049B1A7108E09DF817302F
:1050D000012B02D14FF0FF3300E001230793079B20
:1050E000184609B05DF804FB00B587B00190009147
:1050F000019B1B680493009BB3F5001F04D2009B27
:1051000003F01F03002B01D0022363E0019B009AF0
:105110001A61019B9B680593059B002B06D1049B9C
:105120001B78022B02D9049B5B6A0593059B002B1D
:105130000CD1009B5B09049A1289934201D302238C
:1051400048E0049B5A6A019B9A6129E0049B5B89B1
:105150005B02039319E0019B05991846FFF722FDB6
:105160000590059BB3F1FF3F01D1012332E0059B80
:10517000012B04D9049B5B69059A9A4201D302234F
:1051800028E0009A039BD31A0093009A039B9A424B
:10519000E1D205990498FFF7EBFC0246019B9A6166
:1051A000019B059A5A61019B9B69002B01D1022347
:1051B00010E0019B9A69009B5B0A1A44019B9A616B
:1051C000049B03F13002009BC3F308031A44019BC4
:1051D000DA610023184607B05DF804FB00B587B01C
:1051E00001900091019B1B680393019B1B69203375
:1051F0000293019B9B69002B03D0029BB3F5001F18
:1052000001D30423AAE0029BC3F30803002B40F060
:105210009880019B9B695A1C019B9A61019B5B6969
:10522000002B0BD1029B5B09039A12899342C0F0B9
:105230008880019B00229A6104238FE0029B5B0A15
:10524000039A5289013A1340002B7AD1019A019BAB
:105250005B6919461046FFF7A5FC0590059B012BDD
:1052600001D802237AE0059BB3F1FF3F01D101236E
:1052700074E0039B5B69059A9A4258D3009B002B0C
:1052800004D1019B00229A61042367E0019A019BEB
:105290005B6919461046FFF78BFE0590059B002BB6
:1052A00001D107235AE0059B012B01D1022355E0D0
:1052B000059BB3F1FF3F01D101234FE00398FFF7B6
:1052C0006EFB0346002B01D0012347E0039B3033E4
:1052D0004FF4007200211846FFF713FB00230493DC
:1052E00005990398FFF744FC0246039BDA6212E03B
:1052F000039B0122DA700398FFF751FB0346002B52
:1053000001D001232AE0049B01330493039BDB6A51
:105310005A1C039BDA62039B5B891A46049B9342E7
:10532000E6D3039BDA6A049BD21A039BDA62019BE1
:10533000059A5A6105990398FFF71AFC0246019BEA
:105340009A61019B029A1A61039B03F13002029B4E
:10535000C3F308031A44019BDA610023184607B01F
:105360005DF804FB00B587B001900091019B1B68BC
:10537000039300210198FFF7B7FE03468DF817301D
:105380009DF81730002B2FD100230493019B9B69BC
:1053900019460398FFF749FB03468DF817309DF82F
:1053A0001730002B1FD1019BDB691B78E52B04D044
:1053B000019BDB691B78002B07D1049B013304930D
:1053C000049A009B9A4202D10EE00023049301212B
:1053D0000198FFF703FF03468DF817309DF817304B
:1053E000002BD3D000E000BF9DF81730042B02D172
:1053F00007238DF817309DF81730184607B05DF871
:1054000004FB00B585B001900091009B1A3318464B
:10541000FFF7E4F903460393019B1B78032B09D1A3
:10542000009B14331846FFF7D9F903461B04039A6F
:1054300013430393039B184605B05DF804FB00B5C6
:1054400085B0039002910192029B1A33019A92B2A5
:1054500011461846FFF7F7F9039B1B78032B09D178
:10546000029B03F11402019B1B0C9BB219461046D0
:10547000FFF7E9F900BF05B05DF804FB00B587B0A0
:105480000190009104238DF81730019B1B68049351
:1054900049E0019B9B6919460498FFF7C6FA034649
:1054A0008DF817309DF81730002B41D1019BDB6937
:1054B0001B788DF80F309DF80F30002B03D104239B
:1054C0008DF8173039E0019BDB690B331B7803F053
:1054D0003F038DF80E30019B9DF80E209A719DF8C8
:1054E0000F30E52B14D09DF80F302E2B10D09DF8E7
:1054F0000E300F2B0CD09DF80E3023F02003082B1C
:105500000CBF01230023DBB21A46009B934211D04B
:1055100000210198FFF762FE03468DF817309DF8D1
:105520001730002B08D1019B9B69002BB1D104E0FF
:1055300000BF02E000BF00E000BF9DF81730002B65
:1055400002D0019B00229A619DF81730184607B0DF
:105550005DF804FB00B587B00190019B1B680493C4
:1055600000210198FFF7C0FD03468DF817309DF824
:105570001730002B02D09DF8173046E0019B9B6945
:1055800019460498FFF751FA03468DF817309DF835
:105590001730002B34D1019BDB691B788DF80F305D
:1055A0009DF80F30002B03D104238DF817302AE02B
:1055B000019BDB690B331B7803F03F03DAB2019BDD
:1055C0009A71019BDB690B331B7803F00803002BF6
:1055D0000AD1019BD869019B20330B221946FFF7A2
:1055E000A6F90346002B0DD000210198FFF7F6FD28
:1055F00003468DF817309DF81730002BBED002E01F
:1056000000BF00E000BF9DF81730184607B05DF8F6
:1056100004FB00B585B00190019B1B68029301213A
:105620000198FFF79FFE03468DF80F309DF80F306D
:10563000002B1ED1019B9B6919460298FFF7F5F9D3
:1056400003468DF80F309DF80F30002B11D1019BD0
:10565000DB69202200211846FFF753F9019BD86926
:10566000019B20330B221946FFF72FF9029B0122E1
:10567000DA709DF80F30184605B05DF804FB00B5F0
:1056800087B001900091009B00225A72019B9B6998
:10569000002B53D000230493049B059326E0019B29
:1056A000DA69059B591C059113441B788DF80F305E
:1056B0009DF80F30202B00D118E09DF80F30052BFE
:1056C00002D1E5238DF80F30059B092B06D1049BF1
:1056D0005A1C0492009A13442E225A72049B5A1C9C
:1056E0000492009A13449DF80F205A72059B0A2BCE
:1056F000D5D9009A049B1344093300221A70019BE8
:10570000DB69DA7A009B1A72019BDB691C3318464D
:10571000FFF77BF80246009B1A60019BDB6916339A
:105720001846FFF772F80290029B9AB2009BDA804B
:10573000029B1B0C9AB2009B9A8000E000BF07B04E
:105740005DF804FB00B58BB001900091009B1B68D5
:105750000593019B203304930B2220210498FFF72B
:10576000D0F800230693069B079308230893079B12
:105770005A1C0792059A13441B788DF827309DF820
:105780002730202B40F290809DF827302F2B07D018
:105790009DF827305C2B10D102E0079B0133079363
:1057A000059A079B13441B782F2BF6D0059A079B6D
:1057B00013441B785C2BF0D077E09DF827302E2B1C
:1057C00003D0069A089B9A420DD3089B0B2B03D05B
:1057D0009DF827302E2B01D0062382E00823069364
:1057E0000B2308935FE09DF82730802B03D99DF8A9
:1057F00027309F2B07D99DF82730DF2B33D99DF811
:105800002730FC2B2FD8079B5A1C0792059A13446C
:105810001B788DF80F309DF80F303F2B03D99DF882
:105820000F307E2B07D99DF90F30002B08DA9DF839
:105830000F30FC2B04D8089B013B069A9A4201D3F7
:1058400006234EE0069B5A1C0692049A13449DF8C8
:1058500027201A70069B5A1C0692049A13449DF83E
:105860000F201A701FE09DF8273019461F48FFF7D8
:1058700080F80346002B01D0062332E09DF8273044
:10588000602B08D99DF827307A2B04D89DF8273053
:10589000203B8DF82730069B5A1C0692049A13442D
:1058A0009DF827201A7062E700BF059A079B1A44EB
:1058B000009B1A60069B002B01D1062311E0049B7C
:1058C0001B78E52B02D1049B05221A709DF8273026
:1058D000202B01D8042200E00022049B0B331A7015
:1058E000002318460BB05DF804FB00BFD48C030006
:1058F00000B587B001900091019B0493049B1B6845
:10590000039302E0009B01330093009B1B782F2B35
:10591000F8D0009B1B785C2BF4D0049B00229A608B
:10592000009B1B781F2B0BD8019B802283F82B2018
:1059300000210198FFF7D8FB03468DF817304DE0A2
:105940006B4619460198FFF7FDFE03468DF81730A8
:105950009DF81730002B3CD10198FFF7FBFD034663
:105960008DF81730019B93F82B308DF80B309DF894
:105970001730002B0DD09DF81730042B2BD19DF83C
:105980000B3003F00403002B25D105238DF81730CD
:1059900021E09DF80B3003F00403002B1DD1049B84
:1059A0009B7903F01003002B03D105238DF81730EA
:1059B00014E0039B03F13002019B1B69C3F308034E
:1059C000134419460398FFF71CFD0246049B9A6096
:1059D000B6E700BF02E000BF00E000BF9DF817304F
:1059E000184607B05DF804FB86B001904FF0FF3316
:1059F0000493019B1B68002B31D0019B1B6805930E
:105A000002E0059B01330593059B1B78202B03D9EE
:105A1000059B1B783A2BF4D1059B1B783A2B1CD1A4
:105A2000019B1B680393039B5A1C03921B78303B1A
:105A30000293029B092B0ED8039A059B9A420AD126
:105A4000029B002B07D1029B0493059B0133059316
:105A5000019B059A1A60049B02E000230493049BB7
:105A6000184606B07047000000B583B00190009161
:105A7000019B0022DA70019B4FF0FF32DA6200993D
:105A80000198FEF7D2FF0346002B01D0042338E033
:105A9000019B303303F5FF731846FEF79FFE034664
:105AA0001A464AF655239A4201D0032329E0019B66
:105AB00093F83030E92B09D0019B93F83030EB2B71
:105AC0001ED1019B93F83230902B19D1019B3033BA
:105AD00036331846FEF799FE034623F07F430B4A00
:105AE000934201D100230CE0019B3033523318461E
:105AF000FEF78BFE0346064A934201D1002300E0E5
:105B00000223184603B05DF804FB00BF4641540071
:105B10004641543300B597B00390029113468DF877
:105B20000730029B00221A600398FFF75DFF0F9079
:105B30000F9B002B01DA0B2331E2A44A0F9B52F892
:105B400023300E930E9B002B01D10C2327E2029BE6
:105B50000E9A1A609DF8073023F001038DF8073084
:105B60000E9B1B78002B1BD00E9B5B781846FEF714
:105B700025FC03468DF837309DF8373003F00103DC
:105B8000002B0DD19DF80730002B07D09DF8373042
:105B900003F00403002B01D00A2300E20023FEE1FE
:105BA0000E9B00221A700F9BDAB20E9B5A700E9B4E
:105BB0005B781846FEF738FB03468DF837309DF8C2
:105BC000373003F00103002B01D00323E7E19DF8F8
:105BD0000730002B07D09DF8373003F00403002B6B
:105BE00001D00A23DBE10023149314990E98FFF7E8
:105BF0003BFF03468DF857309DF85730022B49D1B3
:105C0000002310931EE00E9B03F13002109B1B013A
:105C100003F5DF7313440C930C9B04331B78002BA8
:105C200006D00C9B08331846FEF7EFFD024600E055
:105C30000022109B9B0016A90B4443F8442C109B98
:105C400001331093109B032BDDD900231093109B7D
:105C5000002B02D0109B013B1093109B9B0016AAB7
:105C6000134453F8443C1493149B002B05D014990F
:105C70000E98FFF7F9FE034600E003238DF8573036
:105C80009DF85730012B05D9109B01331093109BC1
:105C9000032BE2D99DF85730042B01D101237EE17B
:105CA0009DF85730012B01D90D2378E10E9B30333D
:105CB0000B331846FEF792FD0346B3F5007F01D083
:105CC0000D236CE10E9B303316331846FEF786FD2C
:105CD00003461393139B002B06D10E9B30332433C2
:105CE0001846FEF792FD13900E9B139A9A610E9B35
:105CF00093F840200E9B9A700E9B9B78012B05D049
:105D00000E9B9B78022B01D00D2348E10E9B9B78C4
:105D10001A46139B02FB03F313930E9B93F83D303B
:105D20009AB20E9B5A810E9B5B89002B08D00E9B6A
:105D30005B891A460E9B5B89013B1340002B01D007
:105D40000D232CE10E9B303311331846FEF746FD30
:105D500003461A460E9B1A810E9B1B8903F00F0304
:105D60009BB2002B01D00D2319E10E9B303313336E
:105D70001846FEF733FD03461293129B002B06D103
:105D80000E9B303320331846FEF73FFD12900E9BDA
:105D900030330E331846FEF721FD0346ADF82E30A2
:105DA000BDF82E30002B01D10D23F8E0BDF82E20D8
:105DB000139B13440E9A1289120992B213440A9348
:105DC000129A0A9B9A4203D20D23E8E0D0B5002034
:105DD000129A0A9BD31A0E9A5289B3FBF2F30993D3
:105DE000099B002B01D10D23D9E003238DF85730F7
:105DF000099B4FF6F572934202D802238DF8573073
:105E0000099B40F6F572934202D801238DF8573072
:105E1000099B9A1C0E9B5A610E9B149ADA61BDF87D
:105E20002E20149B1A440E9B1A62149A0A9B1A4441
:105E30000E9B9A629DF85730032B1ED10E9B303378
:105E40002A331846FEF7CAFC0346002B01D00D2367
:105E5000A5E00E9B1B89002B01D00D239FE00E9B1C
:105E600030332C331846FEF7D0FC02460E9B5A62A4
:105E70000E9B5B699B0011931FE00E9B1B89002BFF
:105E800001D10D238BE00E9B1A6A139B1A440E9BC3
:105E90005A629DF85730022B03D10E9B5B695B0061
:105EA0000AE00E9B5A6913465B0013445A080E9B86
:105EB0005B6903F00103134411930E9B9A69119BD4
:105EC00003F2FF135B0A9A4201D20D2367E00E9B97
:105ED0004FF0FF321A610E9B1A690E9BDA600E9B1F
:105EE00080221A719DF85730032B49D10E9B303315
:105EF00030331846FEF772FC0346012B40D1149B49
:105F0000013319460E98FEF790FD0346002B37D15A
:105F10000E9B00221A710E9B303303F5FF73184657
:105F2000FEF75CFC03461A464AF655239A4227D1EF
:105F30000E9B30331846FEF768FC03461A4A93421C
:105F40001ED10E9B303303F5F2731846FEF75DFC4D
:105F50000346164A934213D10E9B303303F5F47374
:105F60001846FEF752FC02460E9B1A610E9B303318
:105F700003F5F6731846FEF748FC02460E9BDA60FE
:105F80000E9B9DF857201A70094B1B8801339AB25B
:105F9000074B1A80064B1A880E9BDA80002318469E
:105FA00017B05DF804FB00BF52526141727241614B
:105FB000D4B5002000B585B001900091019B002B65
:105FC0001AD0019B1B68002B16D0019B1B681B7805
:105FD000002B11D0019B1B68DA88019B9B889A4299
:105FE0000AD1019B1B685B781846FEF7E7F9034668
:105FF00003F00103002B06D0009B00221A60092346
:106000008DF80F3006E0019B1A68009B1A60002390
:106010008DF80F309DF80F30184605B05DF804FB81
:1060200000B589B00390029113468DF80730029BAA
:10603000049304AB1846FFF7D7FC0790079B002B8F
:1060400001DA0B2329E0174A079B52F82330069305
:10605000069B002B02D0069B00221A70039B002B8C
:1060600002D0039B00221A70039A0E49079B41F845
:106070002320039B002B03D09DF80730012B01D078
:1060800000230AE003A902AB00221846FFF742FDF5
:1060900003468DF817309DF81730184609B05DF8A3
:1060A00004FB00BFD0B5002000B599B00390029169
:1060B00013468DF80730039B002B01D1092382E1A1
:1060C0009DF8073003F03F038DF807309DF8072057
:1060D00005A902AB1846FFF71DFD03468DF85F309A
:1060E0009DF85F30002B40F06581059B0693029A76
:1060F00006AB11461846FFF7FBFB03468DF85F30F1
:106100009DF85F30002B07D19DF843305BB2002B28
:1061100002DA06238DF85F309DF8073003F01C0388
:10612000002B7AD09DF85F30002B11D09DF85F30A6
:10613000042B06D106AB1846FFF76BFA03468DF821
:106140005F309DF8073043F008038DF8073012E008
:106150009DF81E3003F01103002B03D007238DF8A8
:106160005F3008E09DF8073003F00403002B02D0F5
:1061700008238DF85F309DF85F30002B6AD19DF8C1
:10618000073003F00803002B64D0914B14930D9B50
:106190000E3314991846FEF771FB0D9B16331499B4
:1061A0001846FEF76BFB0D9B0B3320221A70059BE4
:1061B0000D9A11461846FFF724F91390059B0D9987
:1061C00000221846FFF73BF90D9B1C3300211846AF
:1061D000FEF754FB059B0122DA70139B002B39D08C
:1061E000059BDB6A149306AB002213991846FEF751
:1061F00074FE03468DF85F309DF85F30002B29D187
:10620000059B14991846FEF710FC03468DF85F3085
:10621000059B139A013ADA601CE09DF85F30002B71
:1062200018D19DF81E3003F01003002B03D0042377
:106230008DF85F300EE09DF8073003F00203002B6D
:1062400008D09DF81E3003F00103002B02D0072375
:106250008DF85F309DF85F30002B12D19DF807302C
:1062600003F00803002B05D09DF8073043F04003EE
:106270008DF80730059BDA6A039B1A620D9A039B1F
:106280005A629DF85F30002B40F09480059B0D9A78
:1062900011461846FFF7B5F80246039B9A600D9B1E
:1062A0001C331846FEF7B1FA0246039BDA60059AE2
:1062B000039B1A60059BDA88039B9A80039B9DF8D9
:1062C00007201A74039B00225A74039B0022DA6190
:1062D000039B00225A61039B28334FF40072002174
:1062E0001846FEF70EFB9DF8073003F02003002B45
:1062F00060D0039BDB68002B5CD0039BDA68039BB8
:106300005A61059B5B895B021293039B9B68169302
:10631000039BDB68159316E0039B16991846FEF75E
:1063200041FC1690169B012B02D802238DF85F309A
:10633000169BB3F1FF3F02D101238DF85F30159A10
:10634000129BD31A15939DF85F30002B03D1159A39
:10635000129B9A42E0D8039B169A9A619DF85F308F
:10636000002B27D1159BC3F30803002B22D0059BDC
:1063700016991846FEF7FCFB1190119B002B03D1D8
:1063800002238DF85F3015E0159B5A0A119B1A44C1
:10639000039BDA61059B5878039B03F12801039B5B
:1063A000DA690123FEF734F80346002B02D00123FB
:1063B0008DF85F309DF85F30002B02D0039B0022E8
:1063C0001A609DF85F30184619B05DF804FB00BFF5
:1063D0000000214800B58DB0039002910192009316
:1063E000029B0793009B00221A60039B04AA11469C
:1063F0001846FFF7DFFD03468DF82F309DF82F304C
:10640000002B07D1039B5B7C8DF82F309DF82F303C
:10641000002B02D09DF82F303FE1039B1B7C03F043
:106420000203002B01D1072337E1039B5A69019B2B
:106430001A44039B5B699A4280F02181039B5B694C
:10644000DB4301931BE1039B5B69C3F30803002B50
:1064500040F0D780039B5B695B0A049A5289013A3A
:1064600013400693069B002B37D1039B5B69002BDF
:106470000CD1039B9B680A930A9B002B0ED1039BB4
:1064800000211846FEF794FD0A9007E0039A039B4B
:106490009B6919461046FEF78BFD0A900A9B002B5C
:1064A00000F0F2800A9B012B04D1039B02225A7454
:1064B0000223F2E00A9BB3F1FF3F04D1039B0122C8
:1064C0005A740123E9E0039B0A9A9A61039B9B6833
:1064D000002B02D1039B0A9A9A60039B1B7C5BB240
:1064E000002B18DA049B5878039B03F12801039BC7
:1064F000DA690123FEF71AF80346002B04D0039B48
:1065000001225A740123C8E0039B1B7C03F07F0324
:10651000DAB2039B1A74049A039B9B6919461046CE
:10652000FEF726FB0590059B002B04D1039B02225E
:106530005A740223B1E0059A069B13440593019B0C
:106540005B0A0893089B002B3CD0069A089B1344D7
:10655000049A5289934205D9049B5B891A46069B8B
:10656000D31A0893049B5878089B059A0799FDF75E
:10657000DDFF0346002B04D0039B01225A74012344
:106580008BE0039BDA69059BD31A089A9A4215D9C6
:10659000039B03F12800039BDA69059BD31A5B0276
:1065A000079A13444FF400721946FEF78EF9039BC5
:1065B0001B7C03F07F03DAB2039B1A74089B5B0217
:1065C00009933FE0039BDB69059A9A4216D0039B2F
:1065D0005A69039BDB689A4210D2049B5878039B4C
:1065E00003F128010123059AFDF712FF0346002B52
:1065F00004D0039B01225A7401234EE0039B059AA9
:10660000DA61039B5B69C3F30803C3F50073099365
:10661000099A019B9A4201D9019B0993039B03F1BB
:106620002802039B5B69C3F308031344099A079983
:106630001846FEF74AF9039B1B7C63F07F03DAB22E
:10664000039B1A74079A099B13440793039B5A6987
:10665000099B1A44039B5A61039BDA68039B5B699D
:106660009A4238BF1A46039BDA60009B1A68099B5E
:106670001A44009B1A60019A099BD31A0193019B4B
:10668000002B7FF4E0AE00E000BF039B1B7C43F0D7
:106690004003DAB2039B1A74002318460DB05DF86C
:1066A00004FB000000B587B00190019B02AA1146CF
:1066B0001846FFF77FFC03468DF817309DF817301A
:1066C000002B6AD1019B1B7C03F04003002B64D09C
:1066D000019B1B7C5BB2002B15DA029B5878019B57
:1066E00003F12801019BDA690123FDF71FFF03462F
:1066F000002B01D0012352E0019B1B7C03F07F03A0
:10670000DAB2019B1A74284B0493029A019B1B6A0C
:1067100019461046FEF789F903468DF817309DF8A3
:106720001730002B39D1019B5B6A0393039B0B331A
:106730001A78039B0B3342F02002D2B21A70019BED
:106740001868019B9B681A460399FEF778FE039B25
:1067500003F11C02019BDB6819461046FEF78EF818
:10676000039B163304991846FEF788F8039B1233EF
:1067700000211846FEF767F8029B0122DA70029B9F
:106780001846FEF783F903468DF81730019B1B7CF2
:1067900023F04003DAB2019B1A749DF817301846B3
:1067A00007B05DF804FB00BF0000214800B585B0CC
:1067B00001900198FFF776FF03468DF80F309DF8A2
:1067C0000F30002B0FD1019B02AA11461846FFF78C
:1067D000F1FB03468DF80F309DF80F30002B02D1EE
:1067E000019B00221A609DF80F30184605B05DF835
:1067F00004FB00B587B001900091019B002B01D1F3
:10680000092356E0019B049303A96B460022184616
:10681000FFF780F903468DF817309DF81730002BED
:106820003ED1039A049B1A60009B19460198FFF71A
:106830005FF803468DF817309DF81730002B28D1EC
:10684000019B93F82B305BB2002B13DB049B9B79ED
:1068500003F01003002B0AD0039A019BDB69194651
:106860001046FEF7CEFD0246049B9A6002E0052327
:106870008DF817309DF81730002B0AD1039BDA886A
:10688000049B9A8000210198FEF72EFC03468DF8A8
:1068900017309DF81730042B02D105238DF81730DF
:1068A0009DF81730002B02D0049B00221A609DF83F
:1068B0001730184607B05DF804FB00B585B00190AD
:1068C0000091019B02AA11461846FFF773FB03468D
:1068D0008DF80F309DF80F30002B2ED1009B002B30
:1068E00007D100210198FEF7FFFB03468DF80F301A
:1068F00023E000210198FEF7C1FD03468DF80F301B
:106900009DF80F30042B02D100238DF80F309DF835
:106910000F30002B11D100990198FEF7B0FE002135
:106920000198FEF75BFC03468DF80F309DF80F30A1
:10693000042B02D100238DF80F309DF80F3018463C
:1069400005B05DF804FB53EA020C61D02DE9F04B71
:10695000B3FA83F51E0007BFB2FA82F502FA05F416
:1069600003FA05F41646C5F120051EBF22FA05F705
:106970003C43203556EA044C4FEA144418BF013416
:10698000A3464FF00009C846904271EB030C39D37F
:10699000094207BFB0FA80F700FA07F6B1FA81F7AB
:1069A00001FA07F6C7F120071EBF20FA07FC46EAE6
:1069B0000C062037B6FBFBFC7F1B103F07F01F04C3
:1069C000C4F120060CFA04F42CFA06F644BF34464F
:1069D0000026202FA4BF2646002454EA060C08BF38
:1069E000012418EB040849EB0609A4FB027CC01B38
:1069F00006FB02CC04FB03CC71EB0C01904271EB63
:106A0000030CC5D20B46024649464046BDE8F08B12
:106A1000B2FBF3F27F2805D8034B185C034B5B5C99
:106A20001840704700207047248D0300A48D030098
:106A3000A0F16103192B98BF20387047A0F14103E2
:106A4000192B98BF203070477F2805D8034B185C5E
:106A5000034B5B5C1840704700207047248D030097
:106A6000A48D0300A0F16103192B98BF2038704753
:106A7000A0F14103192B98BF203070477F299ABF9E
:106A8000017001206FF02E0070475AB10A787F2AFA
:106A90000AD800B10260002119605960501A18BF6D
:106AA00001207047002070476FF02E00704710B52E
:106AB00004460846A2684AB12368616803F1010CE4
:106AC0008C4508BF00208B4208D2D054E3682BB11C
:106AD00021686268914201D22146984723680133B8
:106AE000236010BD70B54C1E09D41646C5B22946A8
:106AF0003046FFF7DCFF013CB4F1FF3FF7D170BD3A
:106B000010F0100F08D108B510F4007F14BF30202A
:106B10002020FFF7E7FF08BD7047000008B5034BD2
:106B20005B689B681B68984708BD00BF902B0020DE
:106B300008B50921FFF7F2FF08BD0EB400B586B015
:106B400007AA52F8041B05920390002304936FF0E8
:106B50000043029301A800F0A3F806B05DF804EB2F
:106B600003B07047037853B159B10144034613F899
:106B7000012F12B18B42FAD10B46181A7047034607
:106B8000FBE70346F9E7844640EA010313F0030FED
:106B900018D18446202A0BD32DE9F007B1E8F80775
:106BA000A0E8F807A2F12002202AF7D2BDE8F007FA
:106BB000042A07D351F8043B40F8043BA2F1040235
:106BC000042AF7D2002A05D011F8013B00F8013B56
:106BD000013AF9D1604670478446002A2DD010F062
:106BE000030F04D000F8011B013A26D0F7E7C9B221
:106BF00041EA012141EA0141202A12D3A2F12002F7
:106C00002DE9F0030B460C460D460E460F4688460E
:106C10008946A0E8FA03203AFBD2BDE8F00320320F
:106C20000BD0042A05D340F8041B043A05D0042AEB
:106C3000F9D200F8011B013AFBD16046704700F120
:106C4000010110F0030F11D010F8012B002A23D0FE
:106C500010F0030F0AD010F8012B002A1CD010F0FE
:106C6000030F03D010F8012B002A15D02DE9700076
:106C70004FF001324FF0803350F8044BA4EB020583
:106C800025EA04051D4000D1F6E7A0F1040070BC20
:106C900010F8012B002AFBD1A0EB01007047000087
:106CA0002DE9F04F89B007460392002303600C469C
:106CB00014F8011B002900F0FC82DFF818B5EBE2A4
:106CC000002507E05E2868D145F4805501E045F0D5
:106CD00040051C46234613F8010B3028F2D81F2824
:106CE00037D9A0F12002102A33D801A151F822F09F
:106CF000CF6C0300536D0300536D0300356D03002B
:106D0000536D0300536D0300536D03003B6D03008F
:106D1000536D0300536D0300536D0300416D030079
:106D2000536D0300476D0300536D0300536D030063
:106D30004D6D030045F08005CBE745F40045C8E7FD
:106D400045F02005C5E745F01005C2E745F400759C
:106D5000BFE72A2821D1039A111D0391D2F800A080
:106D6000BAF1000FBCBFCAF1000A45F0100518784F
:106D7000A31C2AEAEA7A2E2826D00021742847D0BC
:106D80007A2845D06C2800F0A8804C2800F0AB8011
:106D9000682800F0B8801C463DE0A0F13002D2B275
:106DA000092A88BF4FF0000AE3D84FF0000A0AEB27
:106DB0008A0A303800EB4A0A13F8010BA0F13002BE
:106DC000D2B2092AF3D9D4E718782A280AD1039A2B
:106DD000111D03911168587802330029CEDB45F468
:106DE0008075CBE70133A0F13002D2B2092A88BF07
:106DF0000021F4D8002101EB8101303800EB410182
:106E000013F8010BA0F13002D2B2092AF3D9E4E75A
:106E10001C4614F8010B002800F05782A0F125034E
:106E2000DBB2532B62D8A0F12503532B5ED8DFE8E9
:106E300013F076005D005D005D005D005D005D00AB
:106E40005D005D005D005D005D005D005D005D005A
:106E50005D005D005D005D005D005D005D005D004A
:106E60005D005D005D005D005D005D005D005D003A
:106E70005D005D005D005D005D005D005D005D002A
:106E80005D005D005D005D005D005D005D005D001A
:106E90005D005D005D005D00EC005D005D005D007B
:106EA0005D005D005D005D005D005D005D007B00DC
:106EB00021015D005D005D005D0021015D005D0060
:106EC0005D005D0095000F01D2005D005D00A60031
:106ED0005D001A015D005D00EE001C4614F8010B18
:106EE00045F0010597E745F001051C46B54B1E68C6
:106EF000002E00F0CE8103AB0193009153462A4649
:106F00003946B047C5E11878682803D05C1C45F0C5
:106F1000040580E745F008059C1C58787BE725218F
:106F20003846FFF7C4FDB4E1039B1A1D03921E7897
:106F30000AF1FF3A3A4651462846FFF7E1FD31464D
:106F40003846FFF7B4FDA94619F0100F00F0A181F3
:106F50003A4651462020FFF7C5FD9AE115F0080F8B
:106F600006D03A68039B191D03911B681A7090E1C3
:106F7000039B1A1D03921B683A681A6089E1039B00
:106F80001A1D0392D3F800808F4BB8F1000F08BF91
:106F90009846464625F4007915F4807F16D0404681
:106FA000FFF7E0FD0546AAEB050A3A46514648467A
:106FB000FFF7A6FD002DC7D016F8011B3846FFF7D6
:106FC00076FDA8EB0603EB42F6D1BDE74046FFF79E
:106FD00036FE0546E7E7039B1A1D03921B6815F072
:106FE000800F0CBF0026232645F4807508211A4621
:106FF000002B00F02A8105AB4FF0000805F4005C7F
:10700000A64660468C460146D2E045F4005515F090
:10701000800F1BD043F2780643F25803782818BF3C
:107020001E4615F4807F01D025F4007515F4804FBD
:1070300032D0039B1A1D03921B6815F0040F1FD05A
:107040001BB2002B20DA5B422D262DE00026E8E75C
:1070500015F0800F0CBF0026302615F4807FE5D098
:1070600025F40075E2E715F4807F07D025F400755C
:107070000026DBE745F480450026D7E70026D5E764
:1070800015F0080FDDD0DBB215F0200F61D115F03F
:10709000400F18BF202607E0039B1A1D03921B68B0
:1070A00015F0040F50D09BB215F4807F14BF25F467
:1070B000007501215838202800F2AF8001A252F853
:1070C00020F000BFEF6F03001B7203001B72030070
:1070D0001B7203001B7203001B7203001B72030070
:1070E0001B7203001B7203001B7203001B72030060
:1070F0001B7203007F7103001B7203001B720300ED
:107100001B7203001B7203007F7103001B720300DC
:107110001B7203001B7203001B7203001B7203002F
:1071200057710300EF6F03001B7203001B72030013
:107130001B7203001B7203007F7103001B720300AC
:107140001B720300EF6F030015F0080FACD0DBB229
:10715000AAE72B26A8E71A464FF00008002B5ED0BE
:1071600005A84FF0000803F00703303300F8013B97
:1071700008F10108D2081346002AF4D14FE018465E
:107180004FF00008002B4AD04FF0000805F4004EE5
:107190004FF02C0973468E4619462FE002F00F007F
:1071A0000A4C205C03F8010B08F10108120906D013
:1071B0000029F3D002F00F00054C205CF2E7744682
:1071C00061462CE0D8B50020788F0300588F03006B
:1071D000688F0300CDCCCCCC08AB03EB080CABFB29
:1071E0000032D20802EB8203A0EB430330330CF8E9
:1071F0000C3C08F1010809280DD910460029EBD0F4
:1072000008F00303032BE7D108AB434403F80C9CBD
:1072100008F10108E0E7714601E04FF00008A1EB3A
:10722000080121EAE179AAEB090AAAEB080AFF2E74
:107230000ED9AAF1020AC6F307213846FFF737FC38
:10724000F1B23846FFF733FC04E04FF00008E6E700
:10725000002E3DD13A4651462846FFF751FC3A46AA
:1072600049463020FFF73EFCB8F1000F0EDD0DF16E
:10727000140908F1FF38C84498F80010464638460B
:10728000FFF715FCC14508F1FF38F5D115F0100FD7
:1072900009D114F8011B61B125293FF411AD38461D
:1072A000FFF705FCF5E73A4651462020FFF71AFCA8
:1072B000EFE7BB682BB13A6879688A423CBF00218E
:1072C0009954386809B0BDE8F08F4FF0FF30F9E706
:0872D0000AF1FF3AB4E700BF28
:0872D800FDBD020000000000F2
:1072E0003526030000000000E9F60200000000005F
:1072F0009D30030054A90020711E030074A90020D2
:10730000352403000000000037360300602B002006
:107310009733030068A90020C5F9020000000000AF
:0873200025BE02000000000080
:10732800E93E030000000000C13F03000000000028
:10733800B02C0020E82B0020F02B0020F02B0020A0
:047348001800000029
:10734C008080030000000000148103000000000096
:10735C0050810300000000002483030000000000A3
:10736C00E4810300000000007C82030000000000A8
:10737C008074030000000303F47503000000000098
:10738C00EC76030000000000D8870300000000002A
:10739C00148003000000000080860300000003033B
:1073AC004088030000000303F4880300000003037B
:1073BC00148C030000000303D478030000000000C9
:0873CC007879030000000000C5
:1073D400F47303000000000008740300D82A00209E
:1073E400E87503000000000018740300E02A002080
:1073F400B9640200EB640200E16402000338FDD8C2
:10740400704700007274745F6C6F675F6261636BD6
:10741400656E6400756172745F6C6F675F6261634F
:107424006B656E6400000000443A5C53444B313792
:107434005F454D475C636F6D706F6E656E74735C12
:107444006C69627261726965735C6C6F675C73729C
:10745400635C6E72665F6C6F675F64656661756CB2
:10746400745F6261636B656E64732E630000000079
:10747400B82C00207F000000382D002061707000BF
:10748400443A5C53444B31375F454D475C636F6D01
:10749400706F6E656E74735C6C696272617269653B
:1074A400735C6C6F675C7372635C6E72665F6C6F47
:1074B400675F66726F6E74656E642E630000000011
:1074C4004261636B656E647320666C757368656492
:1074D400000000006572726F720000007761726EC6
:1074E400696E6700696E666F00000000646562750E
:1074F400670000001B5B306D000000001B5B313B2C
:1075040033306D001B5B313B33316D001B5B313B12
:1075140033326D001B5B313B33336D001B5B313BFE
:1075240033346D001B5B313B33356D001B5B313BEA
:1075340033366D001B5B313B33376D0025734C6F65
:1075440067732064726F7070656420282564292530
:10755400730D0A00257300003C25733E2025733A01
:10756400200000000D0A00002025303278000000C1
:10757400202020007C000000256300002000000083
:10758400443A5C53444B31375F454D475C636F6D00
:10759400706F6E656E74735C6C696272617269653A
:1075A400735C6C6F675C7372635C6E72665F6C6F46
:1075B400675F6261636B656E645F756172742E638D
:1075C40000000000FFFFFFFFFFFFFFFFFFFFFFFFC3
:1075D400FFFFFFFF00000000000000000000D601D4
:1075E40006010000697702009D770200917702008E
:1075F4006170705F627574746F6E0000443A5C531E
:10760400444B31375F454D475C636F6D706F6E65FA
:107614006E74735C6C69627261726965735C6275C5
:1076240074746F6E5C6170705F627574746F6E2ECB
:1076340063000000534F46544445564943453A209D
:10764400415353455254494F4E204641494C4544B9
:1076540000000000534F46544445564943453A20E0
:10766400494E56414C4944204D454D4F52592041B5
:107674004343455353000000415353455254494F2B
:107684004E204641494C45442061742025733A25D7
:10769400750000004552524F52202575205B25731A
:1076A4005D2061742025733A25750D0A50432061CD
:1076B400743A20307825303878000000456E642014
:1076C4006F66206572726F72207265706F727400DB
:1076D400554E4B4E4F574E204641554C54206174E5
:1076E40020307825303858006170705F74696D659A
:1076F40072000000443A5C53444B31375F454D47B8
:107704005C636F6D706F6E656E74735C6C696272CE
:1077140061726965735C74696D65725C6170705FD8
:1077240074696D6572322E6300000000010006006A
:10773400443A5C53444B31375F454D475C636F6D4E
:10774400706F6E656E74735C6C6962726172696588
:10775400735C7574696C5C6170705F7574696C5F7F
:10776400706C6174666F726D2E630000443A5C53F2
:10777400444B31375F454D475C636F6D706F6E6589
:107784006E74735C6C69627261726965735C626168
:107794006C6C6F635C6E72665F62616C6C6F632E9F
:1077A40063000000443A5C53444B31375F454D4716
:1077B4005C65787465726E616C5C667072696E7417
:1077C400665C6E72665F667072696E74662E6300C4
:1077D400443A5C53444B31375F454D475C6578749C
:1077E40065726E616C5C667072696E74665C6E72F2
:1077F400665F667072696E74665F666F726D6174DF
:107804002E63000030313233343536373839414253
:1078140043444546443A5C53444B31375F454D47F6
:107824005C636F6D706F6E656E74735C6C696272AD
:1078340061726965735C6D656D6F626A5C6E7266B8
:107844005F6D656D6F626A2E63000000643A5C735D
:10785400646B31375F656D675C636F6D706F6E6508
:107864006E74735C6C69627261726965735C65786D
:10787400706572696D656E74616C5F73656374695C
:107884006F6E5F766172735C6E72665F736563744C
:10789400696F6E5F697465722E680000643A5C7388
:1078A400646B31375F656D675C636F6D706F6E65B8
:1078B4006E74735C6C69627261726965735C6D7518
:1078C4007465785C6E72665F6D74782E6800000073
:1078D4007077725F6D676D7400000000443A5C530A
:1078E400444B31375F454D475C636F6D706F6E6518
:1078F4006E74735C6C69627261726965735C7077D3
:10790400725F6D676D745C6E72665F7077725F6DC7
:10791400676D742E6300000020730300207303005E
:1079240004000000443A5C53444B31375F454D47F3
:107934005C636F6D706F6E656E74735C6C6962729C
:1079440061726965735C6578706572696D656E7482
:10795400616C5F73656374696F6E5F766172735C8B
:107964006E72665F73656374696F6E5F6974657266
:107974002E630000736F72746C69737400000000EE
:10798400443A5C53444B31375F454D475C636F6DFC
:10799400706F6E656E74735C6C6962726172696536
:1079A400735C736F72746C6973745C6E72665F730C
:1079B4006F72746C6973742E63000000556E6B6E85
:1079C4006F776E206572726F7220636F646500005A
:1079D4004E52465F53554343455353004E52465F00
:1079E4004552524F525F5356435F48414E444C45B3
:1079F400525F4D495353494E470000004E52465F73
:107A04004552524F525F534F46544445564943459D
:107A14005F4E4F545F454E41424C454400000000C8
:107A24004E52465F4552524F525F494E5445524E54
:107A3400414C00004E52465F4552524F525F4E4FEA
:107A44005F4D454D000000004E52465F4552524F77
:107A5400525F4E4F545F464F554E44004E52465F60
:107A64004552524F525F4E4F545F535550504F52F0
:107A7400544544004E52465F4552524F525F494E60
:107A840056414C49445F504152414D004E52465F6D
:107A94004552524F525F494E56414C49445F5354EC
:107AA400415445004E52465F4552524F525F494E33
:107AB40056414C49445F4C454E4754480000000031
:107AC4004E52465F4552524F525F494E56414C49C1
:107AD400445F464C414753004E52465F4552524F15
:107AE400525F494E56414C49445F44415441000061
:107AF4004E52465F4552524F525F444154415F5388
:107B0400495A45004E52465F4552524F525F5449BE
:107B14004D454F55540000004E52465F4552524F5A
:107B2400525F4E554C4C00004E52465F4552524FE8
:107B3400525F464F5242494444454E004E52465FBE
:107B44004552524F525F494E56414C49445F41445D
:107B5400445200004E52465F4552524F525F4255C6
:107B6400535900004E52465F4552524F525F434FA5
:107B74004E4E5F434F554E54000000004E52465F38
:107B84004552524F525F5245534F5552434553004D
:107B94004E52465F4552524F525F4D4F44554C45ED
:107BA4005F4E4F545F494E495449414C495A4544EC
:107BB400000000004E52465F4552524F525F4D55F1
:107BC4005445585F494E49545F4641494C45440029
:107BD4004E52465F4552524F525F4D555445585F81
:107BE4004C4F434B5F4641494C4544004E52465F1F
